:020000040000FA
:10000000F80601204DAB00006FB8050021AB0000E1
:1000100021AB000021AB000021AB000021AB0000B0
:1000200000000000000000000000000051A30000DC
:1000300021AB000000000000F5A2000021AB000091
:10004000D1A30000D1A30000D1A30000D1A30000E0
:10005000D1A30000D1A30000D1A30000D1A30000D0
:10006000D1A30000D1A30000D1A30000D1A30000C0
:10007000D1A30000D1A30000D1A30000D1A30000B0
:10008000D1A30000D1A30000D1A30000D1A30000A0
:10009000D1A30000D1A30000D1A30000D1A3000090
:1000A000D1A30000D1A30000D1A30000D1A3000080
:1000B000D1A30000D1A30000D1A30000D1A3000070
:1000C000D1A30000D1A30000D1A30000D1A3000060
:1000D000D1A30000D1A30000D1A30000D1A3000050
:1000E000D1A30000D1A30000D1A30000D1A3000040
:1000F000D1A30000D1A30000D1A30000D1A3000030
:10010000D1A30000D1A30000D1A30000D1A300001F
:10011000D1A30000D1A30000D1A30000D1A300000F
:10012000D1A30000D1A30000D1A30000D1A30000FF
:10013000D1A30000D1A30000D1A30000D1A30000EF
:10014000D1A30000D1A30000D1A30000D1A30000DF
:10015000D1A30000FFFFFFFF81F0004102E000BFDC
:1001600083F0004330B54FEA41044FEA430594EA77
:10017000050F08BF90EA020F1FBF54EA000C55EAB2
:10018000020C7FEA645C7FEA655C00F0E2804FEA83
:100190005454D4EB5555B8BF6D420CDD2C4480EA65
:1001A000020281EA030382EA000083EA010180EA95
:1001B000020281EA0303362D88BF30BD11F0004FE3
:1001C0004FEA01314FF4801C4CEA113102D0404219
:1001D00061EB410113F0004F4FEA03334CEA133354
:1001E00002D0524263EB430394EA050F00F0A7806C
:1001F000A4F10104D5F1200E0DDB02FA0EFC22FA67
:1002000005F2801841F1000103FA0EF2801843FA5A
:1002100005F359410EE0A5F120050EF1200E012A4B
:1002200003FA0EFC28BF4CF0020C43FA05F3C01889
:1002300051EBE37101F0004507D54FF0000EDCF102
:10024000000C7EEB00006EEB0101B1F5801F1BD3AB
:10025000B1F5001F0CD349085FEA30004FEA3C0CAF
:1002600004F101044FEA445212F5800F80F09A80A5
:10027000BCF1004F08BF5FEA500C50F1000041EBA9
:10028000045141EA050130BD5FEA4C0C404141EBAD
:100290000101013C28BFB1F5801FE9D291F0000FA8
:1002A00004BF01460020B1FA81F308BF2033A3F157
:1002B0000B03B3F120020CDA0C3208DD02F1140C4E
:1002C000C2F10C0201FA0CF021FA02F10CE002F189
:1002D0001402D8BFC2F1200C01FA02F120FA0CFC82
:1002E000DCBF41EA0C019040E41AA2BF01EB0451CB
:1002F000294330BD6FEA04041F3C1CDA0C340EDCC9
:1003000004F11404C4F1200220FA04F001FA02F30B
:1003100040EA030021FA04F345EA030130BDC4F1C9
:100320000C04C4F1200220FA02F001FA04F340EABE
:100330000300294630BD21FA04F0294630BD94F06F
:10034000000F83F4801306BF81F480110134013D56
:100350004EE77FEA645C18BF7FEA655C29D094EAC7
:10036000050F08BF90EA020F05D054EA000C04BF45
:100370001946104630BD91EA030F1EBF0021002030
:1003800030BD5FEA545C05D14000494128BF41F0CF
:10039000004130BD14F580043CBF01F5801130BD33
:1003A00001F0004545F0FE4141F470014FF00000BE
:1003B00030BD7FEA645C1ABF194610467FEA655C6F
:1003C0001CBF0B46024650EA013406BF52EA033511
:1003D00091EA030F41F4002130BD00BF90F0000FFF
:1003E00004BF0021704730B54FF4806404F132043B
:1003F0004FF000054FF0000150E700BF90F0000FF4
:1004000004BF0021704730B54FF4806404F132041A
:1004100010F0004548BF40424FF000013EE700BFEA
:1004200042004FEAE2014FEA31014FEA02701FBF7A
:1004300012F07F4393F07F4F81F06051704732F0AC
:100440007F4208BF704793F07F4F04BF41F4002103
:10045000704730B54FF4607401F0004521F0004161
:100460001CE700BF50EA010208BF704730B54FF0EB
:1004700000050AE050EA010208BF704730B511F0EC
:10048000004502D5404261EB41014FF4806404F124
:1004900032045FEA915C3FF4D8AE4FF003025FEAAA
:1004A000DC0C18BF03325FEADC0C18BF033202EB2E
:1004B000DC02C2F1200300FA03FC20FA02F001FA88
:1004C00003FE40EA0E0021FA02F11444BDE600BF2B
:1004D00070B54FF0FF0C4CF4E06C1CEA11541DBFDA
:1004E0001CEA135594EA0C0F95EA0C0F00F0DEF8A5
:1004F0002C4481EA030621EA4C5123EA4C5350EA8A
:10050000013518BF52EA033541F4801143F48013DA
:1005100038D0A0FB02CE4FF00005E1FB02E506F06B
:100520000042E0FB03E54FF00006E1FB03569CF0C0
:10053000000F18BF4EF0010EA4F1FF04B6F5007FC6
:1005400064F5407404D25FEA4E0E6D4146EB060638
:1005500042EAC62141EA55514FEAC52040EA5E50C1
:100560004FEACE2EB4F1FD0C88BFBCF5E06F1ED86B
:10057000BEF1004F08BF5FEA500E50F1000041EBA2
:10058000045170BD06F0004646EA010140EA02004F
:1005900081EA0301B4EB5C04C2BFD4EB0C0541EA71
:1005A000045170BD41F480114FF0000E013C00F386
:1005B000AB8014F1360FDEBF002001F0004170BDAA
:1005C000C4F10004203C35DA0C341BDC04F11404C3
:1005D000C4F1200500FA05F320FA04F001FA05F24F
:1005E00040EA020001F0004221F0004110EBD3701C
:1005F00021FA04F642EB06015EEA430E08BF20EA48
:10060000D37070BDC4F10C04C4F1200500FA04F3EA
:1006100020FA05F001FA04F240EA020001F000417C
:1006200010EBD37041F100015EEA430E08BF20EAEF
:10063000D37070BDC4F1200500FA05F24EEA020E37
:1006400020FA04F301FA05F243EA020321FA04F066
:1006500001F0004121FA04F220EA020000EBD3701D
:100660005EEA430E08BF20EAD37070BD94F0000F1D
:100670000FD101F00046400041EB010111F4801F51
:1006800008BF013CF7D041EA060195F0000F18BF02
:10069000704703F00046520043EB030313F4801F3E
:1006A00008BF013DF7D043EA0603704794EA0C0FF8
:1006B0000CEA135518BF95EA0C0F0CD050EA41060E
:1006C00018BF52EA4306D1D181EA030101F000418B
:1006D0004FF0000070BD50EA410606BF10461946B3
:1006E00052EA430619D094EA0C0F02D150EA0136BF
:1006F00013D195EA0C0F05D152EA03361CBF104600
:1007000019460AD181EA030101F0004141F0FE419E
:1007100041F470014FF0000070BD41F0FE4141F422
:10072000780170BD70B54FF0FF0C4CF4E06C1CEA22
:1007300011541DBF1CEA135594EA0C0F95EA0C0FD7
:1007400000F0A7F8A4EB050481EA030E52EA033592
:100750004FEA013100F088804FEA03334FF08055B3
:1007600045EA131343EA12634FEA022245EA1115E0
:1007700045EA10654FEA00260EF000419D4208BF91
:10078000964244F1FD0404F5407402D25B084FEA3E
:100790003202B61A65EB03055B084FEA32024FF4EA
:1007A00080104FF4002CB6EB020E75EB030E22BF47
:1007B000B61A754640EA0C005B084FEA3202B6EB07
:1007C000020E75EB030E22BFB61A754640EA5C00B6
:1007D0005B084FEA3202B6EB020E75EB030E22BF46
:1007E000B61A754640EA9C005B084FEA3202B6EB47
:1007F000020E75EB030E22BFB61A754640EADC0006
:1008000055EA060E18D04FEA051545EA16754FEA67
:1008100006164FEAC30343EA52734FEAC2025FEA85
:100820001C1CC0D111F4801F0BD141EA00014FF014
:1008300000004FF0004CB6E711F4801F04BF0143E5
:100840000020B4F1FD0C88BFBCF5E06F3FF6AFAE01
:10085000B5EB030C04BFB6EB020C5FEA500C50F191
:10086000000041EB045170BD0EF0004E4EEA113114
:1008700014EB5C04C2BFD4EB0C0541EA045170BD1B
:1008800041F480114FF0000E013C90E645EA060E5F
:100890008DE60CEA135594EA0C0F08BF95EA0C0F8D
:1008A0003FF43BAF94EA0C0F0AD150EA01347FF4D5
:1008B00034AF95EA0C0F7FF425AF104619462CE7AC
:1008C00095EA0C0F06D152EA03353FF4FDAE10460F
:1008D000194622E750EA410618BF52EA43067FF460
:1008E000C5AE50EA41047FF40DAF52EA43057FF4F0
:1008F000EBAE12E74FF0FF3C06E000BF4FF0010CFB
:1009000002E000BF4FF0010C4DF804CD4FEA410C5E
:100910007FEA6C5C4FEA430C18BF7FEA6C5C1BD02B
:1009200001B050EA410C0CBF52EA430C91EA030FAC
:1009300002BF90EA020F0020704710F1000F91EA09
:10094000030F58BF994208BF90422CBFD8176FEAD7
:10095000E37040F0010070474FEA410C7FEA6C5CA5
:1009600002D150EA013C07D14FEA430C7FEA6C5CAC
:10097000D6D152EA033CD3D05DF8040B704700BFD8
:100980008446104662468C461946634600E000BF26
:1009900001B5FFF7B7FF002848BF10F1000F01BDF8
:1009A0004DF808EDFFF7F4FF0CBF012000205DF8C3
:1009B00008FB00BF4DF808EDFFF7EAFF34BF012048
:1009C00000205DF808FB00BF4DF808EDFFF7E0FFE1
:1009D00094BF012000205DF808FB00BF4DF808ED32
:1009E000FFF7CEFF94BF012000205DF808FB00BF99
:1009F0004DF808EDFFF7C4FF34BF012000205DF87B
:100A000008FB00BF4A0011D212F5001211D20DD519
:100A10006FF47873B3EB62520ED44FEAC12343F004
:100A2000004343EA505323FA02F070474FF00000AE
:100A3000704750EA013002D14FF0FF3070474FF05D
:100A4000000070474FEA4102B2F1E04324BFB3F522
:100A5000001CDCF1FE5C0DD901F0004C4FEAC00235
:100A60004CEA5070B2F1004F40EB830008BF20F019
:100A70000100704711F0804F21D113F13872BCBFD3
:100A800001F00040704741F480114FEA5252C2F128
:100A90001802C2F1200C10FA0CF320FA02F018BF71
:100AA00040F001004FEAC1234FEAD32303FA0CFCC4
:100AB00040EA0C0023FA02F34FEA4303CCE77FEA53
:100AC000625307D150EA01331EBF4FF0FE4040F49D
:100AD0004000704701F0004040F0FE4040F400004C
:100AE000704700BF7BB972B90029BEBF00204FF02C
:100AF000004106E008BF00281CBF6FF000414FF026
:100B0000FF3000F075B8ADF1080C6DE904CE002996
:100B100009DB002B1ADB01F0B4F8DDF804E0DDE9B5
:100B2000022304B07047404261EB4101002B1BDB04
:100B300001F0A7F8DDF804E0DDE9022304B040424B
:100B400061EB4101524263EB43037047524263EB56
:100B5000430301F096F8DDF804E0DDE9022304B078
:100B6000404261EB41017047524263EB430301F0A5
:100B700088F8DDF804E0DDE9022304B0524263EBBB
:100B80004303704753B94AB9002908BF00281CBF66
:100B90004FF0FF314FF0FF3000F02AB8ADF1080CF4
:100BA0006DE904CE01F06DF8DDF804E0DDE9022323
:100BB00004B07047D0B500220B4B06460F46FFF736
:100BC00087FCFFF71FFF0446FFF708FC0022074BD6
:100BD000FFF77EFC02460B4630463946FFF7C0FA67
:100BE000FFF710FF2146D0BD0000F03D0000F041AE
:100BF000704700BF844641EA000313F0030349D164
:100C0000403A23D30B6803604B6843608B68836072
:100C1000CB68C3600B6903614B6943618B69836176
:100C2000CB69C3610B6A03624B6A43628B6A83625E
:100C3000CB6AC3620B6B03634B6B43638B6B836346
:100C4000CB6BC36340304031403ADBD230320BD300
:100C50000B6803604B6843608B688360CB68C3603C
:100C600010301031103AF3D20C3205D351F8043B56
:100C700040F8043B043AF9D2043208D0D2071CBF32
:100C800011F8013B00F8013B01D30B88038060465B
:100C9000704700BF082A13D38B07B1D010F00303AD
:100CA000AED0C3F10403D21ADB071CBF11F8013B1D
:100CB00000F8013BA4D331F8023B20F8023B9FE748
:100CC000043AD9D3013A11F8013B00F8013BF9D2BB
:100CD0000B7803704B7843708B7883706046704755
:100CE00080EA010C1CF0030F37D110F0030C20F048
:100CF000030021F0030150F8042B08BF51F8043B16
:100D00000ED08CF0030C6FF07F434FEACC0C23FA2B
:100D10000CFC51F8043B42EA0C0243EA0C0300BF0E
:100D2000A2F1013C9A4201BF2CEA020C1CF0803F68
:100D300050F8042B51F8043BF2D04FEA02604FEA1E
:100D40001222012828BFB0EB036F08BF1B0AF4D0A2
:100D500003F0FF03000EC01A704710F0030F0AD013
:100D600010F8012B11F8013B012A28BF9A42F4D058
:100D7000A2EB030070474DF8045D50F8042B01F01E
:100D8000030521F0030151F8043B022D26D04DD874
:100D900022F07F45B5EB132FA2F1013C2CEA020CA7
:100DA0000DD11CF0803C08BF51F8043B0AD185EA04
:100DB0000205B5EB036F0CD150F8042BE8E74FEABE
:100DC00013235BE03CF07F4C54D10B784FEA126563
:100DD00054E04FEA126503F0FF034FE04FEA02458B
:100DE000A2F1013C4FEA15452CEA020CB5EB134F7A
:100DF00018D11CF0803C08BF51F8043B07D185EAAC
:100E00000205B5EB034F09D150F8042BE6E75FEA82
:100E10000C4C2FD10B884FEA12452FE04FEA0343C9
:100E20004FEA12454FEA134328E000BF02F0FF05E6
:100E3000B5EB136FA2F1013C2CEA020C0DD11CF0B2
:100E4000803C08BF51F8043B0AD185EA0205B5EBA6
:100E5000032F0AD150F8042BE8E74FEA13630DE0A3
:100E600012F0FF0F06D051F8043B4FEA122523F091
:100E70007F4303E04FF0000020BC704705F0FF0205
:100E800003F0FF00012828BF904204BF2D0A1B0A6F
:100E9000F4D0A2EB000020BC704700BF4FEA410C29
:100EA0007FEA6C5C02D150EA013C0AD14FEA430C64
:100EB0007FEA6C5C02D152EA033C02D14FF00000A1
:100EC00070474FF0010070474FEA410212F50012DF
:100ED00015D211D56FF47873B3EB625212D94FEA81
:100EE000C12343F0004343EA505311F0004F23FA6B
:100EF00002F018BF404270474FF00000704750EAC0
:100F0000013005D111F0004008BF6FF0004070477C
:100F10004FF00000704700BF2DE9F14F03F11C04B2
:100F200002EB840C4FEA930B8A68CB680868496827
:100F300000F046F93CE9F0006040694072407B40B7
:100F40000BF1060E4EE083EA134480EA134582EA71
:100F5000134746BA96EA3444604000F00F1684EA1C
:100F6000063420F00F1684EA161054BA94EA0106EB
:100F7000724002F00F1486EA043622F00F1486EA5B
:100F800014124CBA6540694001F00F1485EA04352B
:100F900021F00F1485EA14115CBA67407B4003F01E
:100FA0000F1487EA043723F00F1487EA141344BAA6
:100FB00044404DBA4D4056BA56405FBA5F4087EA4A
:100FC000174886EA174B84EA17464FEA38488BEAF7
:100FD0001B4485EA1B4788EA1B4580EA3440694088
:100FE00072407B4000F0703400F0803500F00F302C
:100FF00040EA440040EAD50080EA900404F033243B
:1010000080EA8400604001F0703401F0803501F026
:101010000F3141EA440141EAD50181EA910404F02B
:10102000332481EA8401614002F0703402F080359B
:1010300002F00F3242EA440242EAD50282EA920406
:1010400004F0332482EA8402624003F0703403F037
:10105000803503F00F3343EA440343EAD50383EAC0
:10106000930404F0332483EA84036340C943DB43DD
:1010700081EA000483EA044686EA020183EA014326
:1010800082EA334583EA14435C4084EA00077FEA3E
:10109000040A8AEA024A8AEA010B87EA11488AEAC4
:1010A000374A80EA060181EA1A418AEA030A04EA19
:1010B0000A00454088EA040707EA0B0041408AEA33
:1010C0000B0608EA060084EA34428AEA3A4602EA53
:1010D000060358404540414087EA37438BEA3B408E
:1010E00003EA000985EA090582EA0309464006EA9F
:1010F0000906714085EA010005EA3546464006EAE0
:10110000314181EA304181EA364606EA304686EAD4
:10111000354634400F4086EA010508EA050886EAAC
:101120003640024088EA020881EA314213405C40BE
:1011300080EA020309EA030987EA0907674088EAA7
:10114000040806EA0A0601EA0B018AEA0B042540B4
:101150008AEA3A44204045408BEA3B4B02EA0B02C4
:10116000564084EA0B04234059406E40694087EAA8
:10117000364080EA384080EA060380EA104481EA7B
:10118000134585EA344585EA17427D4082EA3541B8
:1011900080EA05403CE9F0006040694072407B40D5
:1011A000BEF1010E3FF6CFAE20BC00F05FF8286024
:1011B0006960AA60EB60BDE8F08F00BF00F000BA84
:1011C00080EA101404F0F01480EA0410604081EA10
:1011D000111404F0F01481EA0411614082EA12143F
:1011E00004F0F01482EA0412624083EA131404F05B
:1011F000F01483EA0413634080EA102404F47F446B
:1012000080EA0420604081EA112404F47F4481EAEA
:101210000421614082EA122404F47F4482EA042219
:10122000624083EA132404F47F4483EA0423634086
:1012300081EA500404F0553480EA4400614083EAB6
:10124000520404F0553482EA4402634082EA900476
:1012500004F0333480EA8400624083EA910404F0AD
:10126000333481EA84016340704700BF82EA90040E
:1012700004F0333480EA8400624083EA910404F08D
:10128000333481EA8401634081EA500404F0553428
:1012900080EA4400614083EA520404F0553482EA53
:1012A0004402634080EA102404F47F4480EA04206E
:1012B000604081EA112404F47F4481EA0421614002
:1012C00082EA122404F47F4482EA0422624083EA20
:1012D000132404F47F4483EA0423634080EA101457
:1012E00004F0F01480EA0410604081EA111404F064
:1012F000F01481EA0411614082EA121404F0F0143F
:1013000082EA0412624083EA131404F0F01483EAC0
:1013100004136340704700BF2DE9F14F94464FEA34
:10132000930B8A68CB6808684968FFF749FF0BF19F
:10133000060E33E083EA134480EA134582EA13473A
:1013400046BA96EA3444604000F00F1684EA063448
:1013500020F00F1684EA161054BA94EA010672407F
:1013600002F00F1486EA043622F00F1486EA1412F3
:101370004CBA6540694001F00F1485EA043521F04C
:101380000F1485EA14115CBA67407B4003F00F1418
:1013900087EA043723F00F1487EA1413BCE8F0003F
:1013A0006040694072407B4000F0E03400F010354E
:1013B00000F00F3040EA540040EAC50080EA900493
:1013C00004F0332480EA8400604001F0E03401F04E
:1013D000103501F00F3141EA540141EAC50181EABB
:1013E000910404F0332481EA8401614002F0E03486
:1013F00002F0103502F00F3242EA540242EAC5020E
:1014000082EA920404F0332482EA8402624003F008
:10141000E03403F0103503F00F3343EA540343EA9A
:10142000C50383EA930404F0332483EA840363400E
:1014300081EA324787EA134581EA354690EA060495
:1014400084EA034B82EA1B4280EA044484EA0544AE
:1014500083EA144A85EA14448BEA044B84EA37444D
:1014600081EA0B4181EA164104EA0A00454082EA1A
:1014700004082BEA080041408AEA0B0602EA06004B
:1014800084EA34438AEA3A4603EA0607784045404C
:10149000414088EA38478BEA3B4007EA000985EA81
:1014A000090583EA0709464006EA0906714085EA0C
:1014B000010005EA3546464006EA314181EA3041FD
:1014C00081EA364606EA304686EA3546344008EA7E
:1014D000010886EA01052A4086EA364003405A4060
:1014E00081EA31431F407C4080EA030709EA07098B
:1014F00088EA0908544088EA020806EA0A0601EA6E
:101500000B018AEA0B0215408AEA3A421040454034
:101510008BEA3B4003405E404240174079404D40DB
:101520004E40E443F64386EA18435D4085EA0540B1
:1015300083EA134386EA034183EA384284EA11438B
:1015400083EA04435FEA3343BEF1010E3FF6F2AE95
:101550001ED4BCE8F0006040694072407B4020BC73
:10156000FFF784FE28606960AA60EB60BDE8F08F39
:101570002DE9E0414FF2F00280EA1031114080EA9B
:101580000130484041088208C3084FF0000E4FE781
:1015900000F0113001F0113102F0113203F011337B
:1015A00040EA410040EA820040EAC3004FF2F00204
:1015B00080EA1031114080EA01304840BDE8E08106
:1015C0002DE9F04F02F11C050646074600EB8508A1
:1015D00051F8040B043A46F8040BF9D14FF0010C12
:1015E000FFF7C6FF5FEA302080EA0C001ECF4140C3
:1015F0004A4053405C401EC62000464517D04FEA83
:101600004C0C1CF4807F18BFACF1E50C2C2DE7D0FE
:101610003C2D06D1FFF7ACFF06CF41404A4006C63D
:10162000100006CF41404A4006C61000D8E736E910
:101630000F00FFF7C5FD043D86E80F00F7D1BDE8B8
:10164000F08F00BF2DE9F04FB0E8FE0783B02DE921
:10165000010790E8005F4FF00A0006900198DB193F
:101660009CEA030C18EB3C4897EA080713EB375346
:1016700093EA3C4C18EB3C6898EA375724189EEAEA
:10168000040E19EB3E4990EA090014EB305494EA39
:101690003E4E19EB3E6999EA3050CDE90489DDE907
:1016A000028949199AEA010A18EB3A4895EA0805AD
:1016B00011EB355191EA3A4A18EB3A6898EA3555F8
:1016C00092199BEA020B19EB3B4996EA090612EBC9
:1016D000365292EA3B4B19EB3B6999EA365613EBCB
:1016E000706393EA3B6B18EB3B4898EA706013EB2E
:1016F000305393EA3B4B5FEA3B6B18EB0B0898EADD
:1017000030505FEA706014EB756494EA3C6C19EB3E
:101710003C4999EA756514EB355494EA3C4C5FEA10
:101720003C6C19EB0C0999EA35555FEA7565CDE912
:101730000289DDE9048911EB766191EA3E6E18EBCE
:101740003E4898EA766611EB365191EA3E4E5FEAE2
:101750003E6E18EB0E0898EA36565FEA766612EB94
:10176000776292EA3A6A19EB3A4999EA776712EB9B
:10177000375292EA3A4A5FEA3A6A19EB0A0999EA59
:1017800037575FEA77670190069801387FF465AFB5
:1017900001BC80E8005FBDE8000700E9FE0703B078
:1017A000BDE8F08F30B44FF0000310F8014B11F892
:1017B000015B013A84EA050443EA0403F5D1A3F18D
:1017C00001034FEAD37030BC704700BF4FF00003F5
:1017D00010F8012B013943EA0203F9D1A3F1010307
:1017E0004FEAD370704700BF30B411F8014B12F8C4
:1017F000015B6C4000F8014B013BF6D130BC7047F7
:101800002DE9F14FF8C892E8005E19EB03095AEB95
:10181000040A5BEB050B5CEB060C4EEB070E91E844
:10182000E001A9FB0502AAFB0543E9FB6624EAFBEC
:101830006634A9FB0765E9FB6845B1E80003EBFBEB
:101840006836ECFB6846EEFB6856ABFB0987ECFBA1
:101850006957EEFB696791E80202EAFB6148EBFB1E
:101860006158ECFB6168EEFB61784FF00001EAFB28
:101870000951EBFB6961ECFB6971EEFB69814FF487
:10188000A03C4FEA154949EA06495FF0000AE9FB26
:101890000C0A4FEA164646EA0746E6FB6C2A4FEA70
:1018A000174747EA0847E7FB6C3A4FEA184848EA07
:1018B0000148E8FB6C4AADB25544AF0805F003059A
:1018C00007EB8707C01952F1000153F1000254F1F0
:1018D000000345F1000420BC1FC5BDE8F08F00BF28
:1018E00030B490E83C10511D53F1000154F1000157
:1018F00055F100014CF100014FEA9101494201F01C
:101900000501521853F1000354F1000455F100058C
:101910004CF1000C0CF0030C80E83C1030BC70471C
:101920002DE9F04F90E8F00F00F140004FF0040E69
:1019300059E0F0B4826BC36B0468052524268759EF
:101940003C444FEA724787EAF24787EA92273C44D1
:1019500042684FEAF21787EAB24787EAD2073C4467
:1019600040F8044B032D08BF6FF01B0687593A441B
:101970004FEA734787EAF34787EA93273A44436875
:101980004FEAF31787EAB34787EAD3073A4440F8A8
:10199000042B87593B444FEA744787EAF44787EAA8
:1019A00094273B4444684FEAF41787EAB44787EA30
:1019B000D4073B4440F8043B013DC0D1A0F13C00BA
:1019C000076A3C444FEA724787EAF24787EA922760
:1019D0003C4402684FEAF21787EAB24787EAD20727
:1019E0003C44C463F0BC4FF0020288EA781C8CEAE5
:1019F000F84C0BEBBC1C8AEA090303EA080383EAF0
:101A00000A039C4450F8043B9C4451F8043B9C441A
:101A1000674444EA050B0BEA060B04EA05034BEAAC
:101A2000030BE34484EAF42383EA34530BEBB30B54
:101A300087EA771C8CEAF74C0AEBBC1C89EA08039E
:101A400003EA070383EA09039C4450F8043B9C44DF
:101A500051F8043B9C4466444BEA040A0AEA050A2E
:101A60000BEA04034AEA030AE2448BEAFB2383EA13
:101A70003B530AEBB30A86EA761C8CEAF64C09EB78
:101A8000BC1C88EA070303EA060383EA08039C44B4
:101A900050F8043B9C4451F8043B9C4465444AEA9A
:101AA0000B0909EA04090AEA0B0349EA0309E144BC
:101AB0008AEAFA2383EA3A5309EBB30985EA751CEB
:101AC0008CEAF54C08EBBC1C87EA060303EA050325
:101AD00083EA07039C4450F8043B9C4451F8043BC0
:101AE0009C44644449EA0A0808EA0B0809EA0A0324
:101AF00048EA0308E04489EAF92383EA395308EB0A
:101B0000B30884EA741C8CEAF44C07EBBC1C86EA2C
:101B1000050303EA040383EA06039C4450F8043BEC
:101B20009C4451F8043B9C44E34448EA090707EA13
:101B30000A0708EA090347EA0307674488EAF82323
:101B400083EA385307EBB3078BEA7B1C8CEAFB4C28
:101B500006EBBC1C85EA040303EA0B0383EA0503D6
:101B60009C4450F8043B9C4451F8043B9C44E244A0
:101B700047EA080606EA090607EA080346EA0306F2
:101B8000664487EAF72383EA375306EBB3068AEA0B
:101B90007A1C8CEAFA4C05EBBC1C84EA0B0303EAC2
:101BA0000A0383EA04039C4450F8043B9C4451F824
:101BB000043B9C44E14446EA070505EA080506EAB9
:101BC000070345EA0305654486EAF62383EA3653AC
:101BD00005EBB30589EA791C8CEAF94C04EBBC1CD3
:101BE0008BEA0A0303EA090383EA0B039C4450F8D7
:101BF000043B9C4451F8043B9C44E04445EA060401
:101C000004EA070405EA060344EA0304644485EA97
:101C1000F52383EA355304EBB304013A7FF4E5AED0
:101C2000A0F14000BEF1010E7FF483AEA0F1400CA4
:101C30009CE80F00001949199219DB19ACE80F0054
:101C40009CE80F004044494452445B44ACE80F0018
:101C5000BDE8F08F38B50022002304460D46FEF79C
:101C6000A9FE28B920462946BDE83840FEF7A2BFA4
:101C7000204605F10041FEF79DFF404261EB410126
:101C800038BD2DE9F04786468C460846089E154625
:101C900074461946002B40F0C1808542B2FA82F2A8
:101CA00045D94AB1C2F1200300FA02FC95409440A4
:101CB0002EFA03F343EA0C0C4FEA154EA8B2230C9C
:101CC000BCFBFEF80EFB18CC08FB00F943EA0C4302
:101CD000994528D9EB1808F1FF3704D2994502D964
:101CE000A8F102072B44A3EB0903A4B2B3FBFEFC4B
:101CF0000EFB1C330CFB00F044EA0344A04214D951
:101D00002C190CF1FF3304D2A04202D9ACF102032A
:101D10002C44241A43EA07401EB1D4400023346007
:101D20007360BDE8F0874746DDE76346F1E792BBA5
:101D3000431B01214FEA154EAFB2200CB3FBFEFC52
:101D40000EFB1C330CFB07F840EA0343984561D9AE
:101D5000EB180CF1FF3004D2984502D9ACF1020027
:101D60002B44A3EB0803A4B2B3FBFEFC0EFB1C3315
:101D70000CFB07F744EA0344A7424DD92C190CF198
:101D8000FF3304D2A74202D9ACF102032C44E41B76
:101D900043EA0040C0E7C2F120039540944020FA96
:101DA00003F12EFA03F34FEA154E9040AFB203430E
:101DB000B1FBFEFC0EFB1C10190C0CFB07F841EAF2
:101DC0000041884522D969180CF1FF3004D28845BA
:101DD00002D9ACF102002944A1EB08019BB2B1FB8E
:101DE000FEFC0EFB1C110CFB07F743EA01439F426C
:101DF0000ED9EB180CF1FF3104D29F4202D9ACF19D
:101E000002012B44DB1B41EA004193E76046E3E714
:101E10006146F7E76046A4E76346B8E7834206D920
:101E200016B9002108467CE7C6E900E0F9E7B3FAF5
:101E300083F78FB9834201D3724508D8BEEB020401
:101E400060EB030301209C461EB9002169E7384678
:101E5000FAE7C6E9004CF8E7C7F1200CBB400EFAE0
:101E600007F522FA0CF42EFA0CF1BA401C4320FAC2
:101E70000CF3B8404FEA144901431FFA84FEB3FB48
:101E8000F9F809FB18300B0C08FB0EFA43EA004383
:101E90009A4540D9E31808F1FF3004D29A4502D997
:101EA000A8F102002344A3EB0A0389B2B3FBF9F8BB
:101EB00009FB183308FB0EFE41EA03418E452CD97D
:101EC000611808F1FF3304D28E4502D9A8F102034C
:101ED000214443EA0040A1EB0E01A0FB02984145DA
:101EE000CE46434602D306D14D4504D20138B9EB64
:101EF000020E68EB0403002EA7D0B5EB0E0261EBD7
:101F0000030101FA0CFC22FA07F3F9404CEA03033F
:101F1000C6E9003199E74046C5E74346D9E70000E6
:101F20002DE9F04182B06D4D00AFD5F85C31996874
:101F300011F001011AD140F603403A1D0AF06CF885
:101F40000446002840F0C5807868C3681B785BB9F8
:101F500005F1CC03D3E8AF2F02F00902D3E8EF1F5D
:101F6000C3E8E42F002CF9D111F0C6F9002141F2A9
:101F700003003A1D0AF050F80446002840F0A980FA
:101F80007B68574EDA68D2F80100D2F8051003C614
:101F9000184611F0B1F9214641F201003A1D0AF04C
:101FA0003BF80446002840F094807868C3685A786B
:101FB00085F868205A88A5F86A201A7985F869207A
:101FC000B3F80720A5F86C20B3F80530A5F86E30FB
:101FD00011F092F9214641F202003A1D0AF01CF874
:101FE0000446002875D1D7F804C0DCF80C20531C37
:101FF0004132344618685968083303C49342264670
:10200000F7D1604611F078F90BF0C8FF04460028BC
:102010005FD195F88230990626D46C4688B06A461E
:10202000304B4FF4C45153612F4B3048936103231D
:1020300042F8103F59F056FDA54695F874305A06FF
:102040005AD46C4688B06A46294B4FF4C25153614A
:10205000284B26489361032342F8103F59F042FD74
:10206000A5466FF0120434E0072140F6334009F032
:1020700099FF0646002800F0458107210C305BF0EF
:10208000CAFD6FF0680303700623C0F80240847134
:10209000447004712246C370314640F6334009F063
:1020A000BBFF0446A8B9012140F6314009F07AFF90
:1020B0000646002800F0268101210C305BF0BAFDB5
:1020C0002246314640F6314009F0A6FF044600287A
:1020D000B3D020460837BD46BDE8F081000000209F
:1020E00070000020BEE507005FEB0700C409070091
:1020F000F0E5070057EB0700002142F203003A1D0C
:1021000009F08AFF04460028E3D17B68AC4EDA6808
:10211000D2F80100D2F8051003C6184611F0ECF809
:10212000214642F202003A1D09F076FF04460028DB
:10213000CFD17C68E368B3F8012091B2A5F8FC2008
:1021400029B1DA78114606F1280069F09AFF204695
:1021500011F0D2F895F8746016F0200618D102211B
:1021600040F66D4009F01EFF0446002800F0CA80CA
:1021700002210C305BF04FFD0123214603704670B5
:10218000324640F66D4009F047FF04460028A0D1D2
:1021900095F894301B0712D5002142F21C003A1D1D
:1021A00009F03AFF0446002893D17868C368D3F851
:1021B0000120D3F80530C5E9362311F09DF895F8D4
:1021C000D0309E0622D53846B91C09F0A5FF04463A
:1021D00000287FF47EAF042142F2240009F0E2FEE1
:1021E0000646002800F08E8004210C305BF013FDC1
:1021F0003B88224603807B883146438042F224009C
:1022000009F00AFF044600287FF463AF95F8D03048
:102210005C0610D5002142F22A003A1D09F0FCFEAE
:10222000044600287FF455AF7868C3685B7885F86A
:10223000183111F061F8082142F2010009F0B2FEF4
:10224000044600285ED008210C305BF0E4FC95F8D1
:10225000D01040F2022311F0400F08BF03230246C2
:1022600088074CBF43F02C0043F00C008B0695F818
:10227000D13048BF40F0400013F0090F95F89A3074
:1022800018BF40F4006003F00603CE0748BF40F0DB
:102290001000062B08BF40F4C070002159F02DFC3F
:1022A0002146002242F2010009F0B6FE0446002851
:1022B0007FF40FAF95F87430B5F8FC10980624D46D
:1022C000C9B941F205003A1D09F0A6FE04460028EE
:1022D0007FF4FFAEB5F8FC307C684BB9E368B3F827
:1022E0000120A5F8FC209A883648114669F0C9FEFD
:1022F000204611F001F8082140F6014009F052FE95
:102300000446B8B96FF06804E3E60029F3D16C46DF
:1023100088B06A462C4B4FF4C25153612B4B2C486A
:102320009361032342F8103F59F0DCFBA5466FF0A0
:102330000404CEE608210C305BF06DFC95F8D0303B
:102340000246D90734D44FF00051224859F0D5FB4A
:102350002146002240F6014009F05EFE04460028B6
:102360007FF4B7AE01463A1D4FF6014009F054FE26
:10237000194CA8B36D4688B06A46184BC2E90534BB
:1023800003234FF4C451124842F8103F59F0AAFBFE
:10239000AD460BF051FA044600287FF49AAE0CF0DB
:1023A0007BFE044600287FF494AE0AF0B3FC90E66E
:1023B00001A1D1E90001C9E7908800020080002056
:1023C000D00000200001002018E6070070EB070095
:1023D000C40907001088000232EB07003FE607003F
:1023E0007B686E46DD688AB0B5F80130032B96BF76
:1023F000464A474952F823106A46C2E9071340F299
:10240000013344489384444BC2E905044FF43351EB
:1024100042F8103F414859F065FBB5F80120B54638
:10242000022AB5F803304DD1032B4BD83C4A52F861
:1024300023106E468AB06A46C2E9071340F20133A0
:1024400038489384344BC2E905044FF4335142F8C1
:10245000103F324859F046FBB5466B7995F806C0F7
:10246000032B98BF304AB5F80760D5F809006D46D0
:102470008EB094BF52F8231025496A46C2E907136B
:1024800040F20133DFF8A4E01386294BC2E909C604
:10249000C2E905E4D06244F2C04142F8103F1F484F
:1024A00059F020FBAD46786810F026FF00214FF66A
:1024B00002403A1D09F0B0FD064628B188B06A46D0
:1024C0001C4B5BE71249B4E77868DFF86C80C3689F
:1024D000B3F80130A8F8B93010F00EFF98F8B93011
:1024E0005B077FF556AF31464FF603403A1D09F0C2
:1024F00093FD18B188B06A46104B3FE77868C3680F
:102500005B7888F8B83010F0F7FE42E7BC1507009A
:10251000B2DF070067E6070005000001C4090700F5
:10252000AC15070084E607009C150700A0E607002D
:1025300008000001D1E6070000000020FEE60700C9
:102540002DE9F04F0C46D0F82011A3B00B6B1546C7
:1025500015905BBB159818A9276ED4F88060D5F844
:1025600080B063F0CEFC78B34FF0000A06F59C53C0
:1025700008339B4522D82B6DB3F57A6F179355DD41
:10258000236DB3F57A6FACBF00230123002F1693A0
:102590004EDB0BF59C5308339E4200F24081BAF1AA
:1025A000190F00F33C814FF0020877E00622183142
:1025B00005F1200045F0CEFF0028CBD14FF00108F7
:1025C000404623B0BDE8F08FDDF870A0BAF1000FEF
:1025D00004D1DDF86CA0BAF1000FC7D042F20F7140
:1025E0001D9B189A8B420AD16FF47A63D31840F27C
:1025F000657293428CBF6FF058036FF05B03204607
:10260000AAEB030861F06EFFD4F88C20034604F1B6
:1026100094010AB9D4F89020206D5746CDE9008086
:10262000159833F0D1FCC24606469FE70023ADE77C
:102630002B6E169A03EB42039F4215DD5846FDF7B9
:10264000CDFE804630468946FDF7C8FE4FF0333256
:10265000774BFDF73DFF02460B4640464946FEF7E5
:10266000A9F9002840F0DB800BF59C5308339E420B
:1026700000F2D580BAF1190F00F3D18017F1550F90
:1026800069DB17F1500F8EDB17F14B0F66DB17F18B
:10269000460FB4BF4FF004084FF005083046FDF771
:1026A0009DFE814658468A46FDF798FE02460B4637
:1026B000CDE9122300225F4BFDF70AFF02460B46CD
:1026C00048465146FEF794F900284AD008F10A0816
:1026D000169B0BB1A8F102082B6E0321CDE9103B2C
:1026E000DA1B179B90450F9395F82530524A0E93AD
:1026F00095F82430C8BF4FF000080D9395F82330AB
:10270000D8BF4FF001080C9395F822300B9395F841
:1027100021300A9395F820300797CDE90863236D9F
:10272000069394F82530059394F82430049394F894
:102730002330039394F82230029394F821300193CC
:1027400094F8203000933D4B1598C8BF13463C4A7F
:102750003DF02AFA34E74FF001089FE74FF00308F5
:102760009CE74FF03332DDE91201314BFDF7B0FE4B
:1027700002460B4648465146FEF73AF910B108F1B9
:102780000508A5E728A3D3E90023DDE91201FDF739
:102790009FFE02460B4648465146FEF729F910B106
:1027A00008F1020894E7B34502D208F101088FE767
:1027B0000022204B48465146FDF78AFE02460B4652
:1027C000DDE91201FEF714F910B1A8F10A087FE75C
:1027D0004FF03332164B48465146FDF779FE02461C
:1027E0000B46DDE91201FEF703F910B1A8F1050867
:1027F0006EE70DA3D3E9002348465146FDF768FE76
:1028000002460B46DDE91201FEF7F2F810B1A8F11D
:1028100002085DE7B34588BF08F1FF3858E74FF07D
:102820000008CDE6AFF300809A9999999999F13F04
:102830003333F33F0000F83FACB5080098B508000B
:10284000C2B5080000000000C1F30A5C02460B4656
:102850002DE9F041ACF2FF350C460646132D34DC71
:10286000002D20DBDFF8D0800F4648FA05F801EA9A
:10287000080C5CEA000C2DD02DA3D3E90023FDF752
:1028800071FC00220023FEF7B3F840B1002C03DDF9
:102890004FF480132B411F4427EA080400262146E9
:1028A0003046BDE8F08122A3D3E90023FDF75AFCAE
:1028B00000220023FEF79CF80028F0D0002C33DB28
:1028C0003443EBD000261D4CE9E7332D06DDB5F58A
:1028D000806F26D010461946BDE8F081ACF2134C4B
:1028E0004FF0FF3727FA0CF73842F3D010A3D3E9A3
:1028F0000023FDF737FC00220023FEF779F80028BB
:10290000CDD0002C334609DD142D06D0C5F1340599
:102910000122AA4013449E4200D9013423EA07064B
:10292000BDE7FDF71FFCD7E700264FF00044B6E7F0
:102930009C7500883CE4377EFFFF0F000000F03FED
:10294000F8B5C1F30A5604460D4617460B462EBB92
:1029500021F00043034320D02D4B0022FDF7B8FDAA
:102960002C4B04460D469F4241DBC1F30A560B46F1
:10297000363EBA1940F2FE718A4217DC002A30DC7A
:1029800012F1350F1EDB244E363220461E40234BFB
:1029900046EA02510022FDF79BFDF8BD40F2FF72AE
:1029A0009642E6D10246FDF7DDFBF8BD14A3D3E95C
:1029B0000023ED0F1A481C4665F3DF742146FDF72E
:1029C00087FDF8BD05F00044164844F0D27141F48B
:1029D000B7310DA3D3E9002341F01F01FDF778FDC6
:1029E000F8BD0D4E20461E4046EA0251F8BD06A332
:1029F000D3E90023FDF76CFDF8BD00BFAFF3008005
:102A00009C7500883CE4377E59F3F8C21F6EA5011F
:102A100000005043B03CFFFFFFFF0F800000903CE0
:102A20009C75008859F3F8C22DE9F04F016C9BB0FA
:102A300016461F46279D0490CDE9026749B1426CB6
:102A40000123044693404A608B604DF0E1FE002371
:102A50002364B7F10009C0F2B68000232B607E4BDF
:102A600033EA090300F0BA800022DDE90234184697
:102A700021460023CDE90801FDF792FF804668B1A9
:102A80000123269A1360289B13B1744B289A136074
:102A9000DFF8CC8140461BB0BDE8F08F18AB04983E
:102AA000019319AB0093DDE908234EF0B7FA834692
:102AB0005FEA195540F0A980DDE91885454405F223
:102AC0003243202B40F34D82C3F1400309FA03F94E
:102AD00005F2124326FA03F349EA0300FDF77EFCF0
:102AE000013D0123A1F1F871109300225D4BFDF728
:102AF00037FB53A3D3E90023FDF7EAFC52A3D3E944
:102B00000023FDF72FFB06460F462846FDF776FC0F
:102B10004FA3D3E90023FDF7DBFC02460B4630460A
:102B20003946FDF71FFB06460F46FEF7CDF900229A
:102B30008246002330463946FDF73CFF002840F02E
:102B40000382A8EB0508BAF1160F08F1FF330693CC
:102B500000F2A781444E06EBCA06DDE90801D6E97A
:102B60000023FDF727FF002800F0848000230AF1EE
:102B7000FF3A0F9308F1FF33002BC0F29981002335
:102B80000A93BAF1000F7BDA0A9BCDF82CA0A3EBD5
:102B90000A030A93CAF100034FF0000A0E93249B24
:102BA000092B77D8052B40F3E181043B00272493C0
:102BB000249B023B032B00F25986DFE813F05404F8
:102BC000510447042C04012329F000492B60224BB7
:102BD000CDF80C9033EA09037FF446AFC9F313092B
:102BE00042F20F73269A59EA060913601DD0289BFA
:102BF000DFF87880002B3FF44DAF08F10303289AEB
:102C0000404613601BB0BDE8F08FDDE90812CDF837
:102C10004080A5F2FF35C2F313030846DDF860805B
:102C200043F07F5141F440115FE7289BDFF840807B
:102C3000002B3FF42FAF08F10803E0E7AFF300806B
:102C400061436F63A787D23FB3C8608B288AC63FB2
:102C5000FB799F501344D33F0000F07F41BD070034
:102C600040BD07000000F83F200E0700DCBD070054
:102C7000D0BD0700B8F1000F40F3B1840F900A9067
:102C8000069BCDF82CA05344069300230E93249B5F
:102C9000092B87D900230127CDE924334FF0FF33D7
:102CA0000C970793049B00215964079B1193049888
:102CB0004DF088FD0590002800F0E185079B0E2B64
:102CC0008CBF002707F00107DDE904321A64002FEA
:102CD00000F01B810B9A002A40F34A81BC4E02F09F
:102CE0000F03D4054FEA221806EBC303D3E90067AC
:102CF00040F17083B74B08F00F080325D3E9082390
:102D0000DDE90801FDF70EFDCDE91201B8F1000F74
:102D100012D0DFF8C09218F0010F08D030463946C3
:102D20000135D9E90023FDF7D3FB06460F465FEADC
:102D3000680809F10809EED132463B46DDE9120187
:102D4000FDF7F0FC804689460F9B43B10022A24B61
:102D500040464946FDF72EFE002840F047842846AD
:102D6000FDF74CFB42464B46FDF7B2FB9B4B002266
:102D7000FDF7F8F9079B0646A1F15077002B00F00C
:102D8000AB80079B0B9C1293059B404612995D1CE0
:102D9000CDE914678E4E06EBC10353E90212CDE96B
:102DA00016124946FEF790F800F13007FDF726FBB2
:102DB00002460B4640464946FFB2FDF7D1F9894627
:102DC0000C998046DDE91623002900F00F810020D0
:102DD0008349FDF7A7FCDDE91423FDF7C1F9059E42
:102DE00042464B46377006460F46FDF701FE002867
:102DF00040F02F850023CDF858A0CDF850B09A466A
:102E0000DDF848B012942BE00AF1010ADA4580F2AD
:102E1000BD84304639460022724BFDF759FB002233
:102E2000704B06460F4640464946FDF751FB894622
:102E30008046FEF749F80446FDF7E0FA02460B46E5
:102E4000303440464946FDF78BF932463B4605F89B
:102E5000014B80468946FDF7ADFD002840F09C847B
:102E600042464B4600205C49FDF77AF932463B4624
:102E7000FDF7A0FD0028C7D0DDF850B02F46129C0A
:102E8000059902E08F4200F05F843A4617F8013D51
:102E9000392BF7D00133DBB23B70DDF8148005929B
:102EA0006BE101230F9308F1FF33002BBFF667AEF0
:102EB000C8F101030A930023069362E62846FDF752
:102EC0009DFA42464B46FDF703FB0022434BFDF7BC
:102ED00049F90646A1F15077404649460022424B47
:102EE000FDF73EF932463B4680468946FDF780FDB8
:102EF000002840F0AD8340464946324607F1004382
:102F0000FDF758FD002840F0D5810B9A199B0E2A39
:102F100002DC002B80F2AD810C9A002A00F0B58013
:102F2000249A012A40F38583079A0E9B551EAB42D3
:102F3000C0F2C782002AA3EB050580F25B840A9BDE
:102F4000079AA3EB0208C9E25046FDF757FA32464A
:102F50003B46FDF725FD00287FF4F3AD0AF1FF3A6B
:102F6000EFE5C3F1200306FA03F0B7E501271FE6FA
:102F700000F0A3820B9B164E5D4205F00F0306EB9B
:102F8000C303DDE90801D3E90023FDF7A1FA2E11FF
:102F9000CDE9120100F052840E4C00230225804638
:102FA0008946F00709D5404649460135D4E9002352
:102FB000FDF78EFA3B4680468946761004F10804F8
:102FC000EFD1002B7FF4C0AEDDE91289BCE600BF73
:102FD000200E0700F80D07000000F03F00001C4025
:102FE0000000E03F0000244000001440DDE914012F
:102FF000FDF76EFA059B1F70129B012BCDE90C01AA
:1030000000F00984129F059BCDF840A01F440022C8
:10301000AA4B40464946FDF75BFA89468046FDF7D4
:1030200053FF8246FDF7EAF902460B460AF1300AE1
:1030300040464946FDF794F805F801ABAF4280469B
:103040008946E4D1DDF840A000229D4BDDE90C016A
:10305000FDF788F842464B46FDF7ACFC002840F0EF
:103060007B8300209649DDE90C23FDF779F8424681
:103070004B46FDF7BDFC002840F01982199B002B40
:1030800003DB0B9B0E2B40F3F58000230E9DDDF838
:1030900028801E460C93B8F1000F0DDD069900291B
:1030A0000B4609DD41450A9AA8BF4346D21AA8EB50
:1030B0000308CB1A0A9206930E9B53B10C9B13B1D3
:1030C000002D40F01E8259460E9A04984DF088FD5E
:1030D0008346012104984DF0A3FC0746BAF1000F86
:1030E00040F06381249B012B40F37A8101230699F0
:1030F0000B4413F01F0308D0C3F12002042A00F38D
:10310000B5810AD0C3F13C0300E01C230A9A98441D
:103110001A440A92069A1A4406920A9B002B05DD6D
:1031200059461A4604984DF0B5FD8346069B002B80
:1031300005DD39461A4604984DF0ACFD0746249B40
:10314000022B0F9BD4BF00250125002B40F0BE8031
:10315000079B002B24DC1DB3079B002B00F08F8105
:10316000259BDDF81480DC43394604984DF050FB74
:103170001EB1314604984DF04BFB594604984DF072
:1031800047FB00220599631C0A70269A1360289B4E
:10319000002B3FF47FAC404619601BB0BDE8F08FB8
:1031A0000C9B002B00F0AF80B8F1000F00F3C08142
:1031B000BAF1000F40F0D382B146059D079C6B1E0B
:1031C0001C44029B089403F00103049C0A933946B3
:1031D00058464CF061FD3146824658464DF0CEFDD2
:1031E0004A463946804620464DF0E8FDC268014611
:1031F0000AF13003002A40F0A281CDE906035846C7
:103200004DF0BCFD0699069020464DF001FB249B35
:10321000069A52EA0301079B40F0C2810A9A002AEB
:1032200000F0F282B8F1000FC0F2AD81089AA84612
:10323000AA4208F8013B00F0D282594600230A2234
:1032400020464DF0EFFA4E45834631464FF00003DD
:103250004FF00A02204600F09D814DF0E3FA494606
:10326000064600230A2220464DF0DCFA45468146F8
:10327000ADE7144E0B9B06EBC306D6E90034CDE94F
:103280000234259B002B80F2E881079B002B00F382
:10329000E481079B73B900220B4BDDE90201FDF7C6
:1032A00017F902460B46DDE90801FDF78DFB002802
:1032B00000F0CE8100273E4652E700BF00002440C8
:1032C0000000E03F200E0700000014403946584639
:1032D0004DF054FD0028BFF63BAF0B9B59460A2228
:1032E0000498013B0B9300234DF09CFA0C9B834602
:1032F000002B40F09282119B002B119B079302DC64
:10330000002D7FF429AFDDF814800125079CDDF83E
:10331000109007E0594600230A2248464DF082FAF1
:1033200001358346394658464CF0B6FCA54200F1BB
:10333000300308F8013BEDDB079A0025002ACCBFDB
:1033400090464FF00108059A90445946012204988E
:1033500002934DF09FFC394683464DF00FFD002847
:1033600040F3E481059A02E0904500F0D48118F81A
:10337000013CC24608F1FF38392BF5D001330B9CD4
:1033800088F80030394604984DF042FA002E00F0DB
:10339000C8812DB1B54203D0294604984DF038FAC2
:1033A000DDF81480CDF814A0E3E6014652460498F7
:1033B0004DF016FC249B0746012B40F395804FF0FF
:1033C000000A3B6907EB830318694DF0D5FAC0F199
:1033D00020038CE6DDE908340225CDE9123495E4BA
:1033E000029B002B7FF482AEDDE90212C2F31303CD
:1033F000002B7FF47BAEAD4B134033B10A9B0133FE
:103400000A93069B013306930123BAF1000F40F0A3
:10341000F9819A466AE601230C93259B0B9A134483
:1034200011930133012B1D460793B8BF0125172DBA
:1034300040F31382012204235B001146013203F1A1
:103440001400A842F8D9049B596430E401230C937A
:10345000259B002B40F3BE801D4611930793E6E7A2
:1034600000230C93D9E700230C93F1E7C3F11C036D
:103470000A9A19441A4498440A9206914DE639462C
:10348000052204984DF0CEF90746584639464DF0CE
:1034900075FC00287FF764AEDDF81480059B0B9C5B
:1034A000013301340593312388F800305CE63A4655
:1034B00017F8013D302BFAD0EFE40225DDE9088949
:1034C00042E40E9B0E95EB1A00259A44DDE9063284
:1034D000134406930A9B984613440A9301210498C7
:1034E0004DF09EFA0646D6E5029B002B7FF467AFAF
:1034F000DDE90201C1F313030A46002B3FF47BAF61
:103500005DE7049C31462A4620464DF069FB06469D
:103510005A46204631464DF0B1FA59468346204678
:103520004DF076F90E9B5B1B0E933FF4D2ADCAE5CE
:103530003146424604984DF0ADFB064638E6049805
:1035400006934DF065F9B8F1000F069B08DB029A6F
:10355000249902F0010248EA010852EA08022ED139
:1035600059460122049802934DF094FB3946834654
:103570004DF004FC0028029B40F36581392B00F0DC
:1035800031810AF13103AA460B9C35464E460AF8B2
:10359000013BF7E64DF046F945460646814616E6FC
:1035A000B8F1000FC0F25E81249948EA01080A9937
:1035B00051EA080800F05681002A7FF737AE392B10
:1035C00000F01081AA46013335460B9C4E460AF89E
:1035D000013BD7E6012325930793FFF763BBC8F1AF
:1035E000010306900F900A93FFF74ABB079B002B3D
:1035F0003FF464AC119B002B7FF787AC0B9A4046DD
:1036000049461293541E2A4B0022FCF761FF804664
:103610008946681CFCF7F2FE42464B46FCF758FF11
:103620000022244BFCF79EFD0646A1F15077FFF7E0
:10363000ABBB109A002A00F08B8003F23343069A4A
:103640000E9D1A4406920A9A90461A440A9245E739
:103650000027DDF814803E4620E7DDE90889DDE932
:10366000022340464946FDF75DF8059FFDF72CFC17
:103670000546FCF7C3FEDDE90223FCF729FF0B46F4
:10368000024649464046FCF76BFD05F1300307F85A
:10369000013B079B012B00F08980CDF818B0012673
:1036A000DDF81C90DDE902AB22E000BF0000F07FF6
:1036B0000000244000001C4052465B46204629463C
:1036C000FDF730F80136FDF7FFFB8046FCF796FE6C
:1036D00052465B46FCF7FCFE0B4602462946204656
:1036E000FCF73EFD08F13003B14507F8013B5AD025
:1036F0000022704BFCF7ECFE0022002304460D462E
:10370000FDF74EF90028D7D0DDF818B0DDF81480A9
:103710000B9C059731E50B9C3123059A01341370FE
:1037200030E6DDF81480CDF814A026E503D1029B25
:10373000DB073FF517AE18F8013CC24608F1FF3829
:10374000302BF8D00B9C1DE601343123FFF7A4BBCE
:10375000189BC3F1360372E70599FFF796BB7168B2
:1037600004984DF02FF80546002800F08F8033694B
:1037700006F10C010C3002339A00FDF73BFA2946A2
:10378000012204984DF086FA814616E5DDF858A02E
:10379000DDF850B0FFF7B9BBDDF81480DDF850B0AC
:1037A000129C0595E9E4DDF818B0454602460B4643
:1037B000FCF7D8FC80468946DDE90223FDF718F9BD
:1037C00048B940464946DDE90223FDF7E9F80028FB
:1037D0009CD0E9079AD50B9C0599FFF756BB354657
:1037E0004E46B2E5A84639233546059A4E4608F8B6
:1037F000013BBCE5069B134406930A9B9846134481
:103800000A936BE69A46DCE5392BEBD0B8F1000F52
:103810003FF7B7AEB7E62F4616E4314600230A223B
:1038200004984CF0FFFF119B0646002B119B079359
:103830003FF7BAAC002D7FF48FACB5E4DDE9128917
:103840000225FFF781BA7FF49EAEDA077FF59BAEC3
:1038500094E6DDF8148005958FE40021049B5964FB
:10386000FFF725BA002A3FF77BAE8CE6049B0025C4
:10387000184629465D644CF0A5FF059068B90E4BCB
:1038800000224FF4D5710D4844F0DAFA02460A4B93
:1038900040F2EA21094844F0D3FADDE904322595E3
:1038A0001A644FF0FF33012211930C920793FFF734
:1038B0002CBB00BF00002440E0BD0700F4BD0700A2
:1038C0002DE9F04F1C46794B9FB00E4600258346EC
:1038D000186807921A95089046F02AF800210246C7
:1038E00033460020CDE904019846199313F801AB43
:1038F000BAF12D0F5ED801A151F82AF0933A0000D9
:10390000B5390000B5390000B5390000B5390000FF
:10391000B5390000B5390000B5390000B5390000EF
:10392000E9380000E9380000E9380000E938000013
:10393000E9380000B5390000B5390000B53900009C
:10394000B5390000B5390000B5390000B5390000BF
:10395000B5390000B5390000B5390000B5390000AF
:10396000B5390000B5390000B5390000B53900009F
:10397000B5390000B5390000B5390000E93800005C
:10398000B5390000B5390000B5390000B53900007F
:10399000B5390000B5390000B5390000B53900006F
:1039A000B5390000B539000067400000B5390000A6
:1039B0008140000000230993BAF1300F00F06882C3
:1039C00000230A93AAF13003092B00F25684002742
:1039D00040463D463C460130082C07EB870104F188
:1039E000010405EB850C199090F800A0CCBF03EB07
:1039F000410703EB4C05AAF13003092BEBD90899D9
:103A0000089245F0C3FF089A8146002850D1199BBF
:103A100001460894981819909B5CA3F13002092A7A
:103A200000F2F082013192461998002A40F0F884A1
:103A3000431C19934378F0E74FF0010EB31C199320
:103A4000B378A3F1300CBCF1090F00F2F582199A9A
:103A5000302B0B9240F02B83013219921378302BCC
:103A6000FAD0A3F131000B92082840F21E83002205
:103A70000C9254BB0A9A0A4340F09882BAF1000FA4
:103A800007D1692B00F0398340F318826E2B00F0C8
:103A90001B82079B4FF000084FF0000903B11E6026
:103AA000404649461FB0BDE8F08F00BF58C0070030
:103AB0002AF02002002153460894452A89468A4666
:103AC00000F0AD820C91002CD4D0089A2846A24672
:103AD0001346002A08BF23460893FCF77FFC0B46D9
:103AE0000246102CCDE904230C9BA8BF4FF0100A0E
:103AF000092CA3EB09030B9317DD544B03EBCA030B
:103B000053E91223FCF7E4FC024638460F461646FA
:103B1000FCF764FC02460B4630463946FCF722FBB4
:103B20000F2CCDE9040100F3E1810B9B002B00F089
:103B300097820B9B40F3A782162B40F39A84C4F123
:103B400025030B9A934280F2DA84A4EB0A0616440A
:103B500016F00F000AD03D4901EBC001DDE9042356
:103B6000D1E90001FCF7B4FCCDE9040136F00F0304
:103B70004ED0B3F59A7F00F34684102B4FEA2316FC
:103B800040F3B285DFF8C8E04FF0000CCDF8289084
:103B90007746E246F146DDE9042316F0010F1046B0
:103BA00019464FEA66060AF1010A07D0D7E9002351
:103BB000FCF78EFC4FF0010C02460B46012E07F17C
:103BC0000807EAD1CE46DDF82890BCF1000F01D0FD
:103BD000CDE90423059B0EEBCA0E1E4EA3F15473D0
:103BE0000593DDE90423DEE90001FCF771FC1A4BC3
:103BF0000A460B40B342CDE9040100F204841749A0
:103C00008B4240F2FE844FF0FF33154ACDE9043277
:103C100000230A932346089A4146584600954CF0E3
:103C200053FE1590002800F0EE830B9A4FF0000A27
:103C30000C9B002ACDF820A0A9EB0303A8BF00230A
:103C40000C9322EAE2731493E2E000BF200E070017
:103C5000F80D07000000A07C0000F07F0000907CC1
:103C6000FFFFEF7FD21A1F2AA4EB020400F3C682E3
:103C7000012300259340984626443C440A9BA742D2
:103C80001E443B46A8BF2346B342A8BF3346002B81
:103C900002DDE41AF61AFF1A0C9B002B00F3548283
:103CA000002C00F36A820B9B002B00F39D82002EF8
:103CB00000F38E82002F08DD51463A4658464CF0FC
:103CC000E9FF8246002800F08C824A461A9958463D
:103CD0004DF074F80890002800F08382089A0023C1
:103CE000D168D3600D9151464DF048F80028C0F2DC
:103CF000C584059F00F02284514608984DF0EEF9E6
:103D000000224FF0804304460D46FCF75DFE00287C
:103D100000F00A820D9B002B40F07C82049B002B5C
:103D200040F06183C7F31303002B40F0E6820022CA
:103D3000AB4B20462946FCF73DFE002840F0F583BA
:103D40002046A84B29460022FCF7C2FB03460C463E
:103D50000E90CDE9123401F100430F93A24EA34B14
:103D60003E409E42DDE90E4500F05B820A9B23B394
:103D7000B6F1D46F21D8DDE9127897A3D3E90023F7
:103D800038464146FCF720FEA0B141463846FCF7D4
:103D900039FE012838BF0120FCF720FB0D9BCDE93F
:103DA0001201002B40F0378301F100431690179366
:103DB000DDE9164505F1D6639D1BDDE9107838462F
:103DC00041464DF0ABF802460B4620462946FCF72B
:103DD0007FFB3A464346FCF7C5F90C46CDE90401A2
:103DE000814B2340B34203D10A9B002B00F08E820B
:103DF0001A9958464CF00CFD494658464CF008FDBF
:103E0000514658464CF004FD089958464CF000FDC8
:103E1000159C584661684CF0D5FC8146002800F09E
:103E2000E081226904F10C010C3002329200FCF7AF
:103E3000E1FE1CAB584601931BAB0093DDE9043453
:103E40001A46CDE9103423464DF0E8F81A900028C0
:103E500000F09C81012158464CF0E2FD824600288A
:103E600000F0BF811B9B002BC0F2AE810C9A149E08
:103E70009F180A9A1C9C9B1A5D4A2344C4F136047D
:103E8000013B9342FFF6EEAE012300259846F3E690
:103E900098F8013003F0DF03582B00F07582434699
:103EA0000133199393F800A0BAF1300FF8D0984677
:103EB000BAF1000F7AD001230A9383E5492B00F071
:103EC0001C814E2B7FF4E5AD4A4919A84EF07AF8D3
:103ED00000283FF4DEAD199B1B78282B00F07E8371
:103EE00045484EF07BF98046894663E0A4EB0A061C
:103EF0000B9B1E44002E3FF72BAE3FF489AE76425B
:103F000016F00F020AD03D4B03EBC203DDE90401BA
:103F1000D3E90023FCF706FCCDE9040136113FF498
:103F200077AE1F2E3FDC16F01003354F4FF0000C1C
:103F300018BF6A230A93DDE9042316F0010F104627
:103F4000194607D0D7E90023FCF7C2FA4FF0010C5D
:103F500002460B46761007F10807EED1BCF1000FC0
:103F600001D0CDE904230A9BA3B1DDE90401C1F32B
:103F70000A52C2F16B03002B0ADD1F2B40F3FA83B8
:103F80000020342B049040F321844FF05C730593A0
:103F90006A230A9300220023DDE90401FCF700FDF7
:103FA00000283FF437AE2223CBF800304FF0000852
:103FB0004FF00009079A0AB1199B1360099B002B67
:103FC0003FF46EAD09F100434046994649461FB0A3
:103FD000BDE8F08FAFF300800000C0FFFFFFDF41BE
:103FE0000000F03F0000E03F0000F07F0000E07FB5
:103FF00002FCFFFFCCBE0700D8CB0700200E070055
:10400000E80E07004FF0010A23F02002452A7FF452
:104010002EAD44EA01030A9A13433FF43AAD199EC8
:10402000731C199373782B2B00F023812D2B3FF4F5
:1040300003AD4FF0000E04E5002219960C9218E52E
:104040001C9A03F2334304921D9A22F4801242EA2E
:1040500003530593210703D5059B43F000430593C4
:10406000DDE90489A6E70023099308F10103199308
:1040700098F801A0BAF1000F3FF40BAD98469BE40D
:1040800001230993F1E71633FFF630AF0C9BA9EB40
:104090000309B34B03EBC903DDE90401D3E90023B2
:1040A000FCF740FB8046894684E7A3F1300C0B9B6C
:1040B000581C19905B78A3F13002092A00F2D181D3
:1040C00001300CEB8C0C199003EB4C0C0378ACF129
:1040D000300CA3F13002092AF2D90B9A801A082871
:1040E00040F3BF8144F61F620C92BEF1000F3FF413
:1040F000C0AC0C9A52420C92BBE49A4919A84DF0FC
:1041000061FF00283FF4C5AC199B19A89649013BF3
:1041100019934DF057FF10B9199B013319934FF0C4
:104120000008DFF8489245E7914B204629460022D7
:10413000FCF7CEF90D9BCDE91201002B65D101F101
:1041400000430E900F9309E651461A4658464CF02C
:1041500047FD8246002844D001461A9A58464CF042
:104160008DFC00283DD00D9058461A994CF050FB1C
:104170000D9B002C1A937FF796AD22461A9958464C
:104180004CF088FD1A9000287FF48DAD4F4605460F
:1041900022234FF00008DFF8D491CBF800302946F5
:1041A00058464CF035FB394658464CF031FB5146E9
:1041B00058464CF02DFB159958464CF029FB0899B0
:1041C00058464CF025FBF5E6149A0C9FD61A50E69B
:1041D0004946324658464CF05DFD814600287FF442
:1041E00069AD4F461A9DD3E74946149A58464CF09C
:1041F000F7FC814600287FF45AADF2E75D4AD31AF6
:10420000012202FA03F5904636E5DDE91234CDE9E4
:104210000E34A3E50023584CCDE90E34CDE9123419
:104220009CE5A7F15473514F0593DDE90445204601
:1042300029464CF073FEDDE90E23FCF749F92B46C5
:104240002246FBF78FFF4D4B0F409F42CDE9040103
:1042500040F2DD8003F15473DDE91001994202D18F
:10426000B0F1FF3FBDD04FF0FF33454ACDE90432F6
:10427000BEE54FF0000EFFF7E1BB089940460B92F8
:1042800045F084FB0B9A089048B10022534617462C
:10429000924615461146914614460892B4E6199B7B
:1042A000981819909B5C302B40F0278102461146EC
:1042B000013219921378302BF9D0C0F1010001447A
:1042C000A3F13102082A10D8DDF864800025A3F19B
:1042D000300A01F10109012440462F4605EB85050E
:1042E00000210AEB4505FFF7A3BB4FF000094FF093
:1042F000010A4C464F464D4686E60023214CCDE947
:104300000E3400231C4CCDE9123427E5DDE91256AA
:10431000C4F3130728463146FDF79CFCFCF7AAF8C6
:1043200002460B4628463146FBF71AFF049D0D9EB8
:1043300004462E430D46374343D107A3D3E9002358
:10434000FCF738FB00283FF453AD4F461A9DDDE9DA
:10435000048924E7AFF300809535A094FFFFCF3F99
:10436000200E0700C0BE0700C4BE07000000F07F9B
:104370000000E03FE2FBFFFF0000F03FFFFF9F7CFB
:10438000FFFFEF7F0000F0BF099B19A90294584678
:1043900001931AABB04A00931BAB4DF017FB10F022
:1043A000070504463FF402AE062D7BD1079A12B1F1
:1043B00008F1010313604FF000084FF00009FFF708
:1043C0006FBBA1A3D3E90023FCF7F4FA0028BCD10A
:1043D000204629469EA3D3E90023FCF709FB0028C9
:1043E0003FF406ADB1E7049B012B86D1002F84D1A9
:1043F0004F461A9C222325464FF000084FF0000933
:10440000CBF80030CBE62223CBF8003087E601F171
:1044100054740594E4E4DDE91234CDE91634C7E4BC
:10442000012900F0138204EB010E0EF1FF3CCDF8E0
:104430002CE003E04FEA4E05A4450BD0082C05EB19
:10444000850E04F10104F5D907EB8703102CD8BFC2
:104450005F00F1E7DDF82CE0082C894416DC744697
:104460003CE744F61F629445A8BF9446CDF830C09F
:104470003BE60B98794901EBC001DDE90423D1E962
:104480000001FCF725F88046894693E5BEF1100F40
:1044900074464FF00001DCBF07EB870702EB4707CC
:1044A000FFF7C6BA1A9A3AB135211CA84CF040FE63
:1044B00058461A994CF0ACF9013D1B9B042D3FF670
:1044C000C9AD01A252F825F041400000F1440000BE
:1044D000EB440000DD440000414000004FF0FF339A
:1044E0006FF00040CDE90430B4E55D4B0593B1E5D4
:1044F0001C9B04931D9B0593ACE50899E0E6C4F171
:104500000F04564D05EBC401DDE90423D1E9000198
:10451000FBF7DEFF0B9B1C1B05EBC405D5E9002355
:10452000FBF7D6FF8046894644E500234D4CCDE994
:104530000E3400234C4CCDE912340FE43B460D9869
:10454000C4464F46AE464949C3F31302DDE910891C
:1045500000285BD08A4200F0FB80B5BB049A1CEABD
:10456000020F35D04046494604934CF0D7FC0A9BD5
:1045700004460D46002B00F01F81049BC3F30A5331
:10458000C3F16B06002E40F36481394C002204EB2A
:104590000653FBF79DFF02460B4640464946FBF794
:1045A000E1FD1A9C8046894640464946314B00222F
:1045B000FBF78EFF0B4625468046034389467FF472
:1045C000EEAD2223CBF80030E9E51EEA030FC9D196
:1045D0001A9C0A9B2546002BE6D1E0E519A81CAAE7
:1045E00025494DF009FD05287FF47AAC1D9B43F069
:1045F000FF4343F4E00305931C9B0493DDE9048926
:10460000D8E402F154730593FFF702BB002A71D17D
:10461000DDE904452246002C40F0B4800A9A002AC5
:1046200040F0F08025F00044240D2405A4F580140A
:104630001A9D6FEA14536FEA035305934FF0FF334B
:104640000493DDE90489AAE59535A094FFFFDF3FD7
:1046500035E5AF350000E03FE4BE0700200E07005F
:104660000000F07F0000E0BF0000E03FFFFF0F0010
:104670000000F03F00005039D0BE07000D9B4F46B0
:10468000DDE90401DDE910890343A1D1C1F313037E
:10469000002B9DD121F00044240D2405B4F1D66FE8
:1046A000264695D9089A536913B91369012B8FDDF2
:1046B0000899012258464CF0EDFA514608904CF00A
:1046C0005DFB002884DD0A9B002BAFD0A6F580138C
:1046D0001A9C6FEA13536FEA035305934FF0FF33AD
:1046E0000493DDE904895FE74FF0000ADFF87CE11D
:1046F000FFF770BA002D48D1049A1CEA020F3FF46C
:1047000067AF4046494604934CF008FC0A9B002BD7
:1047100040D0049BC3F30A53C3F16B06002E40F351
:10472000A280534C002204EB0653FBF7D1FE024655
:104730000B4640464946FBF713FD00220023804606
:104740008946FCF72DF900287FF453AE1A9C2BE71D
:10475000DDE904010A9A0446002A40D102460132EA
:104760006DD0BEF1000F7FF430AF14EA0C0F3FF4B0
:104770002FAFF7E64FF0FF3202FA03F3049A1A4024
:10478000049205E4BEF1000FB7D01EEA030F3FF418
:104790001FAFB6E702460B4640464946FBF7E0FC32
:1047A0001A9C00220023804689462546FCF7F8F82B
:1047B00000283FF4F4AC1DE6404649462B4622460D
:1047C000FBF7D0FC1A9D80468946E8E4C2F14B0213
:1047D0004FF0FF3393400B400593FFF7D9BB254AB9
:1047E0001A40B2F1D46F21D9611CBAD122498B424F
:1047F0003FF4F8AC02F58013059300230493DDE940
:104800000489E5E61B4E1E40B6F1D66F3FF65EAF5B
:104810001A9DB6F15C7F2C463FF6C6AE22234FF0C0
:1048200000084FF00009CBF80030B8E4100D4FF04D
:10483000FF31C0F16B0081408C4292D1DAE70E4A21
:1048400093423FF4CFAC01321A40D3E704F1010E9A
:1048500002E64046494622462B46FBF783FC1A9C5B
:1048600080468946A0E602460B4662E7F80D07003F
:104870000000F03F0000F07FFFFFEF7F000000002E
:104880002DE9F04F84468E4687B0002942D032A3EE
:10489000D3E9002332A7D7E9006733A5D5E900455E
:1048A0000FF2CC0BDBE900AB33A1D1E90001CDE97C
:1048B000042333A3D3E90023CDE9022332A3D3E9B0
:1048C0000023CDE9002332A3D3E900234FF00008F1
:1048D0004FF00009CCE90A01DDE90401CCE90C0143
:1048E000DDE90201CCE90E01DDE90001CCE91001AE
:1048F0000020CCE90089CCE90289CCE90467CCE945
:104900000645CCE908ABCCE91223CCF8D0E007B0DF
:10491000BDE8F08F20A3D3E9002321A7D7E90067E2
:10492000CDE9042320A5D5E9004521A3D3E900233F
:104930000FF2840BDBE900ABCDE9022320A1D1E922
:10494000000121A3D3E90023CDE9002320A3D3E96B
:104950000023BBE7AFF30080310BC0FF672633674E
:10496000D89E05C15D9DBBCB07D57C362A299A62AE
:1049700017DD70305A01599139590EF7D8EC2F15BF
:1049800011155868874AB48EA78FF9640D2E0CDB79
:10499000A44FFABE1D48B547D182E6AD7F520E51F5
:1049A00008C9BCF367E6096A3BA7CA8485AE67BB42
:1049B0001F6C3E2B8C68059B2BF894FE72F36E3CAB
:1049C000F1361D5F3AF54FA56BBD41FBABD9831F97
:1049D00079217E1319CDE05B30B58DB009F0FEF979
:1049E000014628B113480DB0BDE8304054F016B967
:1049F000114B5B7CDB0714D5104D02AC0FCD0FC4FF
:104A00002B6802A8236001230D49009303220D4B5C
:104A100009F0B2F9014610B10B4854F0FFF80DB09F
:104A200030BD0A4D07AC0FCD0FC42B6807A823601B
:104A3000E9E700BFDACD0700B5100020D00B070072
:104A40001812070010120700FFCD0700E40B070043
:104A500010B50446044854F0E1F82046BDE8104083
:104A6000052157F0D6BB00BF25CE070030B591B069
:104A70000FF092FB3C220021054601A843F02EFED8
:104A80000123124C237417F0D7FC637CA0B903F008
:104A9000FE03637429463C230D4801AA59F02FFCFC
:104AA00010B9019B052B0ADC637C23F002036374BD
:104AB0008023E37411B030BD43F00103E9E7637C68
:104AC00043F0020363749DF83C30F2E7B510002018
:104AD0000600565110B5FFF7C9FF03210123094A0B
:104AE000094808F0E5FF014610B1084854F096F86F
:104AF000BDE810404FF4203200230549054842F03C
:104B0000A3B800BF10120700181207004DCE07000F
:104B100078170020D817002070B503788AB00446B3
:104B20000E4607AD032B20D8DFE803F002191B1D4A
:104B30001149284644F0AEFC059563781E21049384
:104B4000A37830460393E3780C4A029323790193C8
:104B500063790093A37954F06EF80AB070BD0849E8
:104B6000E7E70849E5E70849E3E70A212846074A55
:104B700054F061F8E0E700BF79CE07009BCE070054
:104B800080CE070087CE070091CE0700FBFC070010
:104B900030B5154689B00C4657F0A9FB6946FFF7BA
:104BA000BBFF35B922466946054854F037F809B0CD
:104BB00030BD2B4622466946024854F02FF8F6E7EE
:104BC000BECE0700E1CE070010B50C4690B01046EF
:104BD0006946FFF7A1FF204608A9FFF79DFF6A4637
:104BE000024808A954F01AF810B010BD0ACF070007
:104BF00010B50C4688B057F07AFB6946FFF78CFF7A
:104C000022466946024854F009F808B010BD00BFBA
:104C10002ACF070000B589B057F069FB6946FFF756
:104C20007BFF6946024853F0F9FF09B05DF804FBC9
:104C300050CF070010B50C4688B057F058FB6946B6
:104C4000FFF76AFF22460A4C69460A4853F0E6FF1E
:104C50004FF4004200232046074941F0F5FF0022AF
:104C600000232046054941F0EFFF08B010BD00BF0A
:104C7000D81700206BCF0700A81700207817002056
:104C800000B589B029B10A4809B05DF804EB53F0CA
:104C9000C5BF57F02CFB6946FFF73EFF6946054844
:104CA00053F0BCFF044867F0D3FA09B05DF804FB89
:104CB00091CF0700B5CF07007817002070B5C6B0B8
:104CC000B822002118A843F009FD0FF065FA064646
:104CD0002022002110A843F001FD356800214FF487
:104CE000004042F0ADFA56480AF0A0F955480AF0E3
:104CF000B7F9002008F0F4F8014620B1524853F00B
:104D00008DFF46B070BD514853F088FF17F0AEFBE1
:104D1000044638BB4E4853F081FF4E4A2D69104679
:104D2000E97853F0D1FE901C297953F0CDFE101D87
:104D3000697953F0C9FE52F8020CD2F8021003ABA5
:104D40008DF8144003C303A808F0AAF8424B5B7C1B
:104D5000DB070BD4414D0BAC0FCD0FC42B680BA858
:104D600023600AE03E4853F059FFCAE73D4D06ACC8
:104D70000FCD0FC42B6806A82360012303220093E4
:104D800039493A4B08F0F8FF044610B1014638485B
:104D9000B5E7384853F042FFFFF768FE364867F042
:104DA00043FA05234FF4805234493348009441F0CC
:104DB000A5FE3349334867F03DFA3349334867F07D
:104DC00039FA00234FF4203230492B4841F00CFFD0
:104DD0002F4818A917F0F6FC219B002B91D02D48E5
:104DE00053F01CFF0DF161031093219B12948DF879
:104DF00044309DF860308DF84C408DF85730149455
:104E00008DF8544023B125AB1293459B8DF84C305F
:104E1000FF238DF85630249B3146C3F3C0038DF831
:104E2000553001231C488DF8583010AA202359F022
:104E300033FA011E01DA194861E7194893E700BF08
:104E40005808002048080020C6CF0700E7CF070019
:104E5000FFCF0700CB100020B5100020E40B0700A7
:104E600030D00700D00B07001812070010120700FF
:104E70006CD0070095D00700D8170020B858002044
:104E8000D9490000A8170020D54A00007817002053
:104E9000AB8A0500BBD0070002005651DFD00700E7
:104EA00012D107002DE9F04F91B0009302F00403F6
:104EB0000293C2F3C2030133840705460E46DDF8B0
:104EC00068800392059340F0BD81041D30B107292D
:104ED00009D86FF01B0011B0BDE8F08F01F0070694
:104EE000341DC6F10806009B4FF000094FF0040A7C
:104EF000591E4FF0FF334F460193CB465346CDF832
:104F000010900DB1009A22600598002800F3EB8004
:104F10009948009A824203D398488242C0F0E380C5
:104F2000039AA4EB050E92074FEA9E0000F106815A
:104F30000F2F00F2B480002D00F0088107F140022D
:104F40000DEB020C019A0CF8200C0CF8102C0498B4
:104F500001300490EAE07A2860D84B280ED8472820
:104F60005CD829282FD8252855D057D820287DD07F
:104F70002338D0F1000B4BEB000B77E0A0F14C0C89
:104F8000BCF12E0F4AD8DFE80CF071494949494974
:104F90004949494949494C49494949494949495A6D
:104FA000494C4C5A5A5A714C6E497149184C18491F
:104FB0004983804C49494C49800000204FF0000B48
:104FC0004FF0040A39E00122A0F12A0C5FFA8CFCB0
:104FD00002FA0CFC1CEA0E0F48D11CF062502ED1D4
:104FE0001CEA020B42D0013C5444CAF1000C04EA12
:104FF0000C04002D61D0A3EB050CA4446645FFF41E
:1050000068AF002868D1042B47D158F8043B2360CF
:10501000042304342AE0019A013A01924FF0000B74
:1050200024E011F8010C6C2834D1002011F8023C66
:1050300083466C2BC4D14FF0080A5346D3E708F1DE
:10504000070828F00708073424F00704F8E802AB43
:1050500035B106982044B0423FF63BAFC4E900ABFF
:105060004FF0000B08344FF0080A534611F8010FB7
:10507000002878D0BBF1000F7FF46DAF2528F5D163
:105080004FF0010B019B013301934FF0040AECE751
:10509000584693E700208346A5E7082B02D06FF01F
:1050A000150018E708F1070828F00708F8E80223B8
:1050B000C4E9002308230834D8E768B9042B02D1D7
:1050C00008F10408A4E7082BE9D108F1070828F043
:1050D000070808F10808EDE7059A013A059258F823
:1050E000042B00920DE7039A900720D54FF0010C96
:1050F000A4EB050E4FEA9E00BEF5007FCFD20F2F26
:10510000CDD8F5B107F140020DEB020E019AC0B205
:105110000EF8200C0EF8102CBCF1000F3FF417AF66
:1051200060F07F000EF8200C09F101090137C5F18C
:1051300008024FF6DA7E0434069297E74FF0000C2F
:10514000DAE7BCF1000F01D00136EFE70298023632
:105150000028EBD10098CDE9063144F0E9FBDDE908
:1051600006310644E2E7631BB3F5806F97D23DB981
:10517000A6F10804E018AEE68C0407002415090027
:10518000029A9B0828602B709DF81030C2B1EB701A
:1051900085F80290B9F1000F05D0002208A8C5F1EA
:1051A000010C97420ED14FF0000AC5F101030DF139
:1051B000200801930DF1300B574512D1601B8AE690
:1051C0006B70E5E710F8013B190608D504EB0C0EEF
:1051D000764503F07F03FFF47CAE04F8013B013217
:1051E000DFE7B9F1000F03D098F90020002A17DBA0
:1051F000029BD3B11AF80B2004F8012B0022019B6B
:10520000981820448642FFF464AE98F80000009994
:1052100004F8010B20460392FBF7ECFC039A1444BC
:105220000AF1010A08F10108C6E798F8002055F8CC
:1052300022300093029B009845F8223044F078FB1E
:10524000421CDCE76FF00D0045E600BF2DE9F04F92
:1052500095B000AFBB61BB6F0446C3F3C003884683
:105260007A62FB6049B903784578807800EB830067
:105270002044454519D8A0EB0408E37894F802B01F
:105280007B61BBF1000F02D0BB6FD80716D47B69DE
:1052900053BB7B6A1BB141462046BA6998474546D5
:1052A00028465437BD46BDE8F08F461C304644F0D2
:1052B0003FFB0130304408F10108DAE723786268E7
:1052C0003B629B003B613B6AFA6104EB830A7B6AA9
:1052D000002B40F0018145460026D0460BEB0A0921
:1052E000C14553D1DA4413E0BB6F9907D1D5237878
:1052F0009A463B629B003B61636804EB8A0AFB6150
:105300007B6A002B7CD14546BBF1000F51D15E4634
:10531000BB6F13F0050F0CBF4FF0020B4FF0010BEA
:105320007B690AEB4309BB6F03F002037B62CA454A
:10533000B6D01AF8021B1AF8013C54F82380AB4B84
:10534000984502D3AA4B98453AD3FB68002B44D02A
:10535000F86953F0F8FB00283FD0E8468AB06A4667
:10536000A44B5361A44B9361FB69C2E9073140F23E
:1053700001339384A14B42F8103F00234FF4325184
:105380009F4801F00FFC023DC546D0E718F8013BED
:1053900054F8230044F0CCFAFB6F01303BB1D7F84E
:1053A00080309E423EBFFB6F23F816000136054455
:1053B00096E7BB6F13F004061CBF7E6ADA44A7E7CA
:1053C000FB6823B1F86953F0BEFB0028C5D1BB6F61
:1053D000DA0705D4A5EB0B05A9E77B6A002BA6D05D
:1053E000404644F0A5FAFB6F43B1D7F880309E42A7
:1053F0003FBFFA6F431C22F816300136054496E78A
:10540000BBF1000F6ED0BB6F13F004066DD0D94610
:10541000002607F140005A465146FBF7EBFB7B693B
:10542000DA445B007B607B690AEB4303BB60BB6FC4
:1054300003F002033B60BB68534558D1B96F6378F2
:10544000B86F890748BF002106EB030258BF4FEA37
:105450005901C507D2B200F19A8010F0040F14BFB1
:1054600048460020FB616270A070E1702046BA6976
:1054700039697B6A9847051EFFF612AF3B6A4946B9
:105480002370FB69BA6963707B6984F802B0E370CA
:1054900007F140007B6A9847B0F10009C0F2A48090
:1054A0003B69A8EB0B01C91A7B685046C91ABA6957
:1054B0007B6A98470028C0F2A5804FF0000BA944F2
:1054C00009EB000507F1300AB34562DB0021BA6938
:1054D00008467B6A9847E3E65E464FF0000907F10D
:1054E000300098E75E46D94699E7B14697E71AF843
:1054F000021B3E4B1AF8015C54F82500984202D377
:105500003B4B98421DD3FB6823B1F86953F01BFB5A
:10551000002890D13B68FBB909F1280307F1280264
:1055200009F1010003EB020C07F1500309F1020934
:1055300053FA80F00CF8101C5FFA89F900F8105C3F
:1055400079E7FB682BB1F86953F0FDFA00287FF486
:1055500072AFBB6FDB0709D506F1280307F12802FC
:10556000711C9E1806F8205CCEB264E7BB6F58072A
:105570007FF561AF09F1280307F1280209F1010164
:1055800003EB020909F8105C5FFA81F953E7002088
:1055900068E71BF80A3054F8239087F82F30FB6F28
:1055A000FBB133F81B800121BA697B6A07F12F0038
:1055B0009847002826DB0544B8F1000F06D148467D
:1055C00044F0B6F900F101081FFA88F84146484650
:1055D000BA697B6A9847002814DB05440BF1010B7C
:1055E00072E7D7F87C80DEE74D4659E68C04070069
:1055F000241509002AD10700D1D1070005000001B8
:10560000040A070005464BE60F2808B506D956F0F0
:105610008EF9092303604FF0FF3008BD044B03EB04
:105620004013D3E8AF3F002BF1D00020F5E700BFD7
:105630007808002030B50D49400100F108030B4403
:10564000D3E8AF2F82B1541ED3E8EF5F954204D167
:10565000C3E8EC4FBCF1000FF6D1F1D1012A01BF34
:1056600000230A180B50536030BD00BF70080020A3
:1056700070B504460D461646FFF7C6FF002809DB45
:10568000064B600145B11A185268AA4204D056F080
:105690004EF90660002070BD1858FCE77008002025
:1056A00070B504460E461546FFF7AEFF00280CDB2A
:1056B000074B610103EB4414626832601DB101F1D4
:1056C0000C021A442A60585870BD0020FCE700BF45
:1056D0007008002010B500244FF0FF334FF0FF3268
:1056E000144840F037FF144BD3E8AF2F7AB10134A0
:1056F000102C03F12003F7D156F019F917234FF0BE
:10570000FF3403600B4853F060FA204610BDD3E825
:10571000EF0F0130C3E8E10F0029F8D1074863011A
:1057200000EB4411C2504A600C33184466F0D6FBBB
:10573000E8E700BFB01200207808002070080020C1
:1057400010B404461046094B620103EB441499500F
:10575000606040B1C46834B10C32134410BC40F2F4
:10576000051253F023BA10BC704700BF7008002028
:105770002DE9F04104460F469046FFF745FF00280B
:1057800019DB0E4E640104F10C0535444FF0FF3275
:105790004FF0FF33284640F0DDFE33195B68305987
:1057A000424639461B6898470446284653F00DFA8E
:1057B0002046BDE8F0814FF0FF34F9E77008002083
:1057C0002DE9F04104460F469046FFF71DFF0028E3
:1057D00019DB0E4E640104F10C0535444FF0FF3225
:1057E0004FF0FF33284640F0B5FE33195B6830595F
:1057F000424639465B6898470446284653F0E5F927
:105800002046BDE8F0814FF0FF34F9E77008002032
:10581000F8B50546FFF7F8FE002819DB0E4F6C01BE
:1058200004F10C063E444FF0FF324FF0FF33304698
:1058300040F090FE3B195B6838599B6898470446D6
:10584000304653F0C2F92846FFF7F4FE2046F8BD73
:105850004FF0FF34FAE700BF7008002073B504462C
:105860000D461646FFF7D0FE00280DDB0849600103
:10587000009601EB44142B46095840F2011260686F
:1058800053F094F902B070BD4FF0FF30FAE700BF5B
:1058900070080020014B1860704700BF700A00209C
:1058A00030B5002587B0CDE903010446009503A972
:1058B0000548059500F090F9DDE904309842B8BF3D
:1058C000255407B030BD00BFF38B05002DE9F0472C
:1058D000058B04462807904611D4022905F00705D8
:1058E00040F0CD80204653F063FC78B10138218B25
:1058F000042811D8DFE800F0C3106D859500012958
:105900000CBF45F0100545F02005258388F311886C
:10591000BFF36F8FBDE8F08701F0070AAA4500F0DA
:10592000A6800027B9463E46A368002B00F0BD8044
:1059300041F00801218388F31188BFF36F8FA168BC
:10594000002900F0BB800D68002900F0B7803346C5
:1059500052462046D1F80480C047002D76D02B68EF
:1059600029461D46F0E701F007035A1F012A1BD8FC
:10597000002221F00701062B276889B2C4E9002222
:1059800009D13B4603E0628B013262831B68002B26
:10599000F9D141F002012046218353F009FC00288F
:1059A0007BD041F0200177E0042B0AD121F00701E0
:1059B00089B22046218353F0FBFB10B141F0200156
:1059C0002183218B01F0070AAA4550D00027B94650
:1059D000AAE7236921F0070141F00601062DD3F85B
:1059E000009021832DD1B9F1000F40D041F0080182
:1059F000218388F31188BFF36F8F20463949C84748
:105A000029E021F00701236941F0040189B2042D46
:105A1000D3F804902183E6D000274FF0040A3E46D5
:105A200082E721F00701236941F0050189B2052DC4
:105A3000D3F808902183D6D000274FF0050A3E46C0
:105A400072E700274FF0060A3E466DE72B4687E7D0
:105A5000B9F1000FD1D14FF02003EFF3118883F398
:105A60001288BFF36F8F238B23F008032383258BCA
:105A7000EA062ED525F01003238305F00705666995
:105A8000218B002EBFF66FAF00232768C4E90033D7
:105A900021F0070141F001012183218B4FF0000922
:105AA00001F0070AAA457FF43FAF002F9BD041F0D9
:105AB0000801218388F31188BFF36F8F002FC7D0AF
:105AC0003D68394633465246204653F09DFB2F46EB
:105AD000F4E7AB067FF51AAF25F02003238305F02A
:105AE0000705FFE63592050010B5094C0A449142BE
:105AF00000D110BD11F8013B58400309E35C0001DF
:105B0000C0B243401809205C1B01DBB25840EEE7ED
:105B1000FBD10700F0B5024601680A270020074EB6
:105B20000B461C780131355D6D0701D41360F0BD63
:105B300007FB0043A3F13000F2E700BFFDB407000C
:105B40002DE9F84F15469A46D378224A6F2B12F862
:105B500003B080460F460BF0030B29D024D8582BF6
:105B60000CBF10260A26DDF8289032460023404656
:105B70003946FBF707F8092AD4B21ED83034B045AD
:105B8000E4B277F1000709F8014D01D3D14511D8EE
:105B90002B789B0605D5082E15D1AB7843F008036A
:105BA000AB704846BDE8F88F03F0F703702BD7E7DA
:105BB0000826D8E780460F46D7E7BBF1010F0CBF98
:105BC00037345734DBE7102EEBD1AB7843F01003BA
:105BD000E6E700BFFDB407002DE9F04F8246174607
:105BE0001C46002597B00391387808B9284649E348
:105BF0007B1C2528049306D00399D0470028C0F2C7
:105C000041830135F0E11822002110A842F066FD21
:105C10007B78252B00F0A380002398469E469C4667
:105C20001846791C0E4611F8012B2B2A00F0C6806D
:105C300000F2BD80202A00F0C480232A00F0C48036
:105C40002BB19DF8483043F040038DF84830B8F14F
:105C5000000F05D09DF8483043F020038DF8483000
:105C6000BEF1000F05D09DF8483043F010038DF8C9
:105C70004830BCF1000F05D09DF8483043F00803D0
:105C80008DF8483028B19DF8483043F004038DF872
:105C900048309DF8483003F04401442903D16FF3A4
:105CA00086138DF848309DF848302A2A43F0800347
:105CB00009968DF8483040F08C809DF8493043F0CB
:105CC00001038DF84930731C1A782E2A0CBF01216C
:105CD00000219DF8492061F341028DF849200CD143
:105CE0005A1C09925A782A2A40F083809DF849204C
:105CF000023342F004028DF849201A786C2A00F031
:105D0000A48000F28680682A00F08C806A2A00F065
:105D1000A5804C2A00F0AA801A4612F8013B782B85
:105D200004928DF84B309DF8492000F217816D2BBD
:105D300000F2A980692B00F21181572B00F2BE807E
:105D4000412B03D0453B022B00F2088104229DF831
:105D50004A3062F302038DF84A300123CAE0BA1CCC
:105D600004928DF84B309DF84930DA0740F1FD8000
:105D700054F8049BB9F1000F07DA9DF84820C9F1E7
:105D8000000942F004028DF848205E0740F1F680D9
:105D900054F804BBBBF1000F80F2F5809DF8493048
:105DA0006FF341038DF849304FF0FF3BEBE02D2AB4
:105DB0000DD0302A7FF444AF012333E74FF0010CBC
:105DC00030E74FF0010E2DE74FF001082AE70120E0
:105DD00028E709A8FFF79EFE099BB3423FF474AF82
:105DE0009DF848201390C00F60F341028DF84820C1
:105DF0006AE709A8FFF78EFE9DF848301490C3F3B8
:105E0000400242EAD07262F341038DF84830099BA8
:105E100073E7742A26D07A2A7FF47EAF06219DF894
:105E200049200CE05A78682A9DF8492006D10121C2
:105E300061F3C6028DF8492002336DE7022161F358
:105E4000C6028DF84920013366E75A786C2A9DF81E
:105E5000492001D10421EBE70321F0E705219DF85A
:105E60004920ECE707219DF84920E8E7BDF84820E4
:105E700022F4F04222F0020242F4804242F0020296
:105E8000ADF84820DFE76E3BD9B201238B4040F2EA
:105E900082410B4238D113F0240F52D1D8075DD57F
:105EA00003219DF84A3061F302038DF84A3002F075
:105EB0007803A3F140014B424B411BE00120A3F1C9
:105EC0005801C9B200FA01F111F4624F7FF43EAFFC
:105ED00040F6010631421DD111F4043F3ED09DF839
:105EE0004A3060F3020302F07802402A8DF84A300B
:105EF00034D000239DF84820C2F340010B4363F3E4
:105F000041028DF848202EE702219DF84A3061F3C6
:105F10000203E8E702209DF84A1002F0780260F3DD
:105F20000201402A8DF84A1002BF9DF8481041F046
:105F300001018DF84810632BDBD1131E18BF01231C
:105F4000D8E703219DF84A3012F0780F61F302037D
:105F50008DF84A3014BF01230023CBE79DF8483069
:105F600043F001038DF84830C3E79DF94820002A2B
:105F7000ACBF4FF0FF39DDF84C9006E798077FF58E
:105F800013AFDDF850B00023CDE913339DF84A304C
:105F90009DF8491003F00703012BC1F3C30133D16E
:105FA000CB1E042B04D8DFE803F021464621210054
:105FB000236801294FEAE372CDE910321CD19DF923
:105FC0004030DA17CDE9103204349DF8483013F030
:105FD000030650D03A465046049B039953F0D0F93B
:105FE0000028C0F24F810544049FFDE554F8043BAE
:105FF000DA17CDE91032E8E70229E5D11AB243F306
:10600000C033CDE91023DFE7022B24D1CB1E042BB4
:1060100004D8DFE803F018101018180001294FF019
:10602000000254F8043B14D00229CDE91032CCD13F
:106030009BB21093C9E7073424F00704F4E8022365
:10604000CDE91023C1E754F8043B109300231193CA
:10605000BBE7DBB2CDE7042B08D1073424F00704FB
:10606000D4E900230834CDE91023AEE7032BACD1EB
:1060700054F8043BDDE79DF84B007828B4D862283B
:106080001CD825283FF4B8AD5828ADD1DDE9100162
:106090000DF13E03009312AA0AABFFF751FDBBF1CD
:1060A000000F074680F29780002F9DD00DF13E082B
:1060B000A8EB0700002E4ED001304CE063381528C5
:1060C00092D801A252F820F047610000AD610000B3
:1060D000E95F0000E95F0000E95F0000E95F0000A0
:1060E000AD610000E95F0000E95F0000E95F0000CA
:1060F000E95F000035620000D1610000F761000037
:10610000E95F0000E95F000021610000E95F000035
:10611000D1610000E95F0000E95F0000D16100008B
:10612000BBF1000F109F0ADB5946384643F0A4FC30
:1061300007EB0008002F3FF457AF00260BE038466E
:1061400043F0F6FBF4E700260120109B0DF129082F
:106150008DF828300AAF9DF84A3013F010020592EE
:1061600000F0838002305B06DDF84CB048BF149B22
:10617000584448BFC018B9F1000F40F390809DF813
:106180004820A9EB0009C2F380035007069300F1F1
:106190008680510679D53EB130460399D047002814
:1061A00070DB069B01351E4630226FE019075ABF8F
:1061B000C3F300135E012B26DDE91023002BBFF68D
:1061C00065AF524263EB43032D26CDE910235DE713
:1061D00000265BE700269DF848200DF13E03DB1BFF
:1061E0006FF386129B458DF848207FF65DAFABEBD1
:1061F0000303139358E7109880B30DF13E080AABE0
:106200000021CDF8008012AAFFF79AFCBDF84A30B1
:10621000BBF1000F03F0EF0343F4F04343F010032E
:106220000746ADF84A30D5DA00283FF4DDAEA8EBDA
:10623000000082E7109B07293FF6D6AEDFE801F0A9
:106240000C04060C08080C0C1D70CDE61D80CBE676
:10625000EA17C3E90052C7E61D60C5E6DFF8BC8057
:106260000646A8F10507052075E71A0748BF013063
:1062700079E71046079306920399D047DDE9062394
:10628000002804DA17B0BDE8F08F20224B461946EB
:10629000002903F1FF33ECDC4D4499466D1A2EB111
:1062A00030460399D0470028ECDB01359DF84A3091
:1062B000DA0601D41B0705D530200399D047002802
:1062C000E0DB0135059B33B103999DF84B00D047C6
:1062D0000028D7DB0135AB4405E030200399D047D7
:1062E0000028CFDB0135ABEB0503002BF5DC434683
:1062F0003A465046039953F043F80028C2DB054460
:10630000A944A9EB0503002B7FF76EAE202003996B
:10631000D0470028B6DB0135F3E700BF10D20700F5
:1063200008B54FF02002EFF3118382F31288BFF318
:106330006F8F04F041FC034852F070FC03F0C4FE80
:10634000FCE700BF11D2070010B5094B094C00F063
:106350001F024009012818BF234603EB8203D3F82C
:10636000002222F0E04242EA0172C3F8002210BD8E
:106370000028845000258450F8B54FF02003EFF337
:10638000118783F31288BFF36F8F0125214B224EB3
:10639000C3F8005502230321C6F8D0360020FFF7CA
:1063A000D3FF2846FFF7D0FF7E237F220024C6F8C4
:1063B0000C37C6F83C39194B2946C3F81821184A3E
:1063C0002120C2F8044EC2F8084E02F54822C2F855
:1063D0001041C3F82441C3F82C4103F5FF1303F522
:1063E0008053C3F8A042C6F80457C6F80459C6F84B
:1063F000005BFFF7A9FF2020FFF7A6FF2520FFF78E
:10640000A3FF2420FFF7A0FF87F31188BFF36F8F4E
:106410002046F8BD00100050004000500020005001
:106420000090035005232DE9F041224D00AF2C7858
:10643000DFF884800134B4FBF3F303EB8303E41A45
:106440005AF09CF81D4A1E4E1378E3B158F82430D8
:10645000C01A072817D833788BB96C4688B06A46BB
:106460001849516118499161032142F8101F4FF4F6
:10647000C451164800F096FB0123A5463370002056
:10648000BD46BDE8F08100214FF050233170D3F8B4
:10649000140138B1C3F81411D3F814312C700CB9AD
:1064A000012313702C785AF069F848F82400012071
:1064B000E6E700BF0A560020C83200200956002037
:1064C000085600203AD2070067D207005C0B07008D
:1064D00048B1054B054A1B68B3FBF2F35843044B24
:1064E00043F0010318477047780D002040420F0029
:1064F000F00D0700062807D10122044BC3F8002540
:10650000BFF34F8F20BFFDE7704700BF0040005032
:10651000F0B583B000AF381D3DF0B4F9284B984278
:106520004BD114F097FF041E15DA38793DF0B0F91D
:106530006D4688B06A46234B5361234BC2E906344B
:10654000042342F8103F00234FF401511F4800F08C
:1065500029FBAD462DE040F607031D4D7C71AE686A
:10656000FB8074687B6814B96FF05704E0E708217A
:106570002846184AA047041EDADB3369002BF3D003
:106580000122082128469847041ED1DB01233D79CA
:10659000114AAB40C2F804357879FE7959F0E3FF2F
:1065A0000E4B45F00045B600C0F880509D51002CC0
:1065B000BED120460C37BD46F0BD6FF01204B7E7E0
:1065C0000000AD0B7FD20700ABD20700640B0700C1
:1065D0003C060700256600000070015080A10250B3
:1065E00038B5049CC4F30725284614F0ADFD0021FE
:1065F0000A4BA20B02F0FC02C0F880109950012354
:10660000E4B2074AA3402846C2F8083514F040FF18
:106610002046BDE838403DF03BB900BF80A00250A5
:1066200000700150F7B5144683681B690BB1002256
:106630009847C4F30726304614F08EFD05463046D1
:1066400059F091FF0027104B220E9200C0F8807085
:106650009F50304614F078FDA20B0C4B02F0FC0268
:106660001344E2B242F000421A60094BC0F88020A5
:1066700005F13202009330463B460194520059F036
:106680007BFF03B0F0BD00BF80A1025080A002508C
:10669000E16500003CF0A2BF2DE9F0470446074643
:1066A0004FF00109DFF8508014B93846BDE8F08793
:1066B00094FAA4F5B5FA85F509FA05F32E0108EB6D
:1066C00005156FEA030A24EA03042B7B002BEBD0A9
:1066D00058F806301B694BB94644736804222846B3
:1066E000196807EA0A0700F049FADDE728469847E3
:1066F0000028D9D1F0E700BFA40B070030B5002275
:1067000089B00F490F4865F0BCFF00220023002428
:10671000CDE906230E230C4DCDE903344FF440722E
:106720002846CDE90144094B094900943FF06EFE2B
:106730000849284665F0BCFB204609B030BD00BFC3
:10674000596700003021002090180020296A0000BD
:10675000B8680020C3D2070001483FF0E7BF00BF80
:10676000D01300202DE9F04780461F480F4653F014
:1067700041F80646002830D000252846BDE8F087BD
:10678000237B73B12368DB680BB1204698472368ED
:106790001B69D3B9636804222046196800F0EEF93A
:1067A000013610344C45EBD3B8F1000FE5D0002D85
:1067B000E2D02846FFF770FF0546002FF7D00021F2
:1067C0004FF4A47040F03CFDF1E7204698470028C4
:1067D000E0D00AFA06F31D43E2E705464FF0010A4E
:1067E000024CDFF80C90DDE7EC320020A40B070030
:1067F000B40B0700014B53F82000704754120700F8
:1068000008B5034608462BB1044A136000F03EFC6D
:10681000002008BD6FF01500FBE700BF740A0020E0
:1068200010B5044C237813B903483FF07FFF0123D0
:10683000237010BD0B560020D013002010B5044665
:10684000064852F0D7FF3CB1054BD3E8EF1F0139A2
:10685000C3E8E21F002AF8D110BD00BFE4320020D7
:10686000E832002000200146034BD3E8EF0FC3E8D5
:10687000E21F002AF9D17047E432002070B5FFF71B
:10688000F1FF0546074C084EB44200D370BD636863
:106890005B792BB123685B6813B129462046984782
:1068A0001034F1E7A40B0700B40B070010B5044C3B
:1068B0000449204652F035FE034B1C6010BD00BF5A
:1068C0006011002040120700DC32002008B50023D0
:1068D000064A4FF400411370054A06481360FFF75B
:1068E0008FFFBDE80840FFF7E1BF00BF0C56002056
:1068F000E4320020F1970500014600220023014800
:1069000052F030BE60110020014852F0C9BE00BFF5
:1069100060110020024B0146186852F011BF00BF01
:10692000DC320020014852F03FBF00BF6011002060
:1069300070B5264B1878002847D0FFF7E5FF0546CD
:1069400070B1234BD3E8EF1F0139C3E8E21F002ADF
:10695000F8D1204C204EB4422DD32846FFF7DAFF61
:106960001E4B1F4C1B68002B19DD65F062FE4FF4B7
:106970007A72A0FB020302FB0131C30B43EA4143DD
:10698000D4E900209B1A40F2E9324FEAD13161EBA1
:106990000001934271F1000101D3FFF76FFFD4E9C9
:1069A000003213F57A7342F10002C4E90032BDE807
:1069B0007040FFF7B7BF63685B7923B1236829464E
:1069C00020461B6898471034C5E770BD0B56002061
:1069D000E8320020A40B0700B40B0700E4320020CB
:1069E0002821002070B50D4D297861B90120FFF7ED
:1069F000B9FE0B4C0B4EB44206D3FFF799FF0028AB
:106A0000FBD101232B7070BD63685B791BB12368D8
:106A100020469B6898471034EDE700BF0C560020D5
:106A2000A40B0700B40B070000212DE9F04708462E
:106A3000FFF798FE044648B340F267684FF000093C
:106A400040F032FC1A4B186030B11A4B1B68092B0E
:106A500002DD19483FF06AFE0025184FDFF858A004
:106A600044B12046FFF718FE044618B94FF0FF382E
:106A70004FF0FF39FFF75CFF064628B9B5B942462B
:106A80004B4650463FF078FE3546E9E74FF0FF3879
:106A90004FF0FF39D4E72B689B691BB100222846D1
:106AA000114698471035BD42F5D3E8E7044DFAE7A3
:106AB000E0320020E8320020D0130020B40B0700A1
:106AC000A40B070013B5184852F094FE174B1B781F
:106AD0007BB14FF02003EFF3118483F31288BFF3EF
:106AE0006F8FFFF725FF84F31188BFF36F8F02B01C
:106AF00010BD0F4B1B68002BF9D050B900220023AA
:106B00000C48CDE900234FF40042002340F072FE10
:106B1000EDE70A28EBD1074865F0BFFD064802B053
:106B2000BDE810403FF002BEE83200200C560020C5
:106B3000E032002030210020D013002010B5064B99
:106B400004461B6898472146A060044852F088FD1F
:106B5000BDE81040FFF7B6BF740A002060110020A6
:106B6000044A054B9B1AB1EBD30F34BF52F83100E6
:106B7000002070477C090700A40B0700084B10B4E5
:106B8000C31A44681B110133237143689A710122AF
:106B90004368196043685A7110BCFFF741BE00BFDB
:106BA000A40B07002DE9F04FC1F3CB448FB0C1F324
:106BB00049260D469046994605901734002E3CD044
:106BC0004FF0040B4FF00A0A002209AF31460BAB1D
:106BD0004046CDF808B00197CDF800A0CDE90B22D2
:106BE0000D920796FEF732FBC0F30903181920F047
:106BF000070080081E4663F352250693FFF77CFECC
:106C0000044678B10022069B10300B900C930D9235
:106C10004046CDE9017B0C4A0799CDF800A00BABAB
:106C2000FEF714FB66F352254B462A46204605998B
:106C30000FB0BDE8F04F52F00FBE24F007008008FF
:106C4000FFF75AFE0446EDE72D9805002DE9F04FB9
:106C500087B00446DDE9105ADDE912690F46934614
:106C60009846B6B31021334652460020CDF8009026
:106C7000CDF81490FEF716F90146174B04F00704FF
:106C80000BF0070BE40003EA412305F1170044EA87
:106C90008B141C430844114B20F0070003EAC54342
:106CA00080081C430391FFF727FE054640B13EB123
:106CB000334652460399CDF800901030FEF7F2F8B3
:106CC000434622463946284607B0BDE8F04F52F009
:106CD000C3BD3146D1E700BF00FE07000000F87FCA
:106CE0000EB403B503AB53F8042B014604480193DB
:106CF00052F0D9FD02B05DF804EB03B0704700BF5D
:106D0000CF980500CA0605D48B064CBF024903493B
:106D1000FFF7E6BF704700BF199B0800E0120900AB
:106D20002DE9F04F89B09A46DDE913739DF848B01C
:106D30000593159B04460D46169E06920493BBF1DF
:106D4000000F00F0858006F00803079352F06CFDF9
:106D500006F002090246002849D020468549FFF77F
:106D6000BFFF8046B9F1000F08D016F0440F40D1A4
:106D70002A4620468049FFF7B3FF804406F001030E
:106D800053B17E4B204653F82B207D4B7D49002A82
:106D900008BF1A46FFF7A4FF06F00803002B54D0E3
:106DA000794B204653F82B207849FFF799FF054689
:106DB000069B2BB11A4620467549FFF791FF054403
:106DC000BAF1000F05D0524620467249FFF788FFFE
:106DD00005444544002F49D1049B002B4FD1F307B4
:106DE00000F1C18031462046FFF78CFFB5E08046B8
:106DF000B8E7694B18680028BFD0684B4FF47A7920
:106E00001B684FF46161B5FBF3F5B5FBF0F300FBD4
:106E1000135509FB05F5B3FBF1F2B5FBF0FE4FF09E
:106E20003C0C01FB123100FB1E55B1FBFCF309FBCE
:106E300005F5B5FBF0F50CFB131120460091CDE9EB
:106E400001E55749FFF74CFF97E706F00805AFE764
:106E5000BAF1010F06D1002F65D1049B002B7CD025
:106E600000250CE0002FF8D04E485DE04E483B4630
:106E700022464E4951F036FE049B002B69D0DFF8C4
:106E80003081DFF83091049F3146102F204628BF13
:106E900010274FF0000AFFF735FF554546DC059BEC
:106EA000494620461A78FFF71BFF4FF0010A1AF0F7
:106EB000070F03D141462046FFF712FF57453CD943
:106EC000059B4946204613F80A20FFF709FF0AF1FF
:106ED000010ABAF1100FEAD14FF0000A20463649F4
:106EE000FFF7FEFE5246059B20469A5C334B995CA9
:106EF00011F0970F08BF2E223149FFF7F1FE0AF17A
:106F0000010ABAF1100F1DD01AF0070F03D1414644
:106F10002046FFF7E5FE57455246E4D84146204655
:106F2000FFF7DEFEEBE720485D46A0E7414620463E
:106F3000FFF7D6FE0AF1010AAFE720462149FFF725
:106F4000CFFEC4E7059B3B440593049BDB1B0493E6
:106F500099D1BBF1000F7FF442AF204609B0BDE8E4
:106F6000F04F52F0A7BC2046054A0649FFF7B8FE8D
:106F700038E700BFDDD20700E1D207006412070046
:106F8000D8D20700A1D608007812070006D3070060
:106F90000CD3070010D30700F4320020F032002099
:106FA000EAD20700FD980500CF980500A7980500D4
:106FB0008E10090015D307001BD30700FDB407008E
:106FC0006FDE08008C1009002DE9F0410F884B6836
:106FD00005460C4690468E6886B0C7F382175BB1B3
:106FE000134A9B1A43F3CF0100291FDB2078C0F31B
:106FF000C200FFF7B5FD0346214651F8102B60880B
:10700000C2F34922002A01EB020408BF0021C0F3A9
:10701000CB00CDE90308CDE9011400223146284612
:107020000097FFF77DFE06B0BDE8F0810023E3E79F
:107030007C09070042F20F7373B58B4228BF0B46E1
:1070400005680446052168460D4A51F0F4FD0646E0
:10705000636828460B225B680A4952F017FC636894
:107060003246694628465B6852F010FC63681B2272
:1070700028465B68044952F009FC02B070BD00BFAD
:10708000730A080039D307001DD30700002101232C
:10709000064A904206D8064A01B901231360054BFF
:1070A00018607047012140085B00F2E740420F0082
:1070B000F0320020F4320020014B002019607047AC
:1070C0000C3300200122024B02481A7052F0F2BB2E
:1070D0000E560020A81207000148FFF7ABBF00BF03
:1070E000A812070010B5064B0C461868FFF782FB84
:1070F0002146BDE8104003460F220248184700BF52
:107100000C330020A8120700F8B50D460446064FC0
:107110004618B44201D12846F8BD14F8011BBB68DB
:1071200001485B689847F4E7F40507002DE9F74349
:107130000F4606460821C06A52F07FFC80463C6834
:10714000DFF84890241A3C6004EA0905AC4203D8F1
:10715000002003B0BDE8F08308236A46214630468C
:1071600052F0DBFB0028F4D16946304652F06FFC48
:1071700040B1BDF80230BDF8042005EA090513440A
:107180001D443C60A4EB0804E0E700BF0000FFFFE3
:107190002DE9F04F89B0044600AF00F114084046D5
:1071A00064F09CFEA06A8368DB689847E062B0B92F
:1071B0006C4688B06A46974B5361974B4FF4C25167
:1071C00093610323954842F8103F52F033FC6FF06F
:1071D0001505A54628462437BD46BDE8F08FA06AB0
:1071E0008368DB6898470368013B1F2B04D96C4612
:1071F00088B06A468A4BDFE7A06A216807F114026B
:1072000059F0C7F820B16C4688B06A46854BD3E781
:10721000A5892DB1BB69B5FBF3F203FB125525B16E
:107220006C4688B06A46804BC6E7E389012B04D8D8
:107230006C4688B06A467D4BBEE7E36A3D6093F8D2
:1072400004A04FF0FF334FF0FF3240463FF082F989
:107250000821E06A52F0F1FBA9460646E3891FFACD
:1072600085FB5B4508D8E3894B4523D140463FF079
:10727000EBF96FF02C05ADE7A1892B04891B13FAFC
:1072800081F1524608232046396052F094FB78B1D0
:107290003946204652F04FFB09F1010908235246B6
:1072A000204639681FFA89F952F085FB0028DAD0A8
:1072B0000135D3E75B450BD1396808235246204698
:1072C000891B52F078FB18B93946204652F033FB3F
:1072D00039462046FFF72AFF054618B140463FF0E1
:1072E000B3F977E73B684FEA13494FEA094963600E
:1072F000C4F80890D4E9011399420FD3082320461B
:107300003A1D52F00AFB05460028E7D13B1D13F851
:10731000012B924549D10135082DF8D163683946D2
:107320001B0C1B0420463B6052F005FB52462046D6
:10733000A389396852F03FFB051ECFDB636800F07C
:107340008B804FF6FF7A06EB0309A3891FFA89F2B7
:107350009B1B9A42C7F8009041D36D4688B06A469D
:10736000334B4FF4C6515361324B2C489361032386
:1073700042F8103F52F05EFB2046AD46616852F085
:107380003FFB05460028A9D163682B4AA189134019
:107390000B44A3EB4603636013402046A36052F006
:1073A00038FC0546002D73D098E72046391D52F071
:1073B0004EFB626810B9921B62609BE73D89F988B9
:1073C000E06AC4F80890294452F037FB48449042E0
:1073D000A060F0D1002DEED06FF01C05A5E00823D1
:1073E0004946204607F10C0252F097FA054600285C
:1073F0007FF474AF204607F10C0152F028FB30B146
:10740000BB89534503D13B8A002B00F09480B144E3
:107410009BE700BF97D30700E7D407002C0A0700BB
:10742000BDD30700DED30700FAD3070012D407004C
:107430007FD40700DBD407000000FFFF5246204640
:107440005B1A52F0B8FA051EFFF648AF08D0E26AA0
:10745000A36812681344A360D4E901318B42EDD8CC
:107460006168A38901EB46029A429BD1DFF8009143
:10747000A36801EA0902934294D0204652F0C0FA70
:10748000054600287FF42AAF636803EA0903A36076
:10749000A389A288A3EB46039A4242D040463FF01C
:1074A000D3F80123E8468AB023746D46E289A389A4
:1074B0004FF005092E462F49DFF8BCA06961C5E9E8
:1074C00006A22B6246F8109F32464FF423512B48F8
:1074D00052F0B0FAC5466368AD46294A4FF42351CD
:1074E000C5E9052A1A0C9BB2EA612B623246234891
:1074F000C5F8109052F09EFAC546A368AD46214AE1
:10750000C5F81090C5E9052A1A0C9BB2EA612B62F6
:1075100032464FF42351194852F08CFA0025C546E3
:1075200058E6204652F060FB054640463FF08CF896
:10753000002DB6D04EE66D4688B06A46124B4FF429
:10754000C6515361114B0D489361032342F8103F1C
:1075500052F070FA636839461B0C20461B04AD4696
:107560003B6052F0E8F92046396852F049FA18E7D2
:107570000000FFFF39D40700E7D407002C0A0700FA
:1075800054D407006AD40700AAD40700DBD407004C
:107590002DE9F04F89B01D46037C00AF04469146AB
:1075A0007960B3B96C4688B06A46694B4FF4C251F2
:1075B0005361684B68489361032342F8103F52F0CF
:1075C00039FA6FF00C06A54630462437BD46BDE8B3
:1075D000F08FC26A0821104652F02FFA82462946DF
:1075E000104652F02AFAA3898046A3EB8A03AB42E5
:1075F000C0F0AB801DB1B9F1000F00F0A680636848
:10760000FB60204607F1100207F10C01D7F80CB01F
:1076100052F055FA06460028D6D13B8A7A68934242
:1076200005D06268FB689A42EBD1DDB9CCE7204611
:1076300007F1100152F00BFA0028F2D0788ABB8AC9
:1076400075B1AB420ED14FEA1B41090401442B46F0
:107650004A46204652F07CF9002803DC0646B3E790
:10766000002BB1D0B8F1000F3ED104F114033B6000
:107670004FF0FF324FF0FF3304F114003EF06AFF89
:10768000DFF8D8B0E3899E425CD0D4E9012308EB4F
:1076900003018A422CD37B83FF237A68BB773A832A
:1076A00007F11800BD8352F07DF92B464A46A168C8
:1076B000204652F04EFA29468246E06A52F0BDF961
:1076C000A2680244A260BAF1000F08D1204607F177
:1076D000180152F078FA002814BF8246AA4638688A
:1076E0003EF0B2FF56466FE7D0441FFA88F8BCE779
:1076F0000821E06A52F0A1F94FF6FF733B830023A3
:10770000BB8313187B83A38902EA0B021A44101A65
:10771000606007F1180052F045F907F118012046A2
:1077200052F051FA2046211D52F005F963682046B7
:1077300003EA0B03A36052F06CFA82460028CED114
:1077400001369FE76FF01B0AC9E76FF015063BE7AC
:107750007FD30700D1D407002C0A07000000FFFFE9
:107760002DE9F04F85B01E46037C00AF04468846E5
:107770009146B7F838A0ABB96C4688B06A46304B32
:1077800030485361304B4FF4C2519361032342F8A8
:10779000103F52F04FF96FF00C00A5461437BD466C
:1077A000BDE8F08F0821C06A52F047F9A389A3EB26
:1077B0004003B34240D30025D4F804B0C7F804B066
:1077C00055455946D7F804B008D963685B451ED1C2
:1077D0003B8943451BD06FF00100DFE7204607F1EE
:1077E0000802391D52F06BF90028D7D13B89434577
:1077F00007D1204607F1080152F029F908B10135F7
:10780000ADB262687B689A42DAD15946E0E7BB893B
:10781000002BE0D0AA45DED87889090CB3424FEAA4
:10782000014128BF334601444A46204652F075F8CC
:107830000028B3D1B889B1E76FF01500AEE700BFFB
:107840007FD307002C0A0700C3D4070098B500AF08
:1078500098B96C4688B06A46154B16485361164B6A
:107860004FF4C2519361032342F8103F52F0A9FA3A
:107870006FF01500A546BD4698BD836893B96C4668
:1078800088B06A460D4B0B4853610B4B4FF4C25105
:107890009361032342F8103F52F093FA6FF0040013
:1078A000A546E8E71B680BB19847E4E71846E2E70E
:1078B000F8D40700340A0700C0D507000DD507002B
:1078C000B0B500AF08B101B19AB96C4688B06A464C
:1078D000164B17485361174B4FF4C2519361032362
:1078E00042F8103F52F06DFA6FF01500A546BD4604
:1078F000B0BD84680CB1E56895B96C4688B06A463D
:107900000D4B0B4853610B4B4FF4C2519361032352
:1079100042F8103F52F055FA6FF00400A546E6E732
:1079200041F8040BE3689847E1E700BF2FD5070053
:10793000340A0700A2D507000DD50700B0B51346DD
:10794000044600AF98B96C4688B06A46204B21487F
:107950005361214B4FF4C2519361032342F8103F0E
:1079600052F02FFA6FF01500A546BD46B0BD006875
:1079700090B96C4688B06A46184B16485361164B4E
:107980004FF4C2519361032342F8103F52F019FAA9
:107990006FF00100A546E8E782680AB1956895B9DD
:1079A0006C4688B06A460E4B0A4853610A4B4FF446
:1079B000C2519361032342F8103F52F002FA6FF074
:1079C0000400A546D1E70A466168A847CDE700BF95
:1079D0005FD50700340A070091D5070074D507006A
:1079E0000DD507000020014B1860704700000720EC
:1079F00030B50C460E4985B00291D0F8AC11054661
:107A0000CDE9003100F1E0014FF0FF3320463EF0B8
:107A10009BF850B9012384F86430D5F8A83123B11C
:107A2000204605B0BDE83040184705B030BD00BF66
:107A3000B99E050038B50C461146054652F03EFA8F
:107A4000034638B92846044952F038FA0346002064
:107A5000236038BD0120FBE7180E09002DE9F04F27
:107A6000012381460569466885B005F55F77D7E84B
:107A7000EF2F002A03D1C7E8E13F0029F7D140F0FA
:107A8000B880B368B26A043B2632B3EB420F4FEAC8
:107A9000420126BFB3FBF1F3B3FA83F300234FF0A7
:107AA000010428BFC3F12003013B9C4005F5E478A5
:107AB00000F099801022082170689A4002EB44027D
:107AC000043099400932C5F86002063122F0030201
:107AD0000A44B16A01FA03FC510001EB4C01C5F8FC
:107AE0006412B16A994000EB4103C5F85832033380
:107AF000134423F00303C5F854327368C5F85C429D
:107B0000C5F850323C4B4046C5E9A963316800F0E6
:107B10001DFA044630BBD9F804A0D9F81090DAE970
:107B2000073409F5307B012B584608BF103C64F040
:107B30007BFB0023DAF8240030494FF4806201EB2C
:107B400080210093584623463EF0D8FF09F52C705B
:107B50002B4964F01BFBDAF8140083685C681CB9DD
:107B60006FF05704002137E04B46264ADAF8181028
:107B7000A04704460028F5D1DAF8140083681B6991
:107B8000002BEDD00122DAF818109847044600289F
:107B9000E8D11D4B2846C5F8A8311C4BC5F8AC31BF
:107BA0001B4B0393D5F810320293D5F80832CDE978
:107BB0000083D5F86832B26AD5F8781300F08EF9F0
:107BC00004460028CED105F1E0003EF06BF8002815
:107BD000C5F880030ADB0221384652F0A4F920469A
:107BE00005B0BDE8F08F6FF00B04BBE76FF0150434
:107BF000B8E76FF07704F2E70F9F0500B86B00203D
:107C0000F59E0500E99E0500D97C0000C79F050090
:107C1000579F05002DE9F84306464FF00109056915
:107C2000D0F8048005F55F77D7E8EF3F022B03D14A
:107C3000C7E8E29F002AF7D149D1264805F1400163
:107C4000F9F74EF820B16FF00F042046BDE8F88335
:107C5000204805F1B001F9F743F80028F3D1284690
:107C6000D5F8781352F0E2F9044670BB71683669B2
:107C7000486983681B6933B322468969984704467B
:107C800018BB06F53076494630463EF06FFF304669
:107C900005F5E47602F0DAFF3046D8F8001052F02D
:107CA00002FA044688B90146E822304640F016FD43
:107CB00021464FF4E272284640F010FD2146384636
:107CC00052F031F9C1E76FF057040221F7E76FF086
:107CD0007704BAE7180E090013B5044640B1002333
:107CE0000122CDE90032074BD0E909123DF0E0FE58
:107CF000A36E1B6823B1E06E02B0BDE810401847C8
:107D000002B010BD180E090013B5044608462169DB
:107D100001F55F71D1E8AF1F022910D193B1A0B175
:107D20000121CDE900311346D0E909123DF0C0FE32
:107D3000074B984208BF6FF00B0002B010BD6FF008
:107D40000F00FAE76FF04C00F7E76FF00100F4E77F
:107D50002EF8FFFF2DE9F74388461546066906F51C
:107D60005F73D3E8AF3F022B5FD1136823B96FF085
:107D7000150003B0BDE8F0831B78002BF7D0D6F8D0
:107D80007893B9F1000F33D106F5D8774FF0FF3271
:107D90004FF0FF3338463EF0DDFB30462A6801A93C
:107DA000FFF748FE019C1CB9384652F0BAF8DEE7EE
:107DB00005F10803A3666B6984F86490E366E463E5
:107DC00060B1384652F0ADF821463046236E2A683D
:107DD000FFF70EFE0020C8F80040CAE720222968FD
:107DE00004F1400041F014FE384652F09AF8F1E7F1
:107DF00030460F4952F062F804460028B7D005F12A
:107E0000080383666B69C063C366002380F864302F
:107E100020222968403041F0FBFD224601213046F6
:107E200000F03EF80028D5D0A1E76FF00F00A0E7E2
:107E3000180E09002DE9F04F05460E469046002722
:107E4000D0F8B0A085B0AAF5AE7421463046F8F758
:107E500047FFE0B9114BA4F1400B0293DAF8103060
:107E60003246CDE9008329464FF0FF335846AAF544
:107E7000CE793DF069FE60B97023012203FB0793C0
:107E800083F86420DAF80C300BB158469847703408
:107E900017B105B0BDE8F08F0127D6E729A005008E
:107EA0001FB5144690B18AB1012912D10A4B00F1D5
:107EB000E0010293D0F8AC31403201934FF0FF3330
:107EC000204600933DF040FE04B010BD6FF0150059
:107ED000FAE70020F8E700BF29A005002DE9F043EC
:107EE00087B00E46DDE90E811446DDE910251F46F8
:107EF00030B329B3DFF850C000F1E009002D08BF0E
:107F000065469EB9CDE9034400F5CE74204605963A
:107F100063F0E3FE03ABCDE900432A463B4641460E
:107F200048463DF0E5FE07B0BDE8F083002241463B
:107F30000E9248462A4607B0BDE8F0433EF002B82C
:107F40006FF01500EFE700BF357E0000F0B50E467C
:107F5000044689B000286FD001230246C363002382
:107F6000D0F89810364F403040F80C7C42F8301F63
:107F7000CDE901334FF0FF330093C36D62F04EFF44
:107F8000304A06AB92E8030083E8030018463CF051
:107F900025FC0546D8B904F134003CF0FFFB05464A
:107FA000A8B93946284805AA62F00AFF054670B903
:107FB000059B9A6872B10C33D4F89400C4F8A030D1
:107FC00052F063F8C4F8D40030B96FF00B052846BE
:107FD00009B0F0BD0346EFE7D4F8940052F055F82D
:107FE000C4F8D8000028F0D0D4F88C30D4F8A01011
:107FF000C4F8A8300423C4F8AC30C4F8C430022359
:10800000A362124BB4F89420D4F8D470C4F8B8101A
:10801000C4F8D010D4F89010236204F1A403A4F89B
:10802000B020C4F8A470C4F8C010A4F8C820C4F8E4
:10803000BC00A661E362CAE76FF01505C7E700BFA1
:10804000EBD50700F80B0700F5D50700E412070091
:10805000F7B507460E461446FDF73CFB051E17DB39
:108060003CB97B1E012B04D8022E16D0012E08BF6E
:108070000624F1B201ABA2B2B8B20DF0ADF8061E03
:108080000DDA284650F0A3FD53F051FC764206600D
:108090004FF0FF35284603B0F0BD1124E9E7002377
:1080A000019A13600198C366703063F091FF0198E4
:1080B000883064F064FA062C02D1019856F00CFD69
:1080C0002846024A0199FDF73BFBE3E70813070046
:1080D00037B5069D0446C3B90093002200230C491E
:1080E0000DF03EFC04F1700063F072FF04F18800B3
:1080F00064F045FA05F17000214663F096FF2046D2
:1081000003B0BDE8304056F0E7BC03B030BD00BF5F
:10811000E1A2050080B50B4B00AF8AB06A469B68B0
:1081200013620523084951610849C2E9061042F863
:10813000103F00234FF421510548FEF733FDBD46A3
:1081400080BD00BFA84A002063D60700F3D6070011
:10815000E40A070080B500AF88B06A46084B536157
:10816000084BC2E90630042342F8103F00234FF4C5
:1081700002510548FEF716FD6FF01500BD4680BDA3
:108180008ED60700E3D60700E40A07002DE9F04188
:1081900005460E461746104CDFF84080444507D38D
:1081A00053F0C5FB6A2303604FF0FF30BDE8F08158
:1081B0002368AB4200D063B93A4631462846A368EB
:1081C000984730B13A4631462846E368BDE8F04169
:1081D00018471034E2E700BF04090700240907002C
:1081E00037B505460DF0ECF8041E06DA53F09FFB98
:1081F000644204604FF0FF3006E0B5F89830C3F3F6
:108200008113022B02D0002003B030BD2B68002266
:1082100000932846002303490DF0A2FB041EF2DA66
:10822000E4E700BFE1A205002DE97F4300244FF4FD
:10823000C0384FF000092346CDE900890294064674
:1082400056F0CFFC051E08DA53F071FB6D42056055
:108250004FF0FF3004B0BDE8708333680022009314
:108260003046002303490DF07BFB051EECDB204666
:10827000F0E700BFE1A2050037B5054656F060FC07
:10828000041E07DA53F053FB644204604FF0FF30E2
:1082900003B030BD0022002328460449009556F063
:1082A00016FD041EEEDB0020F2E700BFD1800000C7
:1082B0002DE9F04104460F461646FDF70BFA051E60
:1082C00017DBE36E13F002080CBF4FF0FF32002201
:1082D000134604F170003EF0F5F9044690B92846C3
:1082E00050F075FCB8F1000F08D053F020FB0B23C1
:1082F00003604FF0FF352846BDE8F08153F017FBCF
:108300001623F5E7703063F0B8FEA0B190F837306F
:10831000990710D5E36E284643F00103E36650F059
:1083200056FC204651F0C2FF204656F0DEFB53F0CB
:10833000FEFA7123DCE7B4F898305A050DD553F0F6
:10834000F6FA71230360284650F041FC204651F0B4
:10835000ADFF204656F0C9FBCBE723F40073A4F829
:10836000983077B16EB132683846142A28BF14228B
:1083700004F12C01F8F73EFCA38D012B07D1082353
:10838000336021462846084AFDF7DAF9B3E7022BA5
:1083900001D11823F4E7284650F019FC53F0C7FA2E
:1083A00086230360D2E700BF081307002DE9F04FD2
:1083B00090464FF0FF3A4FF0FF3B0A228BB05B062E
:1083C00004460F46CDE908ABDDF85090079203D480
:1083D000C36E13F0020336D000263546CDE9086699
:1083E0002368002200932046002327490DF0B8FAA5
:1083F000B0F1000A33DB4FF0000B0DF11C0A2168CD
:10840000DDE90823B9F1000F33D0CDE90223159B34
:108410000491009342464B4639462046CDF804B0BD
:1084200056F0E0FC002821DADDE908230146CDE919
:108430000023204632462B46CDF808A051F09BFF82
:108440000028DCDA12E0052108AA0DF087FB4FF4C2
:10845000A020002164F0F3F806460D46C0E753F073
:1084600066FACAF1000303604FF0FF300BB0BDE8BD
:10847000F08FCDE9002302914B4642463946204613
:1084800056F056FCCEE700BFE1A205002DE9F04F03
:1084900093B000AF0546D7E91C683961BB61FA614A
:1084A000002A00F04B81B0F89830C3F38112022A01
:1084B00040F005814FF0FF334FF0FF32C7E908234A
:1084C000BB695C0603D4C36E13F002032CD00022F8
:1084D0000023C7E90823D7E908ABBB6905F170049D
:1084E00013F002037B6139D01022002107F1300024
:1084F00040F0F4F804233C6487F83D3001215246F3
:108500005B4607F130003FF0F1F900F10B020B2A56
:10851000814603D8A74B1341D90716D553F007FA64
:10852000C9F100030360A0E0042107F120020DF06F
:1085300015FB284607F1200152F0C1F8041ECADAE3
:1085400053F0F5F9644204608FE0204663F091FD3A
:10855000044648B953F0EBF90B23E3E752465B4678
:1085600020463EF0AFF8F3E7D0E903A9002E4AD049
:10857000B8F1000F47D0B5F89630D8F80050FB603E
:1085800056F007FE94F837305B09338094F83730A3
:108590005B09012B75D100221423072DC7E90C2399
:1085A00044D907F1300B594620460DF095FC05469D
:1085B00010B96FF068053BE02046796B56F04FFE2E
:1085C0000028F6D1204694F83A1056F048FE0028CC
:1085D000EFD1EA683B7B7260112B49D107F1280388
:1085E0003B63082359467B6320460DF075FC002849
:1085F000DFD003887380C4E903A93388012B43D1FA
:108600000823C8F80030204656F02CFFFE690546C6
:10861000864228BF064639693246204656F0B8FEE3
:1086200000283AD053F083F9692334E06FF0150540
:10863000C4E903A953F07BF96E466B4288B003602E
:108640006A465D4B53615D4BC2E90635042342F82F
:10865000103F00234FF401515948FEF7A3FAB546E5
:108660007B6913B9204656F003FD4FF0FF361EE03C
:10867000062B06D11423C7F828B0FB6207F12801A6
:10868000B2E76FF08505D3E7022B01D11823B8E7D5
:1086900053F04DF986230360E2E77B6963B9204616
:1086A00056F0E6FCBB6913F0200F18BF2E4630468B
:1086B0004C37BD46BDE8F08FC4E903A9F2E7012AB3
:1086C0003CD14FF0FF384FF0FF39BA6913F0010B7E
:1086D000C7E90C8902F4807803D153F028F9092303
:1086E00020E7C3F34103022B03D053F020F980238A
:1086F00018E7BB695B0602D4C36E9E0713D5002240
:108700000023C7E90C23D7E90C0163F098FF00268A
:10871000C7E9011005F1700AEB6E5C070CD52C68F7
:1087200053F005F90FE713F00503ECD1042107F12D
:1087300030020DF013FAE6E7D80701D50026B6E7B8
:10874000D7E90C32134307D0284607F1300151F026
:10875000B6FF041EFFF6F4AE504663F08AFC0446F2
:1087600050B9B8F1000F01D0002EA0D1EB6E59071F
:10877000D5D4DA07E2D4EDE6C3687B610369FB6018
:1087800056F070FEFA6983199A4238BF1346814643
:108790002EBF5B46A3EB060900233B603B694A46BC
:1087A0009919204656F0F4FD3B6858B153F0BFF8D4
:1087B0006923B7E67EF7FFFFB5D60700D2D60700DC
:1087C000E40A0700BA694E4412F002093BD17BB1BA
:1087D0000023002250463DF075FF94F837302046C4
:1087E0009B0742BFEB6E43F00103EB6656F040FC83
:1087F0003B6B7A6B013342F10002022B72F10002F3
:108800000ED33EF073FFBB68181A7B6863EB01015F
:10881000012871F100031BDA00220023C7E90C23B1
:10882000002E3FF479AFB8F1000F03D0FB69B342DB
:108830003FF672AFB9F1000F7FF439AF31462846E9
:1088400056F0F5FA33E77B69E360FB682361CFE715
:10885000C7E90C01E4E700BF2DE9F04F4FF0000835
:10886000A1B0CDE90401194610461D46144663F037
:10887000E6FEDDE9049B4746CDE906010CAB099312
:10888000CDF80C80BBF1000F20D1002F64D0B5F1E2
:10889000FF3F08BFB4F1FF3F17BF4FF47A734FF0AB
:1088A000FF34A4FB0334DB0B18BF43EA4444059BAD
:1088B0004FF4827200934146049B0398019451F057
:1088C000E2FC0646304621B0BDE8F08FD9F8000042
:1088D000002820DB0BAA0AA951F042FD0646D0B1C0
:1088E0004FF0FF324FF0FF330B9851F0DBFC20AB21
:1088F000019309AB00934FF481724B4631460A98BD
:1089000051F0C1FC82461AF1780F0B9808D100246F
:1089100051F0CAFC254609F108090BF1FF3BB1E70C
:108920001AF1120F0BD1039B1BB151F0BDFC0127B3
:10893000F1E70A9BB046039351F0B6FCF7E751F01C
:10894000B3FCBAF1000FE6DA52F0F1FFCAF100030E
:108950004FF0FF360360B5E754EA050310D0B5F1D8
:10896000FF3F08BFB4F1FF3F0AD03EF0BFFE069BB9
:108970001C1A079B63EB0105002DBCBF3C46254636
:108980004FF0000A09990CAF3A4BC91B89105943A3
:108990002B46224638463EF0A9FF00F10B030B2B75
:1089A000804604D8344E1E4116F0010604D052F021
:1089B000BEFFC8F10003CBE7B1460997DDE90478B3
:1089C000B8F1000F1CD1B9F1000F3FF47BAF002EBE
:1089D0007FF478AF54EA05033FF474AFB5F1FF3F7D
:1089E00008BFB4F1FF3FCDD03EF080FE069B1C1ABD
:1089F000079B63EB0105012C75F10003C2DA61E707
:108A00003868A7F806A000282CDB0BAA0AA951F0A9
:108A1000A7FC834618B92023FB80013622E04FF0E3
:108A2000FF324FF0FF330B9851F03CFC09AB594635
:108A300040F2031200930A983B4651F024FC83460F
:108A40000B9851F031FC1BF10B0F0FD0BBF1000F55
:108A500004D052F06CFFCBF1000379E7B7F9063090
:108A6000002BDAD1083708F1FF38A9E74FF00109E8
:108A7000F8E700BFCDCCCCCC7EF7FFFF2DE9F04F5F
:108A80008BB016461F460D461498C9B1D1F800E0C8
:108A9000C6B1D6F80090BFB1D7F800C04EEA0902BF
:108AA00052EA0C025DD0002101238846134226D0F1
:108AB000B8F1030F0ADD52F03AFF0C2303604AE0DD
:108AC0008E46E5E7B146E6E7BC46E7E713EA0E0F58
:108AD00014BF0124002413EA090F18BF44F0040452
:108AE0000DF1280A13EA0C0F0AEBC80A18BF44F06C
:108AF00002044AF8201C2AF81C4C08F10108013134
:108B000020294FEA4303D1D168B33A4A0468436845
:108B1000A4FB024102FB031183683748E41841EBD0
:108B2000E3710029BCBF00242146C90341EA544136
:108B3000E40320184FF000032E4A41F10001F8F73A
:108B400021F802460B46414602A8FFF785FEB0F128
:108B5000FF3F82460BD14FF0FF3420460BB0BDE8FB
:108B6000F08F9046D0E74FF0FF321346EBE715B198
:108B7000284651F006FF16B1304651F002FF17B1FA
:108B8000384651F0FEFE00240DF10809A3461FE00F
:108B9000D90706D52DB12946019351F001FF019B5C
:108BA00001345A0706D52EB13146019351F0F8FE33
:108BB000019B013413F01A0F04D01FB1394651F054
:108BC000EFFE01340AF1FF3A0BF1010B09F108093C
:108BD000D845C2D0BAF1000FBFDDB9F90630002B7D
:108BE000F2D09A06D9F80000D2D552F0A0FE09239F
:108BF00064E700BF40420F003F420F00014BDB68BB
:108C0000184700BF0813070037B505460CF0D8FB1E
:108C1000041E07DA52F08BFE644204604FF0FF300E
:108C200003B030BD2B68002200932846002303497F
:108C30000CF096FE041EEDDB0020F1E70DAA050006
:108C4000F7B507460E461546FCF744FD041E12DB39
:108C500015B9032E08BFFF25AAB201ABF1B2B8B215
:108C60000CF0BAFA051E0BDA20464FF0B0FF52F0B6
:108C70005EFE6D4205604FF0FF34204603B0F0BD4C
:108C80000022019B1A600198703063F0A1F9204620
:108C9000024A0199FCF754FDEFE700BF48130700B3
:108CA0002DE9F04D4FF0FF3A4FF0FF3B88B0DDF873
:108CB000408004460E461746CDE906ABB8F1000FDA
:108CC00009D152F034FE792303604FF0FF3420467F
:108CD00008B0BDE8F08D5B0603D4C36E13F0020349
:108CE00012D000220023CDE906232368002200933E
:108CF0002046002312490CF033FE051E09DA52F01B
:108D000016FE6D420560E0E7052106AA0CF026FF7D
:108D1000EBE7236820460493DDE90623CDE902232F
:108D200000230193119B3A4600933146434656F087
:108D300059F8041ECBDA52F0FAFD64420460C4E72D
:108D40000DAA05002DE9F04F1C4692464FF0FF3367
:108D50004FF0FF328BB00F4661060546CDE9002388
:108D6000159E03D4C36E13F002032DD000220023FE
:108D7000CDE90023DDE9008914F0020405F1700B50
:108D800030D01022002105A83FF0A8FC0423CDF824
:108D900024B08DF82130012142464B4605A83EF013
:108DA000A5FD00F10B020B2A804603D85B4B134153
:108DB000DA070ED552F0BBFDC8F1000303604FF097
:108DC000FF300BB0BDE8F08F6A4604210CF0C6FE00
:108DD000D0E7584663F04DF9804648B952F0A7FDF8
:108DE0000B23EBE742464B4658463DF06BFCF3E75E
:108DF0004FF00009D0F808B0BBF1000F0CD1D145FD
:108E000028BFD14639464A46404656F0C1FA48B1D5
:108E100052F08DFD6923D1E7BBF81030DBF804B0C8
:108E20009944E9E7149B002B52D0002E50D0142215
:108E300059460DEB02003FF051FC95F99A000BF0FA
:108E40005BF90546002843D00323ADF814300BF03E
:108E50003DFC069098F83830DB0627D598F8282096
:108E600008A88DF81F20082A28BF0822D8F8241047
:108E7000F7F7C0FEB8F83430ADF816302B685B7DDC
:108E8000032B08D10123284608F12C0205A9ADF8CF
:108E90001C3051F0DFFD32681498142A28BF1422C8
:108EA00005A9F7F7A7FE1423336011E02B685B7D5B
:108EB000032BF0D1D8E903A7404656F06AF9D8F859
:108EC0000820D36813B1128A0D2A07D8C8E903A76E
:108ED000404604BB56F0CCF8484672E706228DF8AF
:108EE0001F20D3F80600039308905A892846ADF84E
:108EF00024209A8940F2063352BAADF81620012296
:108F000005A9ADF81C2003AAADF8103051F0A2FD60
:108F1000C8E903A7BFE756F03CF9DDE77EF7FFFF9E
:108F200013B5049C43B13CB1074CE46AA4460194D8
:108F300002B0BDE81040604752F0F9FC1623036010
:108F40004FF0FF3002B010BD0813070010B4024C00
:108F5000246BA44610BC60470813070008B5002224
:108F60000449FCF785FB20B1BDE80840203063F0E0
:108F7000E6BD08BD88130700002208B50349FCF7C9
:108F800077FB003818BF012008BD00BF8813070019
:108F900070B50546C0B30068431C1AD1002634469C
:108FA00028464FF0FF33002140F8603B51F0F0FDC0
:108FB00041F27002002128463FF090FB284663F002
:108FC000F0FD0CB306B304F10800BDE8704051F0A9
:108FD000DDBD00220D49FCF74BFB04460028DDD027
:108FE0004FF0FF324FF0FF33083051F0CDFD014616
:108FF00040B920464FF0FF3340F8503B51F0C8FDD8
:109000000126CDE70026CBE770BD00BF881307001F
:109010002DE9F04F0E46174605468DB008B101B157
:109020004AB952F084FC162303604FF0FF352846FE
:109030000DB0BDE8F08F00F1080800230022404683
:1090400051F0A2FD6B68002803F0010917DAB9F1AD
:10905000000F03D052F06BFC0B23E5E74FF0FF321B
:109060004FF0FF33404651F08FFD041E04DA52F0FA
:109070005EFC64420460D8E76B6803F001090022DB
:109080005C492868FCF7F4FA044618B952F04FFC22
:1090900020230EE000F1080A00220023504651F080
:1090A00073FD002836DAB9F1000F04D052F03FFC0E
:1090B0000B23036070E04FF0FF324FF0FF33504658
:1090C00051F062FDB0F1000904DA52F030FCC9F150
:1090D0000003EEE72868FFF741FF70B3002200238A
:1090E000CDE9022301233A460093314607AB04F150
:1090F00020003EF05DFD2868FFF730FF18B904F14D
:10910000600063F016FC012104F1500051F040FDB5
:10911000079D0DE02868FFF721FF0028DED1B9F197
:10912000000F0AD052F003FC0B234FF0FF35036011
:1091300004F1080051F02AFD30E062F0B3FE00288F
:10914000F0D14FF0FF3B0590DDF81490CDF818B04A
:1091500004F1080AB9F1000FC0D11022494607A84E
:109160003FF0BCFA01219DF82930504661F3050318
:1091700060348DF829300B9451F008FD4FF0FF3228
:109180004FF0FF33012107A83EF0B0FB041E09DABF
:1091900052F0CDFB644204604FF0FF35404651F081
:1091A000F5FC44E74A4613492868FCF761FA04468F
:1091B00000283FF46BAF4FF0FF324FF0FF33083021
:1091C00051F0E2FCB0F10009FFF67FAF06AA05A955
:1091D00004F1600063F0B0FB059B002BB4D0069B4C
:1091E0001BB1012B3FF47AAFAEE752F0A0FB202376
:1091F0009BE700BF881307002DE9F7430D4616468D
:10920000044648B952F093FB16234FF0FF34036035
:10921000204603B0BDE8F08300F108074FF0FF32AD
:109220004FF0FF33384651F0AFFCB5F5817F35D0B4
:109230000AD8032D1ED0042D24D052F078FB5F23D2
:109240004FF0FF34036019E040F203139D42F4D164
:10925000D6E90058AE8816F0040609D02068FFF75A
:109260008BFE0646002874D1EB8843F01003EB8098
:10927000B14685E06468A40304F48044384651F0A4
:1092800085FCC5E732686368510404D543F00103E7
:1092900063600024F2E723F00103F9E7D6E9005800
:1092A000AB88B668DA070DD52068FFF765FE0028A1
:1092B00000F0A180D8F800309E4200F09F8004F1B9
:1092C00050021A61AD8815F0040540D02068FFF700
:1092D00053FE0546002800F08E80D8F800309E42EC
:1092E00000F08C80002247492068FCF7C1F94FF05C
:1092F000FF3206464FF0FF33083051F045FC041EA4
:10930000BCDBD8F8003006F160021A610121D8F800
:1093100000305A7B61F305025A73D8F800309A7B0B
:109320006FF345129A73D8F80030DA686FF394320D
:10933000DA60D8F800301433C8F80030002EA8D016
:10934000002DA6D006F1080051F020FCA1E72E4622
:10935000DCE700222B492068FCF78AF94FF0FF3246
:1093600081464FF0FF33083051F00EFC002821DB1E
:109370002068FFF7F3FD78B1EB8843F00403EB803E
:10938000AB88DB0728D52068FFF7F6FDA0B9EB888E
:1093900043F00103EB801FE00090694601AA09F148
:1093A000600063F0C9FA009B002BE9D0EB8843F022
:1093B0001003E4E70026E3E704F1200063F0A2FBDA
:1093C0000028E4D10090694601AA04F1500063F03E
:1093D000B3FA009B002BDAD1D8F800301433C8F868
:1093E0000030B9F1000F3FF454AF002E3FF451AFFD
:1093F00009F10800A8E76FF077043FE76FF00B046E
:109400003CE700BF881307002DE9F3471E46002301
:1094100006281546CDE9003309D052F088FA6A23B0
:1094200003604FF0FF35284602B0BDE8F087012900
:1094300003D052F07CFA6B23F2E71AB152F077FABC
:109440007B23EDE71EB952F072FA0E23E8E7E846F7
:109450001746DFF8C89041F2700063F0A9FB04469C
:1094600090B952F064FA0C23036002AB03EB870758
:10947000002347F8083C0098FFF78AFD0198FFF7A2
:1094800087FDCEE70127E6E741F2700200213FF0B9
:1094900025F920464FF0FF3340F8083B01221146E2
:1094A00062F0EFFD4FF4805204F1700104F12000EE
:1094B00063F0F5FA04F1500063F036FA04F1600A43
:1094C000504663F031FA0121504651F061FBFCF740
:1094D00001F903460133206007D152F028FA17231F
:1094E00003602046FFF754FDBFE74A462146FCF7DC
:1094F00027F948F8044B002FC4D0DDE900473B684A
:1095000022683A6044F8083B2046336051F03EFB45
:109510003B682046736051F039FB84E788130700ED
:1095200070B5114B0D461C68DCB1104B1968002357
:109530008B4202DB6FF0010070BD224612F8106B07
:10954000864202D014460133F2E7E06810B96FF0AA
:109550001200F1E762F0D7FB0028F8D000202C6061
:10956000EAE76FF00C00E7E7BC0A0020C813070029
:1095700070B588B005460C46C0B269461646FFF77E
:10958000CFFF00281BDB0098C8B143682268029314
:1095900083680195CDE903360023CDE906230593C1
:1095A000C56851F005FC6DB12846084901AA56F07E
:1095B000F4FE079808B9059B236008B070BD6FF0F2
:1095C0001500FAE76FF01200F7E700BFB3AD050032
:1095D0002DE9F0410F4B05461C680E461746ACB10D
:1095E0004FF0FF324FF0FF330B483CF0B3FF63689E
:1095F0003246D3F8088029463B462046C0470446F9
:1096000005483DF021F82046BDE8F0816FF00104E7
:10961000F9E700BF10330020281300200023036067
:10962000044B5A6812B9C3E90000704710605860D3
:10963000704700BF14330020014B1860704700BF13
:10964000103300201FB5CDE9010103924FF0FF3325
:109650004FF0FF3209483CF07DFF094B1C682CB9E4
:1096600006483CF0F1FF204604B010BD6368204678
:109670001B6801A998472468F1E700BF2813002060
:10968000143300200022024BC3E90022704700BFC0
:10969000143300200022024BC3E90022FFF7F2BF7F
:1096A0001C3300202DE9F74307460C4609B100237F
:1096B0000B6000261E4DDFF87C904D450FD31E4BEE
:1096C0001D6885B355F8148C3846414601AA143DEF
:1096D00051F095FB10B3D6B914BB2E461EE0D5F859
:1096E00000803846414601AA51F089FB50B116B9B5
:1096F00054B92E4606E000224046316851F07FFB07
:109700000028F5D11435D8E7019B2360F1E700224A
:109710004046316851F073FB0028DDD16D69D0E718
:10972000019B2360D9E7304603B0BDE8F08300BF5A
:10973000B40B0700C80B07001C3300202DE9F047CD
:1097400084B002AFD7F8289004460D4616469846D6
:109750007860B9F1000F07D0D9F8001041BBD9F8F3
:1097600004A0BAF1000F2AD12046391DFFF79AFF55
:1097700018B3D0F808904346324629467868C8475F
:10978000D8B16D468AB002AA134B10625361134BD5
:10979000C2E9063440F201339384114B42F8103F82
:1097A00000234FF431510F48FDF7FCF9AD4604E0BA
:1097B0003A1D51F024FB0028D1D1002007E0D9F850
:1097C000083032460093294643467868D047083728
:1097D000BD46BDE8F08700BF26D707004FD707007A
:1097E00005000001540B070038B50C4D4FF0FF3356
:1097F0004FF0FF320A483CF0ADFE2B783BB9FFF743
:1098000049FF00F06DF8044610B901232B700024C5
:1098100003483CF019FF204638BD00BF0F5600201A
:10982000281300202DE9F04780468946048FDFF891
:10983000ACA0013498B0A4B200F10806651EADB228
:10984000B5F5004F47D04A23294605AA304650F0C7
:10985000B1FA04F57F543F34A4B2074621460123F0
:1098600030460DF10B0250F0A5FA002F014603DC43
:10987000002803DC2C46E1E7002816DCB8F8383075
:10988000AB4209D142466B1E22F8383F4FF40041EB
:1098900002233046FDF77CFE2946304650F086FA1A
:1098A0002146304650F082FAE4E707F160030DEB01
:1098B00003070023524607F84C3C05A8CDF800905A
:1098C00003AB0396ADF81040FFF738FF0028D1D066
:1098D00018B0BDE8F0870020FAE700BF4BAE0500E6
:1098E0007FB50125694628460195FFF719FE044614
:1098F000002834D1284602AA01A9FFF739FE10F149
:10990000130F04462BD038B10C3405D0404080F3FF
:1099100011884FF0040002DF0399B1F5803F23D294
:1099200000231846009A9468084484421AD30133ED
:10993000082BF9D10E4DA982EB8253682846AB6003
:10994000D368EB6351F01BFB044640B9094E28462F
:109950006E60FFF763FE28466E60FFF76DFE2046DF
:1099600004B070BD9BB2E5E76FF02004F7E700BFDD
:1099700024330020A40A00202DE9F84305464FF0C7
:109980002003EFF3118683F31288BFF36F8F4FF03C
:109990000C090D4B0D4F1C68DFF834802CB986F391
:1099A0001188BFF36F8FBDE8F883D4E90123002D40
:1099B00018BF13462BB198F8142009FB02F2B85CCB
:1099C00098472468EAE700BF7C330020703300200A
:1099D000A84A0020012270B5164B1C7D04F01F031D
:1099E0009A40D043144B610903EB8103D3E8EF1F86
:1099F00001EA0005C3E8E65F002EF7D10A4213D062
:109A00000E4B0F4D8BB10C236343EA185178E85C81
:109A10004FF0D5FE0020FFF7AFFF0C235C4300237F
:109A20002A192B51C2E9013370BD83F31188BFF3AA
:109A30006F8FEFE7A84A002084330020BF9705000E
:109A4000703300202DE9F041324B07461D7D4FF069
:109A50002003EFF3118883F31288BFF36F8F0C2478
:109A60006C432D4B2D4E195D1A19002947D007CA9A
:109A700006EB040C8CE8070000221A5588F31188C5
:109A8000BFF36F8F0C236B43F05CF218A8B37B1C01
:109A900010D04FF400400021D2F808C0204C002321
:109AA000ECFB00411F4A2046F7F76CF80121381AF9
:109AB00062F09FFD3DF006FB0120FFF75DFF1A4BB2
:109AC0006A0903EB8203012205F01F018A40D3E8F3
:109AD000EF0F1043C3E8E10F0029F8D1134B3BB15E
:109AE0000C2303FB05F033185978305CFCF702FDBA
:109AF000FFF770FF3DF0FAFA0120BDE8F081014662
:109B0000284600F015F80028B8D007C8344484E887
:109B10000700B3E7A84A0020643300207033002018
:109B20003F420F0040420F0084330020F5640000E4
:109B30002DE9F04F85B00E4603A900F043F84FF42D
:109B4000004704464FF0000B1B4B039DD3F800A0C9
:109B5000431E1BB203EB4303DFF8608005EB830574
:109B600024B9A146484605B0BDE8F08FC446594621
:109B700068680023E0FB07C1114A6046F7F702F866
:109B8000C44659460190A8680023E0FB07C10C4A6F
:109B90006046F6F7F7FFBAF1FF3FA94601D08245CC
:109BA00005D9731CDED0019B1844B042DAD9013CC0
:109BB000A4B20C3DD4E700BFB80A00203F420F001A
:109BC00040420F0008B9024B0B600020704700BFF5
:109BD000C81307000449431E0F3013F8012F8A5C95
:109BE00083421A70F9D1704775D70700F0B5074660
:109BF000264E8DB001AD0C460FCE0FC50FCE0FC552
:109C000096E8070085E807003846002F39D0002C79
:109C100039D0381F0246214610344B780D781B048A
:109C200043EA0563CD7804312B4311F8025C8C4282
:109C300043EA052342F8043FEFD10421144C8A077C
:109C4000036916D1C3F30742A55C1A0EA25C42EA6F
:109C50000562C3F30725655DDBB2E35C42EA0542BA
:109C600042EA032221F0030330336B4453F82C3CC7
:109C7000534050F8042F013153402C290361DED1A9
:109C800001200DB0F0BD2046FBE700BF000C07002F
:109C900075D707002DE9F04F002703689DB00293A8
:109CA0004368DFF8BCA103938368DDE902460493AF
:109CB000C36805930369DDE904BE0693436907930E
:109CC0008369DDE9062C0893C36998460993089BCC
:109CD0000093CD590CAB2DBA5AF8049BDD514FEAD5
:109CE000F223A94483EAB213009D83EA72634B44D2
:109CF00025EA020502EA0C0985EA09052B444344DA
:109D000086EA0B054FEA743888EAB408254006EA6B
:109D10000B0985EA090588EAB4580437A844402F9E
:109D200003EB0E054344DE46DDF8008040F08880FA
:109D30004FF0100A4B490A9151460AF1010A0DF100
:109D4000700E0AF00F070EEB870757F8407C01F002
:109D50000F094FEAB748019788EAF71801F10E0793
:109D600007F00F070EEB870757F8407C09314FEAE1
:109D7000F74E8EEA774ECDF82CE001F00F010DF191
:109D8000700E0EEB81010EEB890959F840EC51F889
:109D9000401CBAF1400F7144DDF804E088EADE08A7
:109DA000DDF82CE041448EEA972E714405EA020862
:109DB0004FEAF52E2CEA050787EA08078EEAB51E5A
:109DC000DDF828808EEA756E774458F804EF49F87C
:109DD000401C77440F4400994FEA733E394484EAAB
:109DE0000607CDF828808EEAB30E07EA030704EAD7
:109DF00006088EEAB35E87EA080777440F4401EB52
:109E00000B0ECDF800C0B34622D10299394401604F
:109E100003991944049B416023448360059B3344A8
:109E2000C360069B73440361079B2B444361089BFB
:109E300013448361099B6344C3611DB0BDE8F08F87
:109E4000B346CDF800C0264694461C462A4640E755
:109E5000944626462A461C4675463B466CE700BF9C
:109E6000FC1307003814070010B50446C8B170226F
:109E7000002151F0B2F80B4B0B4A0C49C4E9002306
:109E80000B4B0C48C4E902130B4BC4E9040301203B
:109E90000A4BA36103F17453A3F52303A3F6924382
:109EA000E36110BD85AE67BB67E6096A72F36E3C7D
:109EB0003AF54FA57F520E518C68059BABD9831F95
:109EC00001484AF02FBE00BFFC14070038B5044615
:109ED00018B90F4B0F485B6898476168B1F5683F48
:109EE0000FD0B1F5680F0CD00B4DA94209D011F479
:109EF000686107D02146094861F0AAFF002323606A
:109F0000656038BD142220683EF0E8FBF8E700BF2A
:109F1000B80F002075D807002C5F5CA98838002096
:109F200008B560B34368B3F5683F0ED0B3F5680F6A
:109F300018D0144A934220D000684FF0FF324FF0FF
:109F4000FF333CF007FB58B115E001220368D3E86A
:109F5000EF1F002903D1C3E8E02F0028F7D10AD171
:109F6000002008BD0368084A1B7803F5807352F887
:109F70002330002BF4D00548F3E70548F1E76FF4F0
:109F8000E040EEE72C5F5CA900000350E98FFFFF83
:109F9000EA8FFFFF08B520B34368B3F5683F09D0E7
:109FA000B3F5680F13D0114A93421DD000683CF0FE
:109FB0004BFB14E000220368D3E8EF1F012903D113
:109FC000C3E8E02F0028F7D109D0094808BD0021D7
:109FD0000368084A1B7803F5807342F823100020B9
:109FE000F4E76FF4E040F1E70348EFE72C5F5CA98A
:109FF000E98FFFFF00000350EA8FFFFF10B5044612
:10A0000018B91D4B1D485B6898476368B3F5683FF6
:10A010002FD0B3F5680F2CD0194A934219D1236879
:10A0200003BB4FF0FF324FF0FF33214615483CF0A1
:10A030006BF908B923681BB90F4B13485B68984745
:10A040001422002120683EF049FB4FF468636360EE
:10A0500008E0B3F5683F0DD83A2B03D040F6BA625A
:10A060009342DED1206861F039FF636843F03A0320
:10A07000636010BD054AF3E7B80F002075D80700EC
:10A080002C5F5CA9883800209BD807003A00003A72
:10A0900008B5064940231422054861F0CBFEBDE80F
:10A0A0000840044904484AF005BE00BF8833002038
:10A0B00088380020041507001815070001491022F0
:10A0C0000A60704710ED00E072B6404080F31188DE
:10A0D000BFF36F8F01B5FCF7A5F9002802D0BFF3DD
:10A0E0004F8F30BFBDE8014062B6BFF36F8F70473E
:10A0F00072B6494081F3118801B5FCF793F9002845
:10A1000002D0BFF34F8F20BFBDE8014080F311881C
:10A1100062B670472DE9F84F82460C4600AF002921
:10A1200052D0D1E900126E468AB0A3686D464FF056
:10A13000060BA8462848DFF8A490C5E90823C5E91E
:10A140000691686148F810BF002342464FF4415120
:10A150002348FCF727FDD4E90312B5466369AD46F1
:10A160002048C5E90712C5E905096B62C5F810B0BA
:10A17000002342464FF441511948FCF713FDB54600
:10A1800088B0E3696D464FF0040BA846164AEB61B0
:10A19000C5E9052948F810BF002342464FF4015194
:10A1A0000F48FCF7FFFCB546A369AD460F4AEB61CB
:10A1B000C5E90529C5F810B0002342464FF4015106
:10A1C0000748FCF7EFFCB546214650463BF000FF40
:10A1D000BD46BDE8F88F00BFC8D8070073D9070097
:10A1E000440B0700FBD807002ED9070041D9070010
:10A1F00040B2002807DB01234109034A00F01F0099
:10A20000834042F82130704700E100E040B200286E
:10A210000CDB01220649430900F01F008240203375
:10A2200041F82320BFF34F8FBFF36F8F704700BFFC
:10A2300000E100E0054B420953F82220012300F021
:10A240001F0003FA00F01040704700BF00E100E07B
:10A2500040B2002801F10101ACBF00F16040064BA3
:10A260004FEA4111C9B2ABBF00F5614000F00F00E9
:10A2700080F800131954704714ED00E030BFFFF769
:10A28000FDBF00BF0B4A08B50B4B22F07F029A605E
:10A29000BFF34F8FBFF36F8FD3F8882022F4700283
:10A2A000C3F888203BF05AFF3DF0BAF800F042FCBA
:10A2B0003BF094FF0000000000ED00E00A4A0B496B
:10A2C00093680968C3F88C00C3F8901008494B687C
:10A2D00043F080534B60002383F31188BFF36F8FEB
:10A2E0009368D3F890007047A84A00208CB4070008
:10A2F00000ED00E014498A684FF030001044EFF39D
:10A30000098C80E8F01F202080F31288BFF36F8F44
:10A310000E4F4FF00066CA698A603E60D2F88C002A
:10A320000023C2F88C3080F3118802F1300090E8ED
:10A33000F01F8CF3098802F1000004B551F09EFA79
:10A34000BDE8044070470000A84A002004ED00E08A
:10A350001EF0040F0CBFEFF30880EFF30980816952
:10A3600011F8021C0229FFD001B551F078FA01BDA5
:10A3700042F8203C009B0B4942F81C3C019B21F019
:10A38000010142F8183C029B42F8081C42F8143CB8
:10A390004FF0807342F8043C0023203A0265C0F875
:10A3A0008C307047518C0500084B9860836E83F3A6
:10A3B0000B88104681F30988002163B681F3118868
:10A3C000BFF36F8F002200234EF042FCA84A00200A
:10A3D00001B572B60B4A906900281EBF0021916139
:10A3E00061F06DFD62B6EFF30580A0F110004FEA59
:10A3F000C0000549014409C99847BDE80140034927
:10A4000008470000A84A00206C06070011A40000BD
:10A41000074B9968D869884203D006494FF08052AB
:10A420000A6001B53BF09EFFBDE8014070470000A7
:10A43000A84A002004ED00E02DE9F843E84600AF0B
:10A4400088B006460D466A464FF003094D4B4E4C08
:10A45000536194614FF4C2514C4842F8109F51F03F
:10A4600011FA4B4BC5469B6ADB060CD588B06A4691
:10A47000484B4FF4C251C2E90534444842F8109F9A
:10A4800051F000FAC546424B9B6A18070ED5E846C4
:10A4900088B06A46404B4FF4C251C2E905340323E9
:10A4A0003A4842F8103F51F0EDF9C546DFF8E09028
:10A4B000D9F8283099072AD5E84688B06A46374B3C
:10A4C0004FF4C251C2E905340323304842F8103F2B
:10A4D00051F0D8F9D9F83430D9F82820C5461206F9
:10A4E00015D588B06A46D36104232D492748C2E9AF
:10A4F00005144FF4015142F8103F51F0C3F9C5461D
:10A500002EB1D9F8283023F08003C9F82830204B29
:10A510009B6ADE070ED56E4688B06A46214B4FF423
:10A52000C251C2E905340323184842F8103F51F0E4
:10A53000A9F9B546164B9B6A98060ED56E4688B0AB
:10A540006A46194B4FF4C251C2E9053403230F4840
:10A5500042F8103F51F096F9B54600200C4B9A6A2C
:10A56000D10658BF9A6A9A6A920642BF5A6A22F482
:10A5700000525A629A6A42F0FF029A622870BD46FF
:10A58000BDE8F8837CD907008FDD0700440B070086
:10A5900000ED00E096D90700CDD90700E4D9070007
:10A5A00000DA07001ADA07003DDA07002DE9F84360
:10A5B000E84600AF88B006460D466A464FF00309EC
:10A5C0004C4B4D4C53614FF4C25194614B4842F88F
:10A5D000109F51F057F94A4BC5469B6AD9040CD5D8
:10A5E00088B06A46474B4FF4C251C2E9053443482C
:10A5F00042F8109F51F046F9C546414B9B6A1A0537
:10A600000ED5E84688B06A463F4B4FF4C251C2E9C6
:10A6100005340323394842F8103F51F033F9C54659
:10A62000DFF8DC90D9F828309B052AD5E84688B0B9
:10A630006A46364B3148C2E9053403234FF4C25110
:10A6400042F8103F51F01EF9D9F83830D9F82820D7
:10A65000C546100415D588B06A46D36104232C4939
:10A660002648C2E905144FF4015142F8103F51F059
:10A6700009F9C5462EB1D9F8283023F40043C9F8AA
:10A6800028301F4B9B6A59050ED56E4688B06A4626
:10A69000204B4FF4C251C2E905340323174842F856
:10A6A000103F51F0EFF8B546154B9A6AD20518D510
:10A6B0006E4688B06A46184BC2E9053403234FF44E
:10A6C000C2510E4842F8103F51F0DCF8B546002068
:10A6D0000B4A936A43F47F4393622870BD46BDE8FA
:10A6E000F8839B6A9B04F2D56E4688B06A460B4B92
:10A6F000E2E700BF70DA070085DD0700440B0700C2
:10A7000000ED00E08ADA0700CDD907009FDA0700E4
:10A71000BCDA0700D5DA0700F4DA07003DDA0700F3
:10A72000F8B56D4600AF88B06A4603264D4B4E4CD7
:10A73000536194614FF4C2514C4842F8106F51F08C
:10A74000A1F84B4BAD469B6A9B010CD588B06A467D
:10A75000484B4FF4C251C2E90534444842F8106FE7
:10A7600051F090F8AD46424B9B6ADD010ED56D4627
:10A7700088B06A46404B4FF4C251C2E90534032306
:10A780003A4842F8103F51F07DF8AD46384B9D6A8B
:10A7900015F480150FD06D4688B06A46374B4FF4DC
:10A7A000C251C2E905340323304842F8103F51F04A
:10A7B00069F8AD4602252E4B9B6A18030ED56E46EE
:10A7C00088B06A462E4B4FF4C251C2E905340323C8
:10A7D000264842F8103F51F055F8B546244B9B6A85
:10A7E00059030ED56E4688B06A46264B4FF4C251C7
:10A7F000C2E9053403231D4842F8103F51F042F8E6
:10A80000B5461B4B9B6A9A030ED56E4688B06A46C6
:10A810001D4B4FF4C251C2E905340323134842F8DB
:10A82000103F51F02FF8B546114B9B6ADB030ED554
:10A830006E4688B06A46154B4FF4C251C2E90534E2
:10A8400003230A4842F8103F51F01CF8B546084A65
:10A850002846936A6FEA03436FEA13439362BD4647
:10A86000F8BD00BF10DB070079DD0700440B0700CF
:10A8700000ED00E02CDB070043DB070061DB070095
:10A880008FDB0700B1DB0700DADB0700F8DB07002E
:10A890002DE9F0478AB08A4B0446D3F8048000269D
:10A8A00000AFC8F3080586F31188BFF36F8F02F07D
:10A8B0007F43B3F17F4F13D102F00C03082B20D15B
:10A8C0006C4688B06A467F4B4FF4C25153617E4B51
:10A8D0007E489361032342F8103F50F0D3FFA54612
:10A8E000002634467A4B1C600023FB71EB1E092BBB
:10A8F00000F2C780DFE803F00AADB0A9C5C5C5C541
:10A90000C5B310074CBF0C460126EBE7E84688B0FC
:10A910006A464FF0030A6F4BDFF8BC915361C2F8EF
:10A9200018904FF4C25142F810AF684850F0AAFF97
:10A930000023634DFB71EB6AC5469A070DD588B0BD
:10A940006A46664B4FF4C251C2E9053942F810AF6E
:10A950005E4850F097FFC54691E0EB6A002B03DAA2
:10A9600088B06A465E4BEDE7EB6A5B0040F187809A
:10A9700088B06A465B4B4FF4C251C2E9053953486F
:10A9800042F810AF50F07EFF6B69A26943F4807308
:10A99000C5466B61BFF34F8FBFF36F8F6B6932F8A2
:10A9A000022C23F480736B61BFF34F8FBFF36F8F63
:10A9B0004DF602739A4208D0AB6ADBB2002B37D057
:10A9C0000120F91DFFF738FD41E088B023686A4691
:10A9D000D361042344493D48C2E9051942F8103FB8
:10A9E0004FF4015150F04EFFC5462368FA79DAB9A9
:10A9F00007F1080504F1200C2A4620686168083434
:10AA000003C264451546F7D17A6A002E52D0C2F3CC
:10AA1000080121B96FEA52226FEA42227A6218468F
:10AA200007F10801FFF776FB2837BD46BDE8F08740
:10AA3000AB6A13F47F4F04D00120F91DFFF7B6FD78
:10AA400005E0AB6AB3F5803F19D3FFF769FE034613
:10AA5000CCE70020F91DB5E70020F91DEEE76D46B3
:10AA600088B06A46214B4FF4C2515361204B1748BE
:10AA70009361032342F8103F50F004FFAD460023DA
:10AA8000B4E71C4A18F4F87FE8468AB01A4B18BF9E
:10AA900013466A461949103D516119491562C2E9C8
:10AAA000061340F201339384164B4FF4315142F8B0
:10AAB000103F4DE722F4FF7222F00102AEE700BF23
:10AAC00000ED00E055DC0700ABDD0700440B07009C
:10AAD000A438002084DC0700A0DD07009FDC07000D
:10AAE000C4DC0700D6DC0700F9DC070019DD07002D
:10AAF0006BDD07003CDC070027DC070041DD0700B9
:10AB000058DD070005000001044B5A6942F01002AD
:10AB10005A615A6942F480625A61704700ED00E060
:10AB2000EFF30880EFF3098101B57246FFF7B0FE3D
:10AB300001BD00BF002320210348C2180133452B6B
:10AB400082F80013F9D1704700E100E0002080F3A3
:10AB50001488BFF36F8F002080F30A8880F30B887E
:10AB6000FBF798FD002011490860BFF34F8F104894
:10AB700080F3088800F044F8202080F311880D4805
:10AB80004FF0AA014FF4006261F0C8F809484FF491
:10AB90000061401880F30988EFF314800221084314
:10ABA00080F31488BFF36F8FFFF76CFB94ED00E028
:10ABB000F8060120B8ED0020BFF34F8F0549064B82
:10ABC000CA6802F4E0621343CB60BFF34F8F00BF4B
:10ABD000FDE700BF00ED00E00400FA050023184681
:10ABE0000649D1F89020C2F30722934200DB704758
:10ABF000C1F89830C1F8A0000133F6E700ED00E09D
:10AC000010B572B6002484F31388FFF7E7FF2346DC
:10AC10004FF0FF300C4A03F120010133102B42F8B2
:10AC20002100F8D100234FF0FF30074A03F1600103
:10AC30000133102B42F82100F8D162B6BFF34F8FD9
:10AC4000BFF36F8F10BD00BF00E100E0084B9B68B1
:10AC500083420BD1EFF3058343B1064B5A6842F0B0
:10AC600080525A605A6A22F400425A623CF022BB77
:10AC7000A84A002000ED00E037B50546144B1868DF
:10AC80001B7900908DF8043005B3124C442200214A
:10AC900020463DF023FD2B68052123606B68684644
:10ACA0006360AB68A360EB68E3602B6923616B6949
:10ACB0006361AB69A361EB69E361074B1B682362C6
:10ACC00000F098FA4421204600F094FA03B030BD19
:10ACD000940D070010560020A43800201FB5094C21
:10ACE000094A23460121094800F034F9002303935F
:10ACF000074B0121E41A01A80193029400F034F9F2
:10AD000004B010BD00000720000000202815070037
:10AD10007817002010B50C7A0B6804F01F0223F09E
:10AD20001F031A43CB68640923F01F03054943EA54
:10AD3000440343F00103C1F89800C1F89C20C1F816
:10AD4000A03010BD00ED00E080B500AF88B06A46CD
:10AD5000084B5361084BC2E90630042342F8103F08
:10AD600000234FF401510548FBF71CFF6FF015005D
:10AD7000BD4680BDB7DD07002FDE07005C0A070077
:10AD80002DE9F04F144606464FF0000987B0614D9B
:10AD900000AF79607B68994539DAD6F80480B8F15C
:10ADA000000F58D0B8F11F0F1DD918F01F0F1AD17E
:10ADB000D6F800B01BF01F0F15D1584650F067FDB4
:10ADC000824608EB0B00013850F061FD824523D02C
:10ADD0006FF0150A6C4688B06A464F4951614F4979
:10ADE000C2E9061A07E06C4688B06A464C4B5361CC
:10ADF0004A4BC2E90639042342F8103F00234FF4BE
:10AE000001514848FBF7CEFEA5466FF015042046D9
:10AE10001C37BD46BDE8F08F1AF1160FDAD0544545
:10AE2000D8DDC5F898A0D5F89C00C5F898A0D5F84D
:10AE3000A02020F01F0042F01F08D6E90021114495
:10AE4000904201F1FF3B1ED1D84508D131465FFA4F
:10AE50008AF050F025FD09F101090C369AE7C5F892
:10AE600098A0D5F89C3021F01F0103F01F030B437D
:10AE70003146C5F89C30E0B250F012FD10F1160FCB
:10AE8000C3D0441CE7E7013AD845E0B222F01F02E4
:10AE9000C5F898A008D1D5F8A030314603F01F03BB
:10AEA0001343C5F8A030E7E7D5F8A01001F01F0163
:10AEB0000A43C5F8A020314650F0F2FC10F1160FFD
:10AEC000A3D0C5F898A0D5F89C203B7C08F1FF38AA
:10AED00062F304033B74D5F8A0303A7C5B0863F35B
:10AEE00047123A74D6E900321344BB6023F01F03C3
:10AEF000441C4344A3EB0B03E0B223F01F030728D9
:10AF00007B6102D9FFF720FFB8E707F10801FFF7DF
:10AF100001FFB6E700ED00E008DE070048DE0700AD
:10AF2000E1DD07005C0A07000522044BC3F894200A
:10AF3000BFF34F8FBFF36F8F704700BF00ED00E08E
:10AF4000BFF35F8F0022024BC3F89420704700BF0D
:10AF500000ED00E010B5034C2278FFF711FF2070E0
:10AF600010BD00BF545600202DE9F74F294D8A46E9
:10AF700006464FF00008AB46274FD0451BDAD6F8FF
:10AF80000490B9F1000F3FD031680846019150F0AC
:10AF90007EFC0199044609EB0100013850F077FC72
:10AFA00084424FF014021D4B08D002FB08F36FF0EF
:10AFB00015024BF8032003B0BDE8F08F14F1160F13
:10AFC0002C60F8D01978A142F5DD02FB08B0C7F873
:10AFD0009840C7F89840D7F89C4000F10801007BE2
:10AFE00064F304000871D7F8A0000C79400860F3FE
:10AFF00047140C71D7F89C1021F01F016960D7F835
:10B00000A01021F01F01296108F1010814350C3648
:10B01000B3E700BFA838002000ED00E05456002040
:10B0200038B50E4D2C68082C15D80020FFF788FF86
:10B030000B4B0C4AC3F8C020844205D10A4B0020B8
:10B040001C70FFF771FF38BD696801EB0011FFF755
:10B0500061FE0130F0E74FF0FF30F4E734150700F0
:10B0600000ED00E0AAFF440054560020014B186098
:10B07000704700BFE00A0020F8B50D46094F461E94
:10B08000C0F10104A3199D4201DC2846F8BD737884
:10B090000A2B02D10D203B6898473B6816F8010F38
:10B0A0009847EFE7E00A00200522012008B5024991
:10B0B000FAF786FBFEE700BF6CDE070010B5074C11
:10B0C0002368C2180648C0F1005101F5E0218A4208
:10B0D00036BF22604FF0FF30C01810BDBC380020D2
:10B0E000549E03201D2208B504490220FAF768FB8C
:10B0F000404080F311884FF0030002DF72DE07004A
:10B1000001282DE9F0410F4609D0042847D050F01E
:10B110000EFC162303604FF0FF30BDE8F0814FF0C6
:10B120002003EFF3118283F31288BFF36F8F224B5A
:10B13000D3E900689D6882F31188BFF36F8F61F0D7
:10B1400078FA4FF47A720446A0FB020302FB013145
:10B15000C00B4FF47A72002340EA4140C90BF5F767
:10B1600011FD4FF0FA7C8619A0FB0C0E48EB01088C
:10B170004FF47A7200230CFB01E1C7E90068F5F790
:10B1800001FD0E4A241AA4FB0243E40B44EA4344A3
:10B190000B4B25449D42BD6005D80020BDE700252E
:10B1A0002E46A846CBE7013648F10003AD1AC7E9A1
:10B1B0000063BD60F1E700BFF024002000CA9A3BA5
:10B1C000FFC99A3B1022044B0020C3F840244FF0E3
:10B1D0005023C3F81406704700300050014B1B6821
:10B1E000184700BFE40A0020014B5B68184700BF06
:10B1F000E40A002018B111B1014B9B681847704751
:10B20000E40A002030B5044685B0C0B1884216D2A9
:10B210004D238DF8043001238DF8053000238DF87F
:10B220000630084B0D1ACDF80700CDF80B1001A819
:10B230000B219B68984729462046FFF7DBFF05B0A6
:10B2400030BD00BFE40A00207FB50D460646144617
:10B25000FFF7C4FF44F25A53ADF804300123ADF8B0
:10B2600006304FF4A0230396029350F00EFB0D4BD3
:10B27000ADF808000C219B6801A8984715B1284635
:10B28000FFF7FAFC4CB1204604F19801FFF7BAFF32
:10B29000D4E91A010144FFF7B5FF04B0BDE87040DE
:10B2A000FFF7A2BFE40A002010B9034B18687047EB
:10B2B0006FF08500704700BFC038002010B9034B05
:10B2C000186070476FF08500704700BFC0380020DD
:10B2D000002298B50D4B00AF1A60FBF729FB04461E
:10B2E0000028FAD1FBF77EFB88B06A46084B536111
:10B2F000084B9361032342F8103F4FF4C251234699
:10B300000548FBF74FFCBD4698BD00BFC038002084
:10B31000B8DE0700FADE0700140A07002DE9F0473F
:10B320000E46044600AF00B121B96FF015020026A9
:10B33000224B1A60DFF88880DFF888906EB1002514
:10B34000207808EB050100094DF043FC0028A246D7
:10B3500006DA6FF01502194B1A60BD46BDE8F0879A
:10B360009AF80000691C58FA81F100F00F004DF0C6
:10B3700030FC002804F10104EBDB0235EDB2402D76
:10B3800006F1FF3601D0002EDAD1002308F805308F
:10B390006D468AB06A460C49C2F81490C2E9061894
:10B3A00040F201311184094942F8101F4FF4115144
:10B3B0000748FBF7F7FBAD46C0E700BFC0380020E9
:10B3C00055560020C7DE070036DF070004000001E5
:10B3D000140A0700B0B5124B124C1B6800AF7BB1CA
:10B3E0006D4688B06A46104BC2E90534032342F823
:10B3F000103F00234FF4C2510C48FBF7D3FBAD467E
:10B4000088B06A460A4BC2E90534032342F8103F6C
:10B4100000234FF4C2510548FBF7C4FBBD46B0BD45
:10B42000C038002019DF0700D2DE0700140A070029
:10B43000EDDE07000E4B402928BF402170B51D46A8
:10B440000C4C4618B04203F1020304D1002305F866
:10B450001130074870BD02781209A25C03F8022C73
:10B4600010F8012B02F00F02A25C03F8012CE9E7AF
:10B47000B456002080DF070030B503788BB0044657
:10B4800007AD032B21D8DFE803F0021A1C1E124976
:10B4900028463DF0FFFF059563781E210493A378AD
:10B4A0000E4A0393E3780E4802932379019363795C
:10B4B0000093A3794DF0BFFB09480BB030BD09499B
:10B4C000E6E70949E4E70949E2E70A212846084A8C
:10B4D0004DF0B1FBDFE700BF79CE07009BCE070040
:10B4E0009656002080CE070087CE070091CE070039
:10B4F000FBFC070030B50024094D0A4B85B02846F7
:10B500000293039460F090FE02AB284600934FF440
:10B51000A3620A2304493BF0F1FA204605B030BD8E
:10B520000025002098DF0700B86F00200146014881
:10B530003BF05ABB00250020037830B5012B13D017
:10B54000022B27D07BB90A46184B03F1100453F89D
:10B55000045BA34242F8045BF9D11B781370438863
:10B560004B731B0A8B7330BD0A46104B03F110045A
:10B5700053F8045BA34242F8045BF9D11B781370C3
:10B580004368C3F307224B731B0CCB731B0A8A73EC
:10B590000B74E8E700F1100350F8042B984241F8CF
:10B5A000042BF9D103780B70DDE700BFA1DF0700A2
:10B5B000012838B505460CBF0648074852F09AFAEC
:10B5C000044620B101210C3052F0A1FA2576204624
:10B5D00038BD00BF6C1500209014002010B50B463C
:10B5E0000A490246D1F8380120B9BDE810400120CF
:10B5F000FFF7DEBF52F0BEFA0121002304460176B8
:10B6000003820C3052F083FA204610BD0000002067
:10B6100070B504460F2C0D461046194605D80D2C62
:10B620000DD9BDE87040FFF7D9BF132C07D10C48E6
:10B6300052F060FA044638B90024204670BD024634
:10B640000B4645B10748F3E701210C3052F05FFA91
:10B6500001232376F1E70120BDE87040FFF7A8BF82
:10B66000F0150020E814002070B506468EB00A4D93
:10B6700001AC0FCD0FC40FCD0FC40FCD0FC42B687D
:10B680000C2E23609DBF0EAB03EB860656F8340CE0
:10B6900002480EB070BD00BF2C0C0700B2DF0700DF
:10B6A00038B5C368B3F801401B7863B9204603F08E
:10B6B000DBF8054640B9084B1A8822B96FEA0450F6
:10B6C0006FEA1050188038BD012103F0D5F82846E4
:10B6D000BDE8384050F05EBDE855002010B5084C7C
:10B6E0000146052294F8670003F01CFB38B994F872
:10B6F00067000422BDE81040024903F013BB10BDEF
:10B700000000002066DF070080B5C36800AF88B086
:10B710006A461B780749084851610849C2E906137F
:10B7200004234FF4025142F8103F50F0DBF9BD46BC
:10B7300080BD00BFBADF0700C40907006FEA070039
:10B7400080B500AF88B06A46064B4FF4C2515361D2
:10B75000054B06489361032342F8103F50F0C2F9AD
:10B76000BD4680BDE6DF070037E90700C4090700D2
:10B7700098B5014600AF0E4852F0CDF90D490E487C
:10B7800060F031FD002810DA6C4688B06A460B4B39
:10B790004FF4015153610A4BC2E9063004230948B2
:10B7A00042F8103F50F09EF9A546BD4698BD00BF37
:10B7B0003C010020340B00205026002004E007004C
:10B7C0002CEA0700C40907000B46B0B50D8A00AF8C
:10B7D00004462946D868FFF72DFE8CB06A460A4B0E
:10B7E000C2E908505361094B4FF45251C2E9063483
:10B7F00040F203531385064B064842F8103F50F0C1
:10B8000071F9BD46B0BD00BF25E0070055EA07004D
:10B8100006000001C409070080B5012100AF0C300B
:10B8200052F029FA88B06A460378074907485161FF
:10B830000749C2E9061304234FF4015142F8103FAF
:10B8400050F050F9BD4680BD4BE00700C409070029
:10B8500001EA0700B0B5C36800AF1C88204603F0BA
:10B8600003F890B96D4688B06A46094B4FF4015110
:10B870005361084B0848C2E90634042342F8103FDC
:10B8800050F030F9AD46BD46B0BD50F083FCFAE74C
:10B8900071E0070061E90700C4090700B0B5C3689B
:10B8A00000AFB3F80140204602F0DEFF90B96D46CC
:10B8B00088B06A46094B4FF401515361084B09485F
:10B8C000C2E90634042342F8103F50F00BF9AD46AC
:10B8D000BD46B0BD50F05EFCFAE700BF71E0070066
:10B8E00074E90700C40907002DE9F041C56800AFFD
:10B8F0002E78BEB9B5F80180404602F0B5FF044687
:10B9000098B96C4688B06A460C4B4FF401515361AC
:10B910000B4B0C48C2E90638042342F8103F50F0A4
:10B92000E1F8A546BD46BDE8F081EB7831460373EA
:10B9300002F0A2FF204650F02DFCF3E799E007004B
:10B94000B8E90700C4090700B0B5044600AF02EB30
:10B95000C303934203D12046FFF736FF1AE0104697
:10B9600010F8085BA5421BD10B8A5078984213D976
:10B970006D468AB06A460B49146251610A490B4808
:10B98000C2E9061305234FF4215142F8103F50F04D
:10B99000A9F8AD46BD46B0BD084653689847F9E7DB
:10B9A0000246D6E7C3E0070041EA0700C4090700E2
:10B9B000F8B5594800AF52F0C4F80446002870D0DA
:10B9C000037E012B6FD0032B40F09F80038A032B53
:10B9D0000CD840F2ED13514A514952484DF0E7FC62
:10B9E000404080F311884FF0030002DF042104F18E
:10B9F0000C0052F040F9FF2243880688218AC6F3E2
:10BA00000B008B426083627612D06D468AB06A4624
:10BA100045481362506145480523C2E906014FF4C9
:10BA2000215142F8103F424850F05CF8AD4668E0C2
:10BA300002F01AFF054670B96D4688B0638B6A46FE
:10BA40003C4951613949C2E9061304234FF40151BD
:10BA500042F8103FE7E703F009F821466076320B21
:10BA6000284602F09BFD284650F094FB324BD3F859
:10BA70003C31B3B13149324860F0B5FB002810DAEF
:10BA80006C4688B06A462F4B4FF4015153612E4BE0
:10BA9000C2E906300423264842F8103F50F022F84D
:10BAA000A546BD46F8BD038A012B0CD840F66D13A0
:10BAB0001A4A1B491B484DF07AFC404080F311881C
:10BAC0004FF0030002DF022104F10C0052F0D3F822
:10BAD000054600784FF0C4FF83070CD440F671137D
:10BAE0000E4A1A490F484DF062FC404080F311881D
:10BAF0004FF0030002DF06232146154A2878FFF79E
:10BB000023FF204607F0F8FBB0E76D4688B06A4691
:10BB1000104951610C4996E73C010020E9E007001B
:10BB20001DE1070036E1070053E1070014EA0700B2
:10BB3000C40907007BE1070000000020340B00204F
:10BB40005026002004E007001CEA0700A1E10700DE
:10BB5000F4150700CFE1070010B5012104460C30B1
:10BB600052F089F82146BDE810400A23014A0078C6
:10BB7000FFF7EABE24160700F8B5C56800AFB5F8B0
:10BB80000160304602F070FE044690B96C4688B001
:10BB90006A46114B4FF401515361104B1048C2E9F2
:10BBA0000636042342F8103F4FF09CFFA546BD46E1
:10BBB000F8BD2B783BB9D5F80330C0F8AD30D5F8D7
:10BBC0000730C0F8B1304FF48051201D4FF073FFA3
:10BBD000204650F0DFFAEAE771E007001FE90700AE
:10BBE000C40907002DE9F843064600AF907A88465D
:10BBF000144607F0BFFA434D85421AD0A47AE846AE
:10BC0000204607F0B7FA8CB06A463F4BC2E90840BD
:10BC100053613E4B9562C2E9063607234FF46251E9
:10BC20003B4842F8103F4FF05DFFC546BD46BDE8BA
:10BC3000F883204607F0A6FA4FF00C09354D09FBB2
:10BC400000504388B34218D0204607F09BFA09FB06
:10BC500000506C468AB06A464388136205232E4919
:10BC60002B4851612949C2E906164FF4225142F886
:10BC7000103F4FF037FFA546D8E7284ED6F83801D9
:10BC800020B107F039FB0023C6F83831204607F011
:10BC900079FA0C2606FB00504368ABB1B8F1000FEF
:10BCA00012D1204607F06EFA012106FB00504268CF
:10BCB000D2E90003127A03F01F06B1405B09DAB142
:10BCC00000EB83004FF0F7FE204607F05BFA0C26EE
:10BCD00006FB00508368002BA8D0204607F052FADC
:10BCE000704305F80080204607F04CFA06FB00552B
:10BCF000A8683AF01BFD99E7C94300EB83004FF0B9
:10BD0000F4FEE1E7C4150020E7E1070062EA07005E
:10BD1000C4090700C438002020E20700000000200A
:10BD200038B5042104460C3051F0A5FF4578017860
:10BD300022464088FFF756FF25B1BDE8384002484B
:10BD40003AF0F4BC38BD00BF2001002038B5032113
:10BD500004460C3051F08FFFE368057822461978CD
:10BD6000B0F80100FFF73EFF25B1BDE838400248BA
:10BD70003AF0DCBC38BD00BF200100202DE9F84FAF
:10BD80000025A946D0F80C80DFF808A100AF98F88C
:10BD900000309D4202DBBD46BDE8F88F08EB85030D
:10BDA000B3F801B0B3F80360584602F05DFD0446F5
:10BDB000D8B100F1280B002E40D04FF02003EFF354
:10BDC000118283F31288BFF36F8FE36903B3013BE2
:10BDD000E36182F31188BFF36F8F204602F0ACFB62
:10BDE000013E3AF0A3FCB6B2E5E76C4688B06A467D
:10BDF000294B4FF401515361284B2948C2E9063BB6
:10BE0000042342F8103F4FF06DFEA5460135BEE712
:10BE10006369BBB982F31188BFF36F8F6E4688B038
:10BE20006A461E4BC2F814A0936103234FF4C2511B
:10BE30001B4842F8103F4FF055FEB546204650F0E3
:10BE4000A9F9E3E7A16918688B42606108BFA061A6
:10BE500082F31188BFF36F8F4FF02002EFF311814F
:10BE600082F31288BFF36F8FDA68E261C3F80C9037
:10BE7000C3F80090626A4AB9C4E9083381F31188B3
:10BE8000BFF36F8F58463AF033FEA6E71360636244
:10BE9000F4E700BF77E2070057E2070085EA0700F2
:10BEA000C4090700F0B583B0C56800AFB5F80160FC
:10BEB000304602F0D9FC044698B96C4688B06A4610
:10BEC0002C4B4FF4015153612B4B2C48C2E90636E1
:10BED000042342F8103F4FF005FEA5460C37BD463F
:10BEE000F0BD2B78061D1A2B17D1C378012B28D152
:10BEF0004FF4806130464FF0DEFD42050DD4D4F89A
:10BF0000A03039463B60D4F8A83020467B6003F06F
:10BF100039FA204650F03EF9E0E72B788BB9B5F8B6
:10BF20000330A4F89E30B5F80530A4F8A430B5F875
:10BF30000730A4F8A6306FF4807130464FF0D5FD7D
:10BF400014E0D6E8AF3FDB05F5D52B78202BF2D1F6
:10BF500094F8AC30002BEED0013B84F8AC304FF4B9
:10BF60002032002304F158003AF068FE204602F027
:10BF70009FFDCEE771E0070007E90700C40907004D
:10BF800010B5C1E900239DF808300C460B7207F08C
:10BF9000F9F80C22024B02FB00335C6010BD00BFBD
:10BFA000C43800202DE9F0474FF0FF324FF0FF3347
:10BFB000064617480F4651F09DFD4FF00008044615
:10BFC00000F10C0A0121504651F0A1FD204684F8F1
:10BFD000188007F0D7F84FF00C090E4D09FB005000
:10BFE0004680204607F0CEF809FB0050C0F80880D4
:10BFF000204607F0C7F809FB005503215046C5F855
:10C00000048051F008FE068087702046BDE8F08766
:10C01000C4150020C43800202DE9F04387B08046C5
:10C0200015460C4600AF21B9FFF7BCFF04460028B7
:10C030005CD001220021384660F023F8204607F04A
:10C04000A1F80C23DFF8AC9003FB0090876020463A
:10C0500051F090FD0146284851F08AFD4FF4A0228E
:10C06000002338463AF088FB064680B140F2491377
:10C07000224A234923484DF09AF9314622484DF08F
:10C0800096F9404080F311884FF0030002DF20460C
:10C0900007F078F80C23584319F80060F6B16D46A4
:10C0A0008AB06A46194B16625361194B4FF42251FC
:10C0B000C2E906380523174842F8103F4FF012FD39
:10C0C0002046AD4607F018F9092E14BF6FF00400A2
:10C0D0006FF06E001C37BD46BDE8F08315B12C60D3
:10C0E0000020F7E7204607F007F9F9E76FF068004E
:10C0F000F0E700BFC438002044010020E9E0070059
:10C1000092E2070036E107009BE20700BBE207006E
:10C11000EBEA0700C4090700F0B583B000AF06469C
:10C120000D4642F22F0000213A1DFFF775FF04462D
:10C1300098B16D4688B06A460D4B4FF4C2515361B9
:10C140000C4B0D489361032342F8103F4FF0CAFC9B
:10C15000AD4620460C37BD46F0BD7868C368B3F8DD
:10C1600001203280B3F803302B8007F0C5F8F0E7E8
:10C17000DBE207003EEB0700C4090700F7B5144BEC
:10C18000054693F993300C46002B1DDA14B920466E
:10C1900003B0F0BD082C4FF0000142F2180001AAD4
:10C1A000264628BF0826FFF737FF0028F0D1019F59
:10C1B0003246F96828460131F4F71CFD384607F08D
:10C1C0009BF83544A41BE1E76FF08500E0E700BF72
:10C1D000000000202DE9F04F89B0B0F80190002652
:10C1E0006FEA09536FEA13530546B14A9BB21188AF
:10C1F00002AF994204BF1680012601F013F92C7892
:10C200001FFA89F8002C3BD03C2C27D101F04CFCC4
:10C210006FF0800110304FF068FC0020FFF75EFAED
:10C22000054698B96C4688B002AAA24B4FF4C25199
:10C230005361A14BA1489361032342F8103F4FF093
:10C2400051FCA5461C37BD46BDE8F08F04730021A4
:10C2500002F012FB28464FF09DFFF3E76D4688B0D1
:10C2600002AA974B4FF402515361964B9348C2E98F
:10C270000634042342F8103F4FF034FCAD46E1E7AA
:10C280002B7905F1040A023B012B2ED8514607F108
:10C2900010004FF020FC3B7C05F11101023B07F13F
:10C2A00009003B744FF012FC01233B72EB78012B29
:10C2B00030D05046FFF7E0F86C468AB002AA824BB5
:10C2C0004FF4115153617F4BC2E9063040F2013304
:10C2D00013847E4B794842F8103F4FF003FC1F2136
:10C2E000A54640464FF019FCACE7EB785146012BD0
:10C2F00004BF774B93F8674020464FF076FD014628
:10C3000007F110004FF0E7FB514607F108004FF02E
:10C31000E2FBCBE707F11000FFF7E0F9EB7804460A
:10C32000012B0AD101F0C0FB83466FF08001103071
:10C330004FF0DBFB58464FF087FE002CB9D020466B
:10C34000002220F8889B07F110014FF0C4FBB5F8DC
:10C350001730A4F89E30B5F81930A4F8A430B5F819
:10C360001B30A4F8A630EB782273012BE37016D1B2
:10C3700007F1080104F18F004FF0ADFB01F094FBD1
:10C38000217A534AC1EBC101114404F196004FF0E8
:10C39000A2FBD2F8DC305D0601D501F07DFD07215E
:10C3A000204602F069FA1EB10121204602F064FA2B
:10C3B00020464FF025FF637B072B74D1231DD3E864
:10C3C000AF3F13F4805F424D2BD1E3781BB195F85A
:10C3D000D030180725D5022142F21600FFF7E2FD02
:10C3E0000646002861D002210C3051F014FC23884D
:10C3F00000220380314642F21600FFF70DFE80B1A5
:10C400006E4688B002AA334B4FF401515361324B50
:10C41000C2E906300423294842F8103F4FF062FB7E
:10C42000B54695F8D130D90718D50021022320460A
:10C430001A4600914FF0AAFB80B16E4688B002AA5E
:10C44000264B4FF401515361234BC2E906300423BC
:10C450001A4842F8103F4FF045FBB54695F8D030EA
:10C460009A0620D5D5F85C319B689B071BD5B91D72
:10C47000381DFFF751FEB0B92046FA88B9884FF051
:10C4800067FB80B16D4688B002AA154B4FF401518D
:10C490005361114BC2E906300423084842F8103FAB
:10C4A0004FF020FBAD462046D5E66FF06800A7E7C9
:10C4B000E8550020FFE20700B2EA0700C4090700C0
:10C4C00024E30700CFEA070041E30700040000016E
:10C4D0000000002061E307009FEA070086E30700F1
:10C4E000A1E3070000B5C16889B00B7801A88DF8F9
:10C4F0000030B1F801300431ADF8013011F8013CE1
:10C500008DF80330B1F80730ADF81730B1F80930C5
:10C51000ADF81930B1F80B30ADF81B304B7B8DF80E
:10C520001D304FF0D8FA07490DF10B004FF0CEFA4D
:10C530000DF111004FF0CAFA6846FFF74BFE09B043
:10C540005DF804FB7ADF070029289ABF014B185CCD
:10C5500009207047BFE70700F8B5C36800AFB3F81C
:10C5600001601D78304602F07FF9044690B96C46B0
:10C5700088B06A46214B4FF401515361204B21484A
:10C58000C2E90636042342F8103F4FF0ABFAA54645
:10C59000BD46F8BD5DB12846FFF7D6FF29460246E5
:10C5A000204602F02DFB20464FF0F4FDF0E78378A3
:10C5B000012BF0D106F0E0FB20464FF063FA002893
:10C5C000E9D10520FFF7C0FF05210246204602F011
:10C5D00017FB6D4688B06A460B4B4FF4C25153614E
:10C5E000074B08489361032342F8103F4FF07AFA53
:10C5F0000521AD4620464FF00CFED4E799E0070038
:10C60000E0E90700C4090700C1E307002DE9F04194
:10C61000C66800AFB6F801803578404602F024F9CC
:10C62000044698B96C4688B06A46274B4FF40151CE
:10C630005361264B2648C2E90638042342F8103FCE
:10C640004FF050FAA546BD46BDE8F0815DB12846E1
:10C65000FFF77AFF29460246204602F0D1FA20462B
:10C660004FF098FDEFE78278F378012AC37205D086
:10C670000020FFF769FF00210246EDE70BB106F04D
:10C680007BFB20464FF0FEF90028F1D10520FFF793
:10C690005BFF05210246204602F0B2FA6D4688B0E3
:10C6A0006A460C4B4FF4C2515361084B08489361E2
:10C6B000032342F8103F4FF015FA0521AD462046FE
:10C6C0004FF0A7FDCBE700BF99E00700CDE90700D9
:10C6D000C4090700C1E30700024BD3F85C315B6972
:10C6E000184700BF00000020F8B505460C4600AF13
:10C6F00019B9FFF757FC044628B340F635439D426D
:10C700001BD12046FFF7E8FF054698B16E4688B07A
:10C710006A460E4B4FF4015153610D4BC2E906308E
:10C7200004230C4842F8103F4FF0DCF92046B54690
:10C7300006F0E2FD2846BD46F8BD2146064851F008
:10C7400017FA0025F6E76FF06805F3E7EBE307005B
:10C7500000EB0700C4090700440100202DE9F04167
:10C760000446458B467E00AF807A06F003FD2146E5
:10C770005FF066FC304B93F882309B062DD5304637
:10C7800002F082FC044688B96C4688B06A462B4B9E
:10C790004FF4025153612A4BC2E90636042342F892
:10C7A000103F28484FF09EF9A54616E0437B073B13
:10C7B000012B15D96D4688B06A46234B2148536139
:10C7C0001F4B4FF4C4519361032342F8103F4FF0C5
:10C7D00089F92046AD464FF0DDFCBD46BDE8F0814D
:10C7E0004FF0D8FC052140F63540FFF7DBFB04464F
:10C7F00060B96C4688B06A46144B4FF4C25153611D
:10C800000F4B9361032342F8103FCAE700F10C0875
:10C810000121404651F0FFF90126042106704046EF
:10C8200051F0F9F9002305808670C370214640F667
:10C830003540FFF759FFD0E70000002011E4070062
:10C8400010EB0700C40907003EE407006EE4070090
:10C850002DE9F04186B0C56802AF2E881FFA86F830
:10C86000404602F001F80446A0B96C4688B002AA1E
:10C87000334B4FF401515361324B3348C2E9063810
:10C88000042342F8103F4FF02DF9A5461037BD465E
:10C89000BDE8F081D5F80220D5F806300197698906
:10C8A000009150F03BFF98B3122142F21A00FFF7BB
:10C8B00079FB054698B96D4688B002AA234B5361AF
:10C8C000234B936103234FF4C2511F4842F8103F9A
:10C8D0004FF008F9AD4620464FF05CFCD6E7122138
:10C8E0000C3051F098F903463A4623F8026B07F1F1
:10C8F000100C164603CE664518605960324603F1A7
:10C900000803F6D1294642F21A00FFF7EDFEE2E7EE
:10C91000022142F21B00FFF745FB054630B96D4688
:10C9200088B002AA094B53610A4BCAE702210C30B6
:10C9300051F071F92946068042F21B00E5E700BF7D
:10C9400071E00700A9E90700C409070095E40700A2
:10C950009CE907008BE90700F0B583B0C36800AF1E
:10C96000D9789A781E8842EA01223A8059791A7950
:10C97000B4B242EA01227A809A79D979204642EA11
:10C980000122BA801A7A5B7A42EA0323FB8001F023
:10C990006BFF0546B8B96D4688B06A461F4B4FF429
:10C9A000015153611E4B1F48C2E90634042342F86B
:10C9B000103F4FF097F80221AD4620464FF032F974
:10C9C0000C37BD46F0BD394602F0B2F838B91E2129
:10C9D00020464FF027F928464FF0DCFBF0E70E2108
:10C9E00042F22000FFF7DEFA04460028F3D00E21C1
:10C9F0000C3051F010F900230680C0F80A303B8853
:10CA0000214643807B888380BB88C380FB88038169
:10CA100042F22000FFF768FEDDE700BF71E007008B
:10CA20004FE90700C40907002DE9F04FDFF86C81DA
:10CA300083B0DFF86C9108F1140A00AFD8F80C301D
:10CA400050466FF39433C8F80C3001F0D5FE451C06
:10CA50004FF0FF324FF0FF33294650483AF046FF7F
:10CA600060B140F6E6134A464E494F484CF09FFCF1
:10CA7000404080F311884FF0030002DF474E15B9A4
:10CA80003AF05CFBDAE7F368C3F38633012B69D92C
:10CA9000042B71D1337B002B67D100220023434844
:10CAA00051F02DF8044660B94FF418634A464049E6
:10CAB0003D484CF07CFC404080F311884FF003006F
:10CAC00002DFDFF8F0B04FF0FF324FF0FF333A48AB
:10CAD00039F052FEDBF83821C2B1C7F804D088B073
:10CAE0006A4636493648516136499161032142F818
:10CAF000101F4FF4C2514EF0F5FFD7F804D0DBF809
:10CB0000380106F0F9FB0022CBF83821204651F01D
:10CB100031F8CBF838012046FFF7DEFD10B3EB46C5
:10CB200088B06A46284B4FF401515361254BC2E946
:10CB300006300423224842F8103F4EF0D3FFDD4672
:10CB40001D4839F0F3FD204606F01CFB0C221F4B5C
:10CB50001F2102FB003022464088FFF743F82046A1
:10CB600006F0CAFB1436013D89E7012BFAD1306982
:10CB7000383802F0F3F9F5E76C4688B06A46144994
:10CB80000F4851611349C2E9061304234FF40251BF
:10CB900042F8103F4EF0A6FFA546E3E7F80A002052
:10CBA000E9E0070092E2070036E1070044010020B7
:10CBB000A30008000000002020010020B0E40700CE
:10CBC000C4090700E9E70700EBE30700C4380020C9
:10CBD000CFE40700F2E707002DE9F041044600F139
:10CBE0000C06304651F057F8B4F810800546B8F1FD
:10CBF000010F0CD840F67B531B4A1C491C484CF0D3
:10CC0000D6FB404080F311884FF0030002DF30462E
:10CC1000022151F030F8074600784EF021FFC2079C
:10CC200006460CD440F67F530F4A124910484CF088
:10CC3000BEFB404080F311884FF0030002DF052364
:10CC400021460D4A3878FEF77FFEB30707D56369A2
:10CC5000A4F8108013FA85F5E560BDE8F081204660
:10CC6000BDE8F04106F048BBE9E007001DE1070020
:10CC700036E10700F4E40700CC150700B0B5037EE9
:10CC80000446012B00AF06D0032B12D1FEF770FD36
:10CC90000020BD46B0BDC36818784EF0E1FEC20763
:10CCA000054602D52046FFF797FFAB07F0D5204693
:10CCB000ECE76D4688B06A4609490A4851610A495D
:10CCC000C2E9061304234FF4015142F8103F4EF01D
:10CCD00009FF2046AD4606F00FFB6FF01500D8E7C0
:10CCE0000DE50700C409070039EA0700084A0346B2
:10CCF000D2F85C0130B9D96839B1596929B1C2F8A3
:10CD00005C3170476FF0770070476FF01500704727
:10CD1000000000202DE9F04F484D83B0042100AF02
:10CD200047484EF0C8FE474CEA79474B2846012A4F
:10CD300088BF1C46E846FEF79FFB8AB06B46434916
:10CD4000434E59614349C3E906647960186203F1AF
:10CD50001002381D03F1230103F1270410F801CB61
:10CD600001F801CFA142F9D101243B493B481961A7
:10CD70004FF443514EF0B6FEDFF8E490C546DFF8BD
:10CD8000DCA0DFF8B880EA7908F1070894423DDBBF
:10CD900095F86880EA464046FEF766FC8CB06C4623
:10CDA000B5F86A20B5F86E3040F20139C4E90708D9
:10CDB000A046C4E909232B492B4BC4E90516A4F866
:10CDC0002C9048F8103F42464FF4735123484EF0E0
:10CDD00089FED54695F869A05046FEF745FCA54664
:10CDE000B5F86C30214A6362214BC4E90526C4E9D9
:10CDF000070A42464FF453511848A4F8289023617B
:10CE00004EF070FE0C37BD46BDE8F08F4046FEF791
:10CE100033FBEB468AB06A4640F20241154BC2E949
:10CE200007409184C2E905364FF43351504642F829
:10CE3000109F4EF057FE0134DD46A4E700000020AD
:10CE4000CC000020180E090025E5070029E50700A1
:10CE5000F6E807000103020405000002C409070008
:10CE60000500000151E507000700000193E50700F8
:10CE7000060000013CE5070010B5F5F751F8034B3B
:10CE80001B6813B1BDE81040184710BD3C390020A5
:10CE9000024BD3E8AF0FC0F380007047CC000020F6
:10CEA00038B505463CF044FD1C28044610D82946F8
:10CEB0000948F3F715FF48B12246294606483CF0D9
:10CEC000A7FD0022054B234483F86021002038BDD4
:10CED0006FF00B00FBE700BF6001002000000020A6
:10CEE000F0B589B0484E0546D6F85C3108AFABB90D
:10CEF0006C4688B02246454B4FF4C2516361444BA7
:10CF00004448A361032342F8103F4EF0EBFDA546D1
:10CF10006FF0120420460437BD46F0BD6FF00201E9
:10CF200006F1CC004EF0E1FD01214EF0C4FDC30737
:10CF300066D43948FFF7B4FF80B16C4688B022460A
:10CF4000364B4FF402516361314BC4E90630042380
:10CF5000304842F8103F4EF0C5FDA546304B1D60ED
:10CF60000122304811465FF08CF82F485FF030F80E
:10CF7000002200230024CDE906236FF008034FF4BC
:10CF80008062CDE90334CDE90144284B284900945F
:10CF9000284839F03BFA284926485EF089FF27489F
:10CFA0005FF042F96FF007034FF4805224492348A1
:10CFB000009439F0A3FD234920485EF079FFD6F8AC
:10CFC0005C31DB689847044688B16D4688B02A46D4
:10CFD0001D4B4FF401516B610D4BC5E90630042325
:10CFE0000C4842F8103F4EF07DFDAD4692E71DB96A
:10CFF000F4F796FF04468DE7144839F079FD89E788
:10D000006FF0770486E700BF000000202BE70700E1
:10D0100001E80700C409070069E7070070E7070097
:10D020003C390020200100204401002029CA0000D2
:10D03000D0740020B825002093E707005026002078
:10D04000D078002099E707009FE70700BC00002088
:10D050000048704760010020F8B506460025094FDA
:10D06000FB79ECB2A34202D86FF0010009E0C4EBF7
:10D07000C401304639444EF0FBFD01350028EFD0A5
:10D080002046F8BD0000002037B504460D4671B1BA
:10D09000284612494EF0ECFD48B929461048C4EB29
:10D0A000C40420444EF0F1FD002003B030BD6846BA
:10D0B0004EF0C8FC0028F8D16846FFF7CDFF0028E5
:10D0C000F5DA074BC4EBC400694618444EF0DDFDA9
:10D0D000002DE9D001462846E4E700BF6DDF0700D8
:10D0E0000000002000212DE9F04383B00446062211
:10D0F000084600AF01F016FE064690B15C4BD3E83F
:10D10000EF1F41F40041C3E8E21F002AF7D1237A60
:10D1100043F0010323724FF03DF80C37BD46BDE8E4
:10D12000F083544D0146544800F0B8FC95F819318D
:10D13000A3B130464EF0EFFD80B16C4688B06A4630
:10D140004E4B53614E4B936103234FF4C45142F84D
:10D15000103F4C484EF0DCFDA5462CE095F8192117
:10D1600095F818319A4238D16E4688B06A464FF029
:10D170000308454BDFF808915361C2F818904FF44B
:10D18000C451404842F8108F4EF0C2FD0022B5460F
:10D19000114642F22900FEF73FFFA0B188B06A466F
:10D1A0003A4B4FF4C251C2E90539364842F8108F64
:10D1B0004EF0AEFDB54601204EF0ADFD00213448E5
:10D1C00000F06CFCA9E795F81931013385F81931A5
:10D1D000237A43F004032372EDE7224604F10108A9
:10D1E000414612F82A0B4EF057FD064660B16C46D8
:10D1F00088B06A46274B5361214B4FF4C25193616B
:10D20000032342F8103FA4E795F81931013385F85C
:10D210001931237A43F00403237295F89F305B079A
:10D2200006D46C4688B06A461B4B53611B4B8AE799
:10D23000414638464EF029FD0123082142F24E00B6
:10D24000FB71FEF7AFFE044660B1082239460C3090
:10D2500050F0E7FC3246214642F24E00FEF7DCFE7B
:10D260000028A8D06C4688B06A460D4BC3E700BFC3
:10D27000CC00002000000020C7BD050079EB0700AE
:10D280005DEE0700DC090700A2EB0700D7EB070003
:10D2900047BD0500FBEB07001FEC070049EE070048
:10D2A0004DEC070038B50622114905463BF052F90E
:10D2B000C8B1062142F20500FEF774FE0446A0B193
:10D2C000062229460C3050F0ACFC0022214642F2E6
:10D2D0000500FEF7A1FE38B9054829464EF0D0FCFE
:10D2E000012300F8013C002038BD6FF06800FBE727
:10D2F0006100002000212DE9F8430622044600AF1A
:10D30000084601F00FFD054688B13D4BD3E8EF1FFD
:10D3100041F40041C3E8E21F002AF7D1237A43F029
:10D32000020323724EF036FFBD46BDE8F883014686
:10D33000344800F0B3FB28464EF0EDFC324D064673
:10D3400090B16C4688B06B46304A4FF401515A6137
:10D350002F4AC3E906201A46042342F8103F2D48FD
:10D360004EF0D6FCA54611E095F8193195F8182134
:10D370009A4216D2013B85F81931237A024623F0EE
:10D38000040302202449237205F0D6FD95F81931D3
:10D3900013B101204EF0BFFC0021204800F07EFBBD
:10D3A000C2E7072142F22800FEF7FCFD04F1010963
:10D3B000804660B96C4688B06A46194B4FF4C2513A
:10D3C0005361134B9361032342F8103FC7E70721D2
:10D3D0000C3050F020FC49464EF057FC3246414696
:10D3E00042F22800FEF718FE0028E3D195F8193123
:10D3F000013B85F81931237A23F004032372C5E732
:10D40000CC000020C7BD0500000000206CEC070028
:10D410003FEE0700DC090700FBBC050047BD050027
:10D420009DEC0700084BD3E8EF2F22F40041C3E83E
:10D43000E01F0028F7D1130404D50022022003497D
:10D4400005F07ABD704700BFCC00002049BE050042
:10D45000002307B50549CDE900036A46022005F01F
:10D460006BFD019803B05DF804FB00BF6DBD0500C6
:10D47000034610B470B10A4991F8184191F8192186
:10D480000CB1944208D2013281F819211A7A42F083
:10D4900004021A7210BC704710BCFFF723BE00BF15
:10D4A00000000020034610B498B10B4C94F81811FA
:10D4B00094F8192129B101318A4203DC10BCFFF72D
:10D4C00019BF12B1013A84F819211A7A22F0040224
:10D4D0001A7210BC704700BF00000020F8B50D465E
:10D4E000044600AF20B94DB36FF01500BD46F8BD3E
:10D4F00023494EF0BDFB0028F5D12378012B04D140
:10D50000A37903F0C003C02B10D06C4688B06A46E4
:10D510001C4B4FF4C25153611B4B1C4893610323B6
:10D5200042F8103F4EF0F4FBA546DDE72046FFF73A
:10D5300093FD0028D7DB6FF07700D7E7144DEB7928
:10D54000012B1AD005F1CC03D3E8AF3FDB070BD595
:10D55000EE7921463046FFF797FD0028C6D1EB79DA
:10D5600030460133EB71C1E7002CBDD020460449A1
:10D570004EF07EFB0028EBD0B6E76FF00B00B5E76E
:10D580006DDF0700C6EC070032EE0700DC0907007C
:10D5900000000020F0B583B0044600AF98B96C4697
:10D5A00088B06A461D4B53611D4B4FF4C4519361C3
:10D5B00003231C4842F8103F4EF0AAFBA54600206A
:10D5C0000C37BD46F0BD002141F209003A1DFEF7BF
:10D5D00023FD064620B16C4688B06A46124BE2E74E
:10D5E0007B680622DD681149013528463AF0B2FF12
:10D5F00018B9786805F080FEE1E7062228460C4954
:10D600003AF0A8FF0028F4D02946601C4EF038FB01
:10D610007868267005F070FE0120D1E7F8EC07006D
:10D620001BEE0700DC09070015ED07007ADF070095
:10D6300074DF070007B56846FFF7ACFF044BD871ED
:10D6400018B169460020FFF71FFD03B05DF804FB29
:10D65000000000202DE9F04182B02D4B054693F8E3
:10D66000BA300E46DB0700AF15D46C4688B06A4668
:10D67000284B5361284B4FF4C4519361032327482F
:10D6800042F8103F4EF044FBA546002420460837E0
:10D69000BD46BDE8F08100214FF609403A1DFEF776
:10D6A000BBFC034620B16C4688B06A461C4BE0E7E1
:10D6B00078684FF0160CC26854780232B44228BF22
:10D6C00034469C4214DC05F017FE002CDED16D467A
:10D6D00088B06A46134B4FF4C45153610E4B0F4848
:10D6E0009361032342F8103F4EF012FBAD46CDE7A5
:10D6F00011460CFB035602F1140E51F8048B7145D0
:10D7000046F8048BF9D10988013331801632D8E705
:10D710000000002037ED070007EE0700DC090700D6
:10D7200067ED07008BED070070B5154D88B0EC79FB
:10D730002CB9012102A8FFF78DFFE871C0B90021C3
:10D74000084608B0BDE87040FFF7C8BE02AB06FB54
:10D7500002310DF101004EF093FA012369461046A3
:10D760008DF80030FFF790FC013410B108B070BDA7
:10D770001626EB79E2B29342E8D80020F6E700BF24
:10D78000000000202DE9F04190460E461D4602465D
:10D7900000284BD0002B49D0CF07047831D5254F36
:10D7A000B8F1000F13D088060AD4C4EBC403FB5CA5
:10D7B000012B15D02B70B2060FD543F002030BE0FE
:10D7C00097F8D0305906F0D46FF0850006E0C4EB2E
:10D7D000C403FB5C012B03D02B700020BDE8F0815B
:10D7E000072101FB0471104601314EF00AFB0028AD
:10D7F000F4D1C4EBC4043B5D2B70B8F1000FECD046
:10D80000D9E74B070ED50B4EC4EBC407F35D012BD4
:10D81000E2D1072111FB043131444EF0F2FAF35DFD
:10D820002B70DBE74EF0F5FA0123F9E76FF01500F6
:10D83000D4E700BF00000020B0B5184D00AFEB7971
:10D840001BB100242046BD46B0BDFFF7F3FE0446E1
:10D8500080B16D4688B06A46114B5361114B4FF44D
:10D86000C25193610323104842F8103F4EF050FA22
:10D87000AD46E7E7EB79002BE3D1FFF755FF044610
:10D880000028E6D1681CFFF70DFD04460028D9D01A
:10D890006D4688B06A46054BDFE700BF00000020F8
:10D8A000B8ED0700FCED0700DC090700DBED070021
:10D8B0002DE9F04F85B00C4600AF20211646B86028
:10D8C000FEF770FB0546002866D020210C3050F092
:10D8D000A2F92022824600213AF000FF04EBC603A1
:10D8E00000260AF1010BFB600023D4F80090626867
:10D8F00093420BD3FB680834A342F5D1002229469A
:10D90000B8688AF80060FEF787FB24E099F80120E8
:10D91000B01C81181F2999F800C022D9BCF1090F49
:10D92000C0F11F0201D1002A19DC6C4688B06A469A
:10D930001B4B53611B4B9361032342F8103F0023A1
:10D940004FF4C2511848F9F72DF92846A54605F0BD
:10D95000D3FC6FF015001437BD46BDE8F08F4FF0D3
:10D96000080C5FFA82F808F101010BF80610711C2F
:10D97000C9B20BF801C0D9F804105BFA80F07B60E3
:10D9800008F10208F3F736F97B68B0445FFA88F6CD
:10D99000013309F10809AAE76FF06800DBE700BF6F
:10D9A0006DEE0700EFEE07009409070070B505461D
:10D9B000164B15F8092B044683F867200E460722FC
:10D9C000284613493AF0C6FD034620786BB9114941
:10D9D00001F03CF9044610B96FF00B0070BD042152
:10D9E00000F04AFF00203460F8E7294601F066F9AC
:10D9F00040B92078294601F029F904460028EBD0E7
:10DA00000521EDE76FF01500E8E700BF00000020FA
:10DA10006DDF070066DF070038B543680446580528
:10DA200001D5002038BD22690AB1D907F9D5194DB1
:10DA30002078EB798342F4D9C0EBC0000722164965
:10DA400028443AF087FD0028EBD06068C20706D46E
:10DA500095F86830082B02D8A3689F2BE1D910F005
:10DA6000300F02D02369002BDBD0C30601D4236919
:10DA700043B9D4E902239A42D3D81F2AD1D9B3F5A6
:10DA8000804FCED800F46030B0F5603018BF012070
:10DA9000C8E700BF000000206DDF07000346014813
:10DAA000184700BF180000200048704718000020E9
:10DAB000F0B5054685B00F484EF0E5F91F46030660
:10DAC000164613D50B484EF0DEF904460A484EF0D0
:10DAD00074FAC4F3C0240A46029033462946CDE9BD
:10DAE000007405484EF0F7F905B0F0BD6FF00A007C
:10DAF000FAE700BF28000020180000202DE9F04FB1
:10DB00008DB004AFC7E900320023D1F810B006464B
:10DB1000BBEB0304924818BF0124FB604EF0B3F93D
:10DB200043070D4640F113810846FFF775FF30B9F2
:10DB30006FF0150420462437BD46BDE8F08F284617
:10DB40004EF07EF982460028F2D006F110094846D0
:10DB50004EF099F9C0F3C013000600F1FB80C7E94D
:10DB60000533C7F81B30AB6868683B82EB687B8283
:10DB70004EF07AF932782B7878779A4204D06FF4A5
:10DB8000005177484EF082F92B78764A337082F84C
:10DB9000673030462246696807F11503FFF7F2FD4A
:10DBA00004460028C6D106F10900BBF1000F13D0CE
:10DBB00029694EF076F928464EF00FFA6B688046D8
:10DBC000D90716D49B0504D4BB6C13B9B8F1020F66
:10DBD0005ED102233B7518E063494EF062F9284696
:10DBE0004EF0FBF96B688046DA07EBD587F814B086
:10DBF0000BE013F0100F0CBF01230423296907F178
:10DC000016003B75A2464EF04CF90F2142F2060079
:10DC1000FEF7C8F90446002800F09F800F2207F1A4
:10DC200010010C304FF0FDFF2146002242F20600A9
:10DC3000FEF7F2F9044600287FF47CAFBBF1000F39
:10DC40002BD06B68DC0736D4012130464EF0D5F975
:10DC50000446002873D06D4688B004AA434B536134
:10DC6000434B9361032342F8103F00234FF4C2510A
:10DC70004048F8F797FFAD46FD68002D3FF45AAFD6
:10DC80002846002100F0F8FD28464EF083FA51E7BF
:10DC90000323D7F848A03B75B7E7CDE901A8FB6C93
:10DCA00030460093BB6CD7E900214EF014F90446CE
:10DCB0000028C6D03EE7304607F10C01FFF776FE9C
:10DCC00004460028C0D010F10C0F7FF433AFBBF135
:10DCD000000F7FF42FAF6B6898073FF52BAF6C6890
:10DCE00084F00204C4F3400404F001020E2148460B
:10DCF0004EF0DEF808F1FF335A425A4108214846F7
:10DD00004EF0D6F8A8F102014A424A41484609219C
:10DD10004EF0CEF86A680A21484602F001024EF041
:10DD2000C7F852460B2148464EF0C2F86A680D21EA
:10DD30004846C2F380024EF0BBF80024FAE6F868C9
:10DD400008B14EF027FABBF1000FCDD1C7E76FF055
:10DD50000A04EFE66FF07704ECE66FF06804E9E69A
:10DD6000CC000020000000206DDF07008AEE0700D5
:10DD7000D8EE07009409070073B51546069A0C46BD
:10DD8000CDE900322B460A4601461148FFF7B6FEA0
:10DD900021460646002340F201109D4202D1304642
:10DDA00002B070BD0A88824204D14A6812B112786A
:10DDB000D20702D401330831EFE7064906485EF086
:10DDC00039FA4FF470220023034838F06BFFE6E77E
:10DDD0001800002061DE00003000002010B51A4855
:10DDE0004EF032F96FF4804118484EF04FF8174862
:10DDF0004EF049F803461A06C0F3C01023D5134865
:10DE00004EF041F8430514D50722114911483AF064
:10DE1000A1FB114B98B904221049187E00F082FF33
:10DE2000044630B10021017300F026FD20464EF07B
:10DE3000B1F9BDE81040002103484EF0DEB80522DC
:10DE400003F12101E9E710BD18000020280000209F
:10DE50006DDF0700210000200000002066DF0700C2
:10DE600080B500AFFFF7BAFF88B06A46074B536131
:10DE7000074BC2E90630042342F8103F00234FF459
:10DE800002510448F8F78EFEBD4680BDA9EE07009A
:10DE9000CCEE07009409070073B51E4C20464DF0E8
:10DEA000F2FF400434D520464DF0EDFF01062FD49B
:10DEB00020464DF0E8FF42052AD501A9A4F1100043
:10DEC000FFF774FD054618BB0121A4F110004EF0C8
:10DED00094F8019E28B9304602B0BDE870404EF07B
:10DEE00059B92946304600F0C7FC6FF480412046FE
:10DEF0004DF0CCFF054630464EF04CF96B0407D58B
:10DF0000D4E8EF3F43F48043C4E8E23F002AF7D16E
:10DF100002B070BD28000020B0B58CB002AF202147
:10DF200007F10800FEF72AF9044650BB5EF081FBBA
:10DF30004FF47A75A0FB052305FB01310823D20BB2
:10DF400042EA4142C90BC7E9002110480093202250
:10DF50003B4607F108014DF01EFC90B96D4688B0B4
:10DF600002AA0B4B53610B4B9361032342F8103F02
:10DF70004FF4C25123460848F8F714FE6FF004042A
:10DF8000AD4620462837BD46B0BD00BF082700205B
:10DF90000CEF070045EF0700D4090700B0B582B0C9
:10DFA00000AF08213846FEF7E9F80446C0B9082258
:10DFB00039460F484DF0CFFBB0B96D4688B06A4680
:10DFC0000C4B53610C4B9361032342F8103F4FF409
:10DFD000C25123460948F8F7E5FD6FF00404AD4649
:10DFE00020460837BD46B0BDFFF796FF0446F7E769
:10DFF0000827002027EF070051EF0700D40907008A
:10E0000038B50D46044698B191B10B4A4DF0DCFB92
:10E01000431C07D1FFF780FF48B929462046064A2E
:10E020004DF0D2FB01280CBF00206FF0040038BD7A
:10E030006FF01500FBE700BF08270020402208B55D
:10E0400003493AF087FAB0FA80F0400908BD00BFF2
:10E050001EF007002DE9F843464B00AF93F89A30C5
:10E0600003F00603062B16D06C4688B06A46424B76
:10E070005361424B9361032342F8103F00234FF456
:10E08000C4513F48F8F78EFD6FF08505A546284638
:10E09000BD46BDE8F883002869D03A4E3268D2B157
:10E0A000131F834213D16C4688B06A46364B5361C6
:10E0B000324B9361032342F8103F00234FF4C451C5
:10E0C0002F48F8F76FFD6FF07705A546DFE75B682F
:10E0D0000BB1043BE5E742607268031D336002B98F
:10E0E00073602A4CD4E8EF8F48F02003C4E8E23F85
:10E0F000002AF7D118F0200801D00025C7E7D4E89E
:10E10000EF3F23F01003C4E8E23F002AF7D1424674
:10E11000414642F22500FDF77FFF05460028ECD07E
:10E12000E94688B06A461A4B5361144B9361032346
:10E1300042F8103F4FF4C25143461148F8F732FD00
:10E14000CD46D4E8EF3F23F02003C4E8E23F002AA5
:10E15000F7D134683CB154F8043C043C0BB10020C6
:10E1600098476468F6E70023C6E900338FE76FF04D
:10E1700015058CE7000000206AEF07000FF007008C
:10E18000B4090700443900208DEF0700CC000020BF
:10E19000ADEF0700044BD3E8AF3F13F0100F034877
:10E1A00008BF0020704700BFCC000020355700207A
:10E1B000F8B5284E0446336800AF8B4243D023B1F4
:10E1C0006FF00F042046BD46F8BD234BD3E8AF2FB8
:10E1D0009206F5D4D3E8AF3FDB0637D5316042F283
:10E1E00026004021FDF7DEFE054648B340210C30F5
:10E1F0004FF011FD234604F1400253F8041B9342F3
:10E2000040F8041BF9D10022294642F22600FDF70E
:10E2100003FF04460028D5D000236D4688B06A4627
:10E2200033600E4951610E49C2E90614042142F8D7
:10E23000101F4FF402510B48F8F7B4FCAD46C1E78C
:10E240006FF06804E8E76FF07704BBE76FF07C04D9
:10E25000B8E700BF40390020CC000020DBEF07000A
:10E2600001F00700B4090700F8B5194BC568D3E8F9
:10E27000EF2F22F02002C3E8E12F0029F7D12A78FE
:10E280008AB914496A1C05F1410052F8044B8242D4
:10E2900041F8044BF9D1D3E8EF1F41F01001C3E876
:10E2A000E21F002AF7D10C4E34686CB1094F043CD0
:10E2B00023682BB12A78002A0CBF384600209847E3
:10E2C00064680CB1043CF3E70023C6E90033F8BDF1
:10E2D000CC000020355700204439002005490B6848
:10E2E00033B1C26800200860117801B9501C18478A
:10E2F000704700BF4039002070B504460A4B1D68C6
:10E3000025B90A4D0A4EB54207D370BD2B6813B12B
:10E310002046217B9847AD69F2E72B6813B1204670
:10E32000217B98471C35EEE77C390020480907001F
:10E330006409070080B500AF88B06A46074B4FF408
:10E34000C4515361064B07489361032342F8103FC1
:10E350004DF0DAFE0020BD4680BD00BF65F007002D
:10E3600033F30700A40907002DE9F04104464FF0FC
:10E370000008144F4FF02002EFF3118382F312884C
:10E38000BFF36F8F216A29B983F31188BFF36F8FB1
:10E39000BDE8F081606A0A68814208BF6262226259
:10E3A00083F31188BFF36F8FD1E901563846C1E975
:10E3B0000188C1F80C805DF038FE0022314620460D
:10E3C000A847D7E778140020002270B50446D1E9A9
:10E3D0000156CA60C1E9012205485DF026FE3146BA
:10E3E00020462B46BDE870406FF06D02184700BF15
:10E3F000781400202DE9F04704460E4692469946CF
:10E400008D6900AF4FF0FF334FF0FF32464838F0D0
:10E41000B3F9637B072B7AD14FF02003EFF311821E
:10E4200083F31288BFF36F8F002D50D000232B6031
:10E43000A369002B48D1C4E9055582F31188BFF3C5
:10E440006F8F042106F10C004FF0FCFB23880AF0CB
:10E45000FD0A43EA0A3AA0F800A0338A043B43804D
:10E46000022330463376FEF737F9002859D0EA46C2
:10E4700088B06A462D4B4FF4015153612C4BC2E9D1
:10E48000063004232B4842F8103F4DF03DFED546A0
:10E490004FF02003EFF3118A83F31288BFF36F8FDD
:10E4A00015B3294604F114004DF008FE8AF31188D3
:10E4B000BFF36F8F1C4838F039F9002329462046F6
:10E4C000B361FFF781FF1BE01D60A561B5E7A3699C
:10E4D00033B103F10C08DB680133C8F80030ACE756
:10E4E000E36904F11C08F7E7D8F80030013BC8F8ED
:10E4F00000308AF31188BFF36F8F0B4838F016F99C
:10E50000B9F1000F09D10020BD46BDE8F0870648EB
:10E5100038F00CF9002DD0D1F2E7304604F0ECFED3
:10E52000F1E70120F0E700BF00010020EBE3070066
:10E5300060F30700A40907000048704700010020AD
:10E5400038B5002204468A4202D10024204638BD54
:10E55000012004F1BC03D3E8EF5F002D04D1C3E830
:10E56000EC0FBCF1000FF6D102D0C0340244EAE750
:10E57000002CEAD0BC22002120463AF0AFF804F18A
:10E58000580004495DF056FE034904F128005DF08F
:10E59000FDFDDBE7D1ED00000FC105002DE9F041E5
:10E5A000164600AF04460D46FFF7DEFE012E38D0BA
:10E5B000022E7BD1236993B16E4688B06A46484BE0
:10E5C00048485361484B4FF4C2519361032342F8CA
:10E5D000103F4DF099FD2046B5464DF09BFD25615D
:10E5E0002169088A012837D9CB681B8804339BB27C
:10E5F000984231D36DD96D468AB06A4613620523BD
:10E600003A4951613849C2E906104FF42151354861
:10E6100042F8103F4DF078FD2046AD464DF07AFDB2
:10E620001AE0206998B96E4688B06A46304B4FF4BC
:10E63000C25153612C4B2B489361032342F8103F86
:10E640004DF062FDB54620464DF064FD01E02E8A96
:10E650002EB9284604F050FEBD46BDE8F0810C30CE
:10E660004FF01DFB864217D96E4688B06A46214B93
:10E670004FF4C25153611C4B1A489361032342F873
:10E68000103F4DF041FD0022B5462046216900F0C3
:10E6900037FE00232361DCE720692A8AE9680C3011
:10E6A0004FF0BFFA284604F027FE99E7E84688B005
:10E6B0006B46114A4FF401515A610B4A0948C3E9AC
:10E6C00006261A46042342F8103F4DF01DFDC546AC
:10E6D000B9E7002301222046236100F011FEBBE7C9
:10E6E00092F00700A40907007AF3070022F107005F
:10E6F000B3F00700D5F0070000F107002DE9F8435B
:10E700009946437B0546072B8846164600AF12D034
:10E710006C4688B06A46314B4FF4C2515361304B5E
:10E7200030489361032342F8103F4DF0EDFCA546BD
:10E730006FF07F0023E0002A4DD038F0B5FD2A4B62
:10E7400083422A4807BF002200234FF0FF324FF0D8
:10E75000FF3337F0B7FF0446A0B96C4688B06A466D
:10E76000234B204853611E4B4FF4C2519361032346
:10E7700042F8103F4DF0C8FC6FF06800A546BD465A
:10E78000BDE8F8836B7B072B18D06D4688B06A46CE
:10E79000184B4FF4C4515361114B1248936103233A
:10E7A00042F8103F4DF0B0FC0023AD462146C4E9CD
:10E7B00001330E48E3605DF038FCB9E70023C0E99F
:10E7C0000169C36005F138004146C8F818404FF0B0
:10E7D000CFF90020D3E71446F4E700BF41F107006A
:10E7E0006AF30700A409070008320020781400200B
:10E7F00054F1070076F1070070B5044617485EF043
:10E8000093F8002201212046144B5EF070F804F1C9
:10E810001406134BD3E8AF2F0AB9012070BDA3F142
:10E82000BC0513F8AF3C53B96FF04001281D4DF003
:10E8300060FC430603D528464DF075FCEDE76B7B85
:10E84000072BEAD13046074B002204215EF04FF837
:10E850000123022084F82030E0E700BF440B0020B1
:10E86000FC280020782800200246012101484DF0B4
:10E87000A5BC00BF40280020F8B5467B04468E4268
:10E880000D4600AF1BD1082E98BF6E4B6C468AB068
:10E8900094BF53F826306C4B6A466C4951616C4901
:10E8A000C2E9061340F201334FF412511384694B4D
:10E8B00042F8103F68484DF027FCA54643E04173FD
:10E8C00026B98378082B01D04DF050FC637B082BD0
:10E8D00000F2B280DFE803F0390537373737371CED
:10E8E000370000265D4D4FF02002EFF3118382F3D5
:10E8F0001288BFF36F8FE269002A79D0013AE26192
:10E9000083F31188BFF36F8F284637F00FFFEAE7D4
:10E91000A378042B17D004F138005DF059FB0021D7
:10E920004F4839F03FF80023C4E91433E378012B52
:10E9300009D103234FF4203284F8AC3004F158009D
:10E94000002338F07BF9BD46F8BDA378042B03D132
:10E9500020464DF01FFCF6E7082EF4D801A353F82B
:10E9600026F000BFD5E9000089E90000C7E90000F2
:10E9700051E9000051E90000C7E90000C7E90000C3
:10E9800047E90000D5E900002046FFF7EDFCA37839
:10E99000012B0AD104F1580528465DF057FC10F010
:10E9A0000C0F02D028465DF053FC0434D4E8EF3F4E
:10E9B00043F04003C4E8E23F002AF7D10021284891
:10E9C00038F0F0FFBFE7237B002BC1D02046FFF7D4
:10E9D00093FCBDE76C4688B06A46224B53611C4BE2
:10E9E0004FF40251C2E90635042342F8103F61E7B3
:10E9F000616921B983F31188BFF36F8FA3E7A06921
:10EA00000A68814208BFA261626183F31188BFF383
:10EA10006F8F4FF02002EFF3118382F31288BFF360
:10EA20006F8FCA68E261CE6083F31188BFF36F8F86
:10EA30002046FFF7C9FC67E76C4688B06A460A4B78
:10EA4000CCE700BF84160700A0F10700AAF1070079
:10EA50004EF3070004000001A40907000001002094
:10EA6000440B0020BFF10700DAF10700034BC01A86
:10EA7000034B80115843C0B2704700BF40280020AC
:10EA8000ABAAAAAA38B50D460849002808BF08460F
:10EA90004FF030F8044618B9BDE83840FFF74ABCDB
:10EAA000691D0C304FF033F8204638BDBC140020EF
:10EAB000F8B504460430D0E8AF3F9B0511D5B4F853
:10EAC0009E30B4F8A0209A420BD8B4F8A2209A4203
:10EAD00007D3D4E929239A4203D16FF400714DF092
:10EAE00008FB104B1D6825B90F4D104FBD420CD3CC
:10EAF000F8BDEE683EB12046B4F8A630B4F8A420C4
:10EB0000B4F89E10B047AD69EDE7EE683EB120461F
:10EB1000B4F8A630B4F8A420B4F89E10B0471C3561
:10EB2000E4E700BF7C3900204809070064090700BA
:10EB30002DE9F041074608460C464DF052F80546CF
:10EB400018B900252846BDE8F081134B1E6846B968
:10EB5000124EDFF84C804645F4D2B36883B91C36B8
:10EB6000F9E7B3680BB9B669F1E72146384698472B
:10EB70000028E6D020464DF034F80028F3D1E0E735
:10EB80002146384698470028DBD020464DF029F82A
:10EB90000028E4D1D5E700BF7C39002048090700F0
:10EBA000640907002DE9F041C378044673B900F108
:10EBB0009606104B04F188071D6855B90E4D0F4F8E
:10EBC00004F18808BD420CD3BDE8F08100F18F0646
:10EBD000EFE72B691BB13A46314620469847AD69AD
:10EBE000EBE72B691BB142463146204698471C355E
:10EBF000E8E700BF7C3900204809070064090700E6
:10EC0000F8B5437A0446837216464DF0E7FB0C4B89
:10EC10001D6825B90B4D0C4FBD4208D3F8BD6B697B
:10EC20001BB132462046617A9847AD69F1E76B69BE
:10EC30001BB132462046617A98471C35ECE700BF8D
:10EC40007C390020480907006409070038B50546EB
:10EC50000C460B480121FFF773FC80B10572236855
:10EC6000C0F88830A388A0F88C30A37980F88E3063
:10EC70000123437283728370024BC0F8A03038BD09
:10EC8000402800201800280070B505460A480E46A6
:10EC90004DF06CFA044620B18378012B04D04DF07E
:10ECA00079FA0024204670BD324629464DF0FFFA1D
:10ECB0000028F7D12046F2E740280020B0B500AF89
:10ECC000FFF7E2FF0446F8B1437B6D46082B98BF7F
:10ECD0000E4A8AB094BF52F823300D4B6A460D4954
:10ECE0000D4851610D49C2E9061340F20133138406
:10ECF0000B4B4FF4125142F8103F4DF005FA2046ED
:10ED0000AD464DF047FA0120BD46B0BD8416070060
:10ED1000A0F10700FAF10700A409070021F307009A
:10ED200004000001F8B505460E480E4617464DF0A2
:10ED30001DFA044620B18378012B03D04DF02AFA46
:10ED400000240DE036B1324629464DF0B0FA08B93C
:10ED50002046F3E7637BBB42FAD1237AAB42F7D17B
:10ED60002046F8BD4028002038B5044608460D4628
:10ED70004CF037FF38B3154B93F8D030990707D4D0
:10ED8000E37873B129462046BDE8384000F0FABA6E
:10ED900094F8AD309A07F3D5231DD3E8AF3F5B0558
:10EDA000EED4294620464DF0A4FA58B92B88A4F891
:10EDB000A0306B88A4F8A230AB88A4F8A830EB8808
:10EDC000A4F8AA3038BD6FF01500FBE70000002062
:10EDD0002DE9F04182B010F84B3C044600AFA0F1A1
:10EDE00058060BBB30464DF0E1FA364B1D685DB955
:10EDF000354DDFF8D88045450ED330464DF0CAF981
:10EE00000837BD46BDE8F0816B681BB1304614F889
:10EE10004C1C9847AD69EAE76B681BB1304614F8A3
:10EE20004C1C98471C35E6E710F8563C012BE7D1FF
:10EE3000A0F154056FF4007128464DF05AF9810590
:10EE400028D5A36C39463B60236D30467B60FFF7C5
:10EE50008BFF68B96FF4807128464DF04AF9D5E808
:10EE6000EF3F43F08003C5E8E23F002AC8D0F6E751
:10EE70006C4688B06A46164B5361164B4FF40251EC
:10EE8000C2E906300423144842F8103F4DF03CF923
:10EE9000A546E4E74FF42813104A39463046C7E93F
:10EEA0000023FFF761FF40B9D5E8EF3F43F48073DB
:10EEB000C5E8E23F002AD2D0F6E76C4688B06A4641
:10EEC000074BD9E77C39002048090700640907008F
:10EED00021F2070086F30700A409070018002800A4
:10EEE0004AF2070001460148FFF7CCBD9815002003
:10EEF0002DE9F04106464FF0FF334FF0FF3200207E
:10EF00000C46FFF7EFFF737B0546072B4FF000061B
:10EF100005D004F0F1F935462846BDE8F081866158
:10EF200000F10C070C4E3846B6F8FC804EF0B7FEE8
:10EF300080450CD2B6F8FC6054F80C1F32463846B7
:10EF40004EF06FFE314620464EF08DFEE4E7384627
:10EF50004EF0A5FE86B2EFE70000002070B5437BBF
:10EF600004465BB96FF0400104304DF0C2F843062F
:10EF700004D52046BDE870404DF0D5B800220023EE
:10EF800004F138004EF0BBFD054660B940F21A337B
:10EF9000224A234923484AF00AFA404080F3118864
:10EFA0004FF0030002DF204E2A8AB6F8FC309A4266
:10EFB00007D80023022229462046FFF71BFA68B92A
:10EFC00005E029462046FFF793FF014638B90023A4
:10EFD000AE692846AB6104F08FF9CEB970BD01234C
:10EFE00000222046FFF706FA0028F0D02A8AB6F859
:10EFF000FC309A4202D800230322DCE7294620464F
:10F00000FFF776FF01460028E1D001231A46E8E722
:10F0100031462046BDE87040FFF7D6B978F20700C8
:10F02000A300080036E10700000000200B4B58B198
:10F030001A6862B902693AB902685AB942684AB9AB
:10F0400082683AB942692AB91860002070476FF0A7
:10F05000770070476FF01500704700BF88390020B7
:10F0600068B10023C360074B00F10C02596819B95D
:10F07000C3E90022002070470A605A60FAE76FF087
:10F08000150070478039002010B902484DF06EB865
:10F09000002070474028002010B50C485CF098FF15
:10F0A0000B490A485CF0C1FF0A4908485CF0BDFF03
:10F0B000094906485CF0B9FF01F0F6F803F0FEFEDE
:10F0C000044608B94DF0D5F9204610BD781400204B
:10F0D0004C3900205C3900206C39002080B500AF2D
:10F0E00088B06A46074B4FF401515361064BC2E9A1
:10F0F00006300423054842F8103F4DF023F9002064
:10F10000BD4680BD94F3070027F50700EC09070012
:10F1100080B500AF88B06A46084B4FF40151536187
:10F12000074BC2E906300423064842F8103F4DF071
:10F1300009F96FF00B00BD4680BD00BFC0F30700AA
:10F140001AF50700EC090700044B1A680AB1FFF72B
:10F15000DFBF0348586010460B6070478C390020B1
:10F16000C8160700F7B5044600261F4D1F4FBD42C5
:10F1700001D303B0F0BD20466B6801A99847002871
:10F180002CDB019B2A889A829A84A86803F11002DA
:10F19000D2E8EF1FC2E8EC6FBCF1000FF8D19E601F
:10F1A000616D03F10802D9B9C4E914221C60D8606A
:10F1B000019843681B6803B19847019B1033D3E85B
:10F1C000EF1F41F00101C3E8E21F002AF7D10198C7
:10F1D0004368DB6913B100F1100198470C35C6E7AD
:10F1E0000A606265E2E700BF2409070048090700DA
:10F1F000F0B583B00B8A0646032B0D4602AF0CD840
:10F200006C4688B002AA364B5361364B9361032398
:10F210004FF4C25142F8103F17E0042105F10C00F1
:10F220004EF029FD298A43880446994215D06C4640
:10F230008AB002AA2C48136250612A480523C2E909
:10F2400006014FF4215142F8103F28484DF07AF85A
:10F25000A54600200437BD46F0BD437823B96C466F
:10F2600088B002AA224BCFE70378012BF1D0132BF1
:10F2700008D10129EDD86C4688B002AA1D4B536114
:10F280001D4BC3E76D4688B002AA1C49174851615F
:10F290001449C2E9061304234FF4025142F8103F07
:10F2A0004DF050F80222AD466178012035684DF0EE
:10F2B0004CF804460028CCD002210C304EF0ABFCB8
:10F2C00000232246037043700521284600934DF029
:10F2D000A5F80028BDD0204604F00EF8B9E700BF1D
:10F2E000EBF307000FF507000DF40700EC0907002A
:10F2F00032F4070057F40700FDF4070077F4070025
:10F30000B0B50B8A0546032B0C4600AF14D86D46EA
:10F3100088B06A46174B4FF4C2515361164B936144
:10F32000032342F8103F15484DF00CF8AD46204637
:10F3300003F0E2FFBD46B0BD042104F10C004EF025
:10F340009AFC418828464DF08BF868B96D4688B024
:10F350006A460B4B5361084BC2E9063104234FF454
:10F36000025142F8103FDEE7436821465B69984747
:10F37000DDE700BFA3F407003FF50700EC09070035
:10F38000C4F4070073B5174B0E46197805460131D2
:10F39000C9B2012938BF01210822122019704CF08E
:10F3A000D4FF0446D0B108210C304EF034FC338831
:10F3B00022460380738805214380B3888380F388C5
:10F3C000C3800023284600934DF028F8054610B16D
:10F3D000204603F091FF284602B070BD6FF00B0588
:10F3E000F9E700BF7557002023281FD81A2804D832
:10F3F000431E182B0ED906207047A0F11B03082BC3
:10F400001ED8DFE803F0051D1B231D19251D05006F
:10F410000320704701230F4A83401A40C2B90E4AA5
:10F420001A40002A14BF01200620704700F07F0315
:10F43000522B05D1002070470120704705207047EE
:10F4400010F0400F0CBF06200020704704207047CA
:10F4500002207047AAAA8A025455450107B504380C
:10F46000019001A902485CF0F3FC03B05DF804FBD5
:10F47000C011002010B504460021142239F02EF9E5
:10F480002146BDE8104001485CF0CFBD601400206B
:10F490002DE9F04F93B0D2F800A002AFDAF80430B3
:10F4A00000257B6042F6010380460E46006887F81F
:10F4B0002C50FB8507F12C0114464CF075FA0028FE
:10F4C00072D04FF42053D8F8000087F82C50FB85F9
:10F4D00007F12C014CF068FA38B1A3681BB15A88C7
:10F4E000B24200D25E80012009E0616808464CF01B
:10F4F000CBFFBAF82A301B1A032B04D8002044375C
:10F50000BD46BDE8F08F08464EF038FB0546606802
:10F510004CF0BAFFBAF82AB005F10C09ABEB000BBE
:10F5200048464EF0BCFB584541D960684CF0ACFFF2
:10F53000BAF82A30181A70B96368987A03F01AFE7C
:10F54000002200234EF0D6FA05460028D6D0014608
:10F5500060684EF024FB002300934146D8F804A0D5
:10F560001023786807F10802D047B0F100081BDBD0
:10F57000227CE068424543D0014607F12C004CF064
:10F5800041FAC0B96D4688B0237C02AA1F49516177
:10F590001F49C2E9061304234FF402511D4842F8E3
:10F5A000103F4DF060F8AD460023A3609BE748464E
:10F5B0004EF075FBBFE75FFA88F207F1080107F12B
:10F5C00018004CF01FFA40B96D4688B002AA124BE1
:10F5D00053610F4BC2E90638DDE707F1180107F167
:10F5E0002C004CF0E1F90028DED1002304216374E3
:10F5F00005F10C004EF00FFBA0600680A36871E7D8
:10F6000007F1080138F0A6FFEDE700BF4DF5070050
:10F6100072F707009C09070070F507002DE9F04715
:10F6200082B006460C46D1F81890CB6802AF022192
:10F6300090304CF043FF00284AD01B78D22B20D1C9
:10F640003368214618684EF0F3F80546C8B16E4697
:10F6500088B002AA204B4FF4C25153611F4B20487F
:10F660009361032342F8103F4CF0FDFFB546A069BB
:10F67000FFF700FF204603F03FFE2846BD46BDE8E9
:10F68000F08704F10C004EF006FBB4F810A0C9F8A6
:10F690000060336880461D68E36804211878FFF72E
:10F6A000A3FE052898BF0F4B224694BF53F8203085
:10F6B0000D4B2846CDF800904CF0B0FE05460028D2
:10F6C000DBD06369A4F810A013FA88F3E360D4E7F1
:10F6D0006FF01505D1E700BF93F507009AF7070013
:10F6E0009C090700F01607004BCA050098B5437B3C
:10F6F00000AF072B12D06C4688B06A46114B4FF40E
:10F70000C4515361104B9361032342F8103F0F48DB
:10F710004CF0A9FF0020A546BD4698BD04214CF041
:10F720009FFE60B96C4688B06A46094B4FF4C251DF
:10F730005361054B9361032342F8103FE7E750F80C
:10F74000040CE9E7AAF50700BFF707009C090700CA
:10F75000BCF5070010B5044600F18C03D3E8EF1F99
:10F7600041F00401C3E8E21F002AF7D11723201F4C
:10F77000E384E3824CF0E4FE04F1AC0003495CF066
:10F7800059FD2068BDE8104001F0DABDC504010054
:10F790002DE9FF414FF000084FF4205305460E4677
:10F7A000006802A9144617688DF80880ADF80A3081
:10F7B0004CF0FAF8A0B142F60103286803A98DF8CD
:10F7C0000C80ADF80E304CF0EFF848B123691BB156
:10F7D0005A88B24200D25E80012004B0BDE8F081B8
:10F7E000616828684CF0E0F810B100232361F3E76A
:10F7F000E368A0681A7832B17B8D018A5B1A934264
:10F8000001DA0020E9E704210C304EF004FA20610F
:10F810000680236929465E80074B01940093384691
:10F820000023A2684CF063FF0028EADB206900385F
:10F8300018BF0120D1E700BFA7C505002DE9F74398
:10F840001768054688460068516814467E684CF083
:10F85000ABF8814600283CD13046952229464DF030
:10F8600099FC0646207540B1E3681B780BB184F81B
:10F870001490002003B0BDE8F083A0684EF07EF93C
:10F8800002210C304EF0C7F9134B2061A0F8008024
:10F8900000930194334629463846A2684CF027FF6E
:10F8A000002807DA10F1FF0F32BF0E204042C0B22D
:10F8B0002075DEE72369002BDBD0A0684CF0E4FD67
:10F8C0007B8D181AE3681B78984294BF00200120B2
:10F8D000D0E70120CEE700BF99C405002DE9F04133
:10F8E00082B000AF04460E460022002339463C4851
:10F8F00036F00AFD0546B8B16D4688B06A46394B08
:10F900004FF401515361384B3848C2E9063404239F
:10F9100042F8103F4CF0A7FEAD466FF00B052846AD
:10F920000837BD46BDE8F08137F0BEFC304BD7F854
:10F93000008029461860282208F1040038F0CEFE25
:10F94000C8F800403C680022C4E90155C4E90955E3
:10F9500000232848391D7D6036F0D6FC054690B15D
:10F9600023686C4688B06A46234920485161234980
:10F97000C2E9061304234FF4025142F8103F4CF041
:10F9800072FEA546C9E77B680146E822184638F0B2
:10F99000A5FE1B4A826098305CF01AFB7B689033AE
:10F9A000D3E8EF2FC3E8E15F0029F9D17B681C6041
:10F9B000636AD7F804801BB904F10C005CF008FB03
:10F9C000626A08F1E003C8F8E020A26A636202B943
:10F9D000A3627B68002BA0D0043333609FE700BF95
:10F9E000A4110020DBF50700B1F707009C09070010
:10F9F000543A0020C011002004F60700A4F70700C5
:10FA0000540B00202DE9B0430D46418D531C8B4211
:10FA100000AF16D96C468AB06A462E481362506110
:10FA20002D480523C2E906014FF4225142F8103F48
:10FA30002A484CF018FEA54600242046BD46BDE8E5
:10FA4000B0832846FFF7D0FC02281BD0042819D029
:10FA50004FF0FF384FF0FF39002142464B46084631
:10FA60004CF0D9FC044690B96C4688B06A461C4BF1
:10FA70004FF401515361184BC2E90635042342F893
:10FA8000103FD5E74FF470284FF00009E4E7154820
:10FA900042464B4636F016FE98B96D4688B06A4627
:10FAA000114B4FF4C45153610B4B0C48936103232A
:10FAB00042F8103F4CF0D7FD2046AD4603F01CFC49
:10FAC000BAE7A061012104F10C004EF0A4F8057022
:10FAD000B3E700BF2DF60700D9F707009C09070020
:10FAE00094F307006014002056F607002DE9F84F44
:10FAF0000B8A0546894600AF9BB96C4688B06A46BA
:10FB0000524B4FF4C2515361514B9361032342F85E
:10FB1000103F50484CF0A7FDA5460020BD46BDE86B
:10FB2000F88F012109F10C004EF0A5F855F8043CBE
:10FB30000446002BF1D000230178DFF81CB12E1F02
:10FB40001BF833004FEAC30A88420BEBC30218D1FB
:10FB500092F80280B8F1010F37D1002105F18C0035
:10FB60004CF06BFE00283ED06C4688B06A463B4B9A
:10FB70005361374B4FF4C4519361032342F8103F54
:10FB8000C7E701330E2BDBD16D4688B06A46344B94
:10FB9000304853612E4BC2E9063104234FF4025121
:10FBA00042F8103F4CF05FFD2178AD460846FFF764
:10FBB0001BFC0028B1D00528AFD00029ADD006230A
:10FBC000002230464CF0A7FFA7E7B8F1050F0AD195
:10FBD000012105F18C004CF030FE20B16C4688B05C
:10FBE0006A46204BC4E7DA44B9F810309AF801208D
:10FBF0009A4219D9E8468AB06A4621781A481162B1
:10FC0000506113484FF42151C2E9060305231148FE
:10FC100042F8103F4CF027FD9AF80230C546012B00
:10FC20007FF47BAF04230CE0DAF804304946304619
:10FC30009847B8F1010F03467FF46FAF00283FF4F7
:10FC40006CAF217800293FF468AFB9E779F6070077
:10FC50008EF707009C09070008170700B6F6070093
:10FC600098F60700D6F60700F9F60700F0B51E462D
:10FC700003680D460039044618BF012187B0186893
:10FC800017464DF048FB48B9052104F190004CF0AF
:10FC9000D4FD002848D0002007B0F0BD002E45D08C
:10FCA00018220021684638F019FD67BB23683146E9
:10FCB0001B68304600930023ADF812300C9B1C4AA1
:10FCC0000393BDF834308DF80850ADF8103001239F
:10FCD0008DF814306B464CF028FC9DF81430E3B1DD
:10FCE000002FD8D0019B9869FFF7C4FB019803F05F
:10FCF00003FB9DF81430002DCDD032462946204616
:10FD00004CF009FFC7E7002239462046FFF77AFE8C
:10FD100001900028CAD10E20BEE701990029BAD06F
:10FD200020464CF0D6FCB6E71220B5E70120B3E739
:10FD3000C9C40500F8B500AF0E461546FFF7D6FC5E
:10FD4000F0B1436A18461BB150F8E03903B1E03B0B
:10FD50006C1C224618B1418DA1421BD293B96D464D
:10FD600088B06A460F4B4FF4025153610E4B0F4857
:10FD7000C2E90634042342F8103F4CF074FCAD464F
:10FD800000200BE01846D3F8E0304BB1418DE03B4A
:10FD90008A42F7D82A463146FFF734FEBD46F8BD01
:10FDA0001446D8E71CF70700C7F707009C090700AF
:10FDB0002DE9F0410E8A0446043EF6B2022E0846B2
:10FDC0008CB001D0102E6AD104210C304DF053FFBD
:10FDD0000DF1080805884788011D324640464BF062
:10FDE00011FE00285DD0002D3AD00026002F36D01D
:10FDF000BD4235D84FF42053404601A98DF8046028
:10FE0000ADF806304BF0D0FD70BB666814220021BF
:10FE100007A838F063FC012211213046FFF78AFF62
:10FE2000099000283DD001210C30CDE907484DF064
:10FE3000F2FE00230A90394603701B4A0B932846B2
:10FE400007AB4CF072FB0A9B1B781BBB099B9869A4
:10FE5000FFF710FB099803F04FFA0A2301E03D4633
:10FE600001232A4610210EE042F60103404607A96D
:10FE70008DF81C60ADF81E304BF096FD0028C4D004
:10FE800010232A46194620464CF045FE00200CB0AF
:10FE9000BDE8F081204609994CF01BFCF6E70420F0
:10FEA000F5E70E20F3E700BF91F700002DE9F043DE
:10FEB000466804460D4685B0012130464DF02BFAC8
:10FEC00050B9052104F190004CF0B7FC00283BD15B
:10FED000122005B0BDE8F08310220021684638F0FA
:10FEE000FDFB002221213046FFF724FF029068B37A
:10FEF0004FF00108DFF85890009405F10C072B8AA9
:10FF0000012B04D8204602994CF0E3FB1CE0384654
:10FF10004DF0B9FE6B464A46014606468DF80C8008
:10FF20004CF003FB9DF80C30002BE8D0029B986945
:10FF3000FFF7A0FA029803F0DFF9324620212046AD
:10FF40009DF80C304CF0E7FD0020C2E70E20C0E722
:10FF5000A3C805002DE9F043466804460D4685B068
:10FF6000012130464DF0D7F950B9052104F1900038
:10FF70004CF063FC00283BD1122005B0BDE8F083B3
:10FF800010220021684638F0A9FB00220F213046DC
:10FF9000FFF7D0FE029068B34FF00108DFF85890E9
:10FFA000009405F10C072B8A012B04D820460299F6
:10FFB0004CF08FFB1CE038464DF065FE6B464A4620
:10FFC000014606468DF80C804CF0AFFA9DF80C30D7
:10FFD000002BE8D0029B9869FFF74CFA029803F0D7
:10FFE0008BF932460E2120469DF80C304CF093FDE3
:10FFF0000020C2E70E20C0E75DC805002DE9FF41E3
:020000040001F9
:10000000D0F8048004460E464046012117461D469E
:100010004DF081F948B9052104F190004CF00DFC38
:1000200078BB122004B0BDE8F0818DB3102200210E
:10003000684638F053FB002239464046FFF77AFE07
:10004000029038B3BDF828302946ADF804300123BA
:1000500028468DF80C30104A6B4600944CF065FA37
:100060009DF80C307BB1029B9869FFF703FA029868
:1000700003F042F92A46314620469DF80C304CF0F8
:100080004AFD0020CEE7204602994CF022FBF8E71B
:100090000120C7E70E20C5E75DC805002DE9F04146
:1000A0000D8A0446043DEDB2022D08468CB001D005
:1000B000102D50D104210C304DF0DDFD0DF1040860
:1000C00006884788011D2A4640464BF09BFC88B1B4
:1000D0009EB18FB1B74210D31822656800210DEB95
:1000E000020038F0FBFA012209212846FFF722FE20
:1000F000089060B90E2007E03E46012332460821F1
:1001000020464CF008FD00200CB0BDE8F081012134
:100110000C30CDE906484DF07EFD002309900370B8
:100120000A2339468DF82C30304606AB0B4A4CF08A
:10013000FCF99DF82C304BB1089B9869FFF79AF9B0
:10014000089803F0D9F89DF82C30D7E72046089995
:100150004CF0BFFAD7E70420D6E700BF3DF8000017
:100160002DE9F0470F460446062186B007F10C0042
:100170004DF081FD0588B0F802808288D7F80C9098
:10018000C5B10023B8F1000F13D0454512D88DF842
:1001900000308DF804304FF42053684601A9ADF8C3
:1001A0000220ADF806304BF0FFFB064660B10A2393
:1001B00001E0454601232A46062120464CF0ABFCCF
:1001C000002006B0BDE8F087D4F804A00146142250
:1001D00001A83F7C38F082FA324607215046FFF7EB
:1001E000A9FD0290F8B10A2341468DF81530284642
:1001F00001AB0E4ACDE9036901948DF814704CF0FF
:1002000094F99DF815304BB1029B9869FFF732F9CC
:10021000029803F071F89DF81530CCE7204602995A
:100220004CF057FACCE70E20CBE700BF91F400006A
:10023000F0B5CB6804461D885E8885B095B186B15F
:10024000B5420FD8476810220021684638F046FAB8
:10025000002205213846FFF76DFD019058B90E20A8
:1002600007E0354601232A46042120464CF053FC82
:10027000002005B0F0BD6B4631462846094A00947F
:100280004CF053F9029B43B9019B9869FFF7F2F8D0
:10029000019803F031F80A23E5E7204601994CF074
:1002A00018FAE5E7C7C5050038B50B4C0B4D2046DD
:1002B0005BF08EFE294620465BF0B7FE204605F136
:1002C00014015BF0B2FE204605F128015BF0ADFEA3
:1002D000BDE8384000F03CBB60140020183A002014
:1002E000002337B505460C46019336F0DDFF0C4B75
:1002F00001A91B68834204BF00252C462A462346D9
:10030000084836F001F8014640B9019B1C22184606
:1003100038F0E4F90346184603B030BD0023FAE78D
:10032000543A0020DC11002007B5836801904BB1DE
:100330009869FFF79FF8019B986802F0DDFF0022A3
:10034000019B9A60034801A95BF082FD03B05DF850
:1003500004FB00BFDC1100202DE9F04F044683B000
:10036000B03002AF0E4690461D465BF071FFD4F8E8
:100370009400B8B96D4688B002AA1C4B4FF4C45122
:1003800053611B4B1B489361032342F8103F4CF011
:100390006AF9AD4620684CF0ECFA00200437BD46FF
:1003A000BDE8F08F144B4FF00009984202D1C4F819
:1003B0009490EFE7D0F804A0C0F80490D4F894002B
:1003C000D0F818B0FFF7B0FF2068C4F894904CF054
:1003D000D0FABAF1000FE0D02068CDF800B0434663
:1003E000324629460068D047D7E700BF3BF70700F1
:1003F0007FF707009C090700583A00202DE9FF41CC
:1004000050F8046C0446002E56D000F1DC0106F1D1
:1004100024004CF0F7F9271F04F194080022002370
:1004200040464DF06CFB054628BBD4F890302BB10C
:10043000024601460E233846FFF78EFF002344F89C
:10044000043C736A002B37D10396039800220023E3
:100450000C304DF054FB0546A0B903984568C5B96A
:10046000056003A916485BF0F3FC206804B0BDE802
:10047000F04100F0BDBFA869FEF7FCFF284602F07E
:100480003BFFCBE7A869FEF7F5FF284602F034FFF3
:10049000DBE782682B689542436008BF83606E6823
:1004A00036B1AB690E210093002300681A46B047AD
:1004B0002846FFF739FFD0E704B0BDE8F08100BF60
:1004C000A4110020B0B500AF6D4688B004466A465E
:1004D000094B4FF4C2515361084B09489361032300
:1004E00042F8103F4CF0BFF8A4F1AC00AD46FFF766
:1004F00085FFBD46B0BD00BF56F7070066F7070091
:100500009C09070070B50646134D40B12A4615F800
:10051000011C6C1E4BF0CBFE98B120460CE0284627
:100520000E494CF0C6FC40B90C4905F110004CF0E6
:10053000C0FC20B105F10F0070BD681EFCE7002073
:10054000FAE73046217C04F111024BF0B0FE00289E
:10055000F5D004F11000EFE78D3A00206DDF0700C1
:1005600070B50E4C054623780E4683420CD0237B93
:10057000AB4210D131460A484CF09BFC58B10123E4
:100580000C2202FB034007E0601C4CF092FC0028A8
:10059000EDD00023F4E7002070BD00BFEA55002035
:1005A000F755002038B54A1C0C46054668B9104678
:1005B0000D494CF07EFC30B90B4904F10B004CF0B6
:1005C00078FC70B10A3420460CE009784BF06FFEDD
:1005D0000028F8D12846A17A04F10B024BF067FEFF
:1005E000EFE7002038BD00BF6DDF07001FB51946DB
:1005F0004FF428131046064ACDE902230823BDF81C
:10060000182000936B444CF08AFC05B05DF804FBA5
:10061000180028002DE9F04700AF1E463B8C8246AB
:100620008846D1F80C90002B51D1731E012B51D864
:10063000012E4946157818BF1588FFF7B3FF044609
:1006400020BB1DB93046BD46BDE8F0874946FFF7DF
:10065000A9FF044690B96C4688B06A461F4B2048F3
:100660005361204B4FF4C4519361032342F8103F70
:100670004CF0DDFC6FF01000A546E4E70AF18801BC
:1006800001304CF040FC9AF808302370D9F81C3047
:100690008BB92581B9F81430AB4203D049464046A6
:1006A0004CF08DFB002DCDD10F49601C4CF02BFC84
:1006B00025702581C6E72A464146504698470028BE
:1006C000C1DB01380128E4D96FF00D00BBE76FF002
:1006D0000600B8E76FF00C00B5E700BFF7F70700BA
:1006E000BC090700F8F907006DDF0700024608B5EE
:1006F000074901304CF007FC00230C3202F8043C9F
:10070000D2E8EF1FC2E8E03F0028F9D108BD00BFE2
:100710006DDF07002DE9F84300AF81468846164695
:100720001D46FFF71DFF0446E0B91549FFF718FF06
:10073000044690B96C4688B06A46124B4FF4C251D9
:100740005361114B11489361032342F8103F4CF061
:100750006EFCA546BD46BDE8F883414600F8019B06
:100760004CF0D1FB228963891AB92BB926816581A6
:10077000F0E7964238BF26819D42EBD9F7E700BFEC
:100780006DDF070015F807000FFA0700BC09070026
:100790002DE9F84300AF98463B8C0646012B914665
:1007A00044D84344012B454643DCFFF7ABFE0446E7
:1007B000C8B9FFF7A7FE0446A8B96C4688B06A46D8
:1007C0001F4B4FF4C45153611E4B1F4893610323C9
:1007D00042F8103F4CF02BFC6FF01005A546284660
:1007E000BD46BDE8F883B8F1000F12D00023217A8E
:1007F00099F8002021FA03F0C00703D522FA03F08C
:10080000C00719D50133032BF4D102F007021143BD
:10081000217206F18801601C4CF075FB2046337A8A
:10082000002100F80C3B4CF026FCD8E76FF00605E1
:10083000D5E76FF00C05D2E76FF01205CFE700BFE8
:1008400038F8070017FA0700BC0907002DE9F04740
:10085000284B1646826807469A422BD1C568AB8A58
:1008600043B34FF000086C1C05F11509B4F80730CC
:100870009BB12246304614F8011C4BF018FDE0B93C
:10088000214614F8010CFEF7FFF930B1437B072B2A
:1008900008BF4FF001084BF07DFC0A344C45E5D110
:1008A000B8F1000F06D1AB69A5F8148013B1414629
:1008B000384698470120BDE8F08706F1880A51467E
:1008C000307A4BF0CCF978B90B4B9D4202D13046CF
:1008D0004CF0B0FB204609494CF015FB002304F80E
:1008E000013CA4F80730D8E7514620464CF00BFBFA
:1008F000D3E700BF15060100940B00206DDF070051
:1009000010B504461148D0E8EF3F23F00203C0E8D9
:10091000E23F002AF7D1D0E8AF3FDA0704D5002242
:100920000023303836F0BEF920464CF01BFA60B197
:100930002046FFF7E7FD40B1037ADB0705D5BDE8A8
:10094000104000210C304CF096BB10BDB82900209F
:10095000012210B51B4BD3E8EF1F002903D1C3E8D8
:10096000E02F0028F7D12CD1174BD3E8EF1F002937
:1009700003D1C3E8E02F0028F7D108D100201349A4
:10098000134A0B88134CA24215D300B10B800022EE
:10099000114B12491248C3E900225BF04BFC4FF4A3
:1009A000A47200230E48FAF7C1FDBDE810400D49BE
:1009B0000D485BF03FBC5068083203449BB20120F5
:1009C000E1E710BDB03A0020AC3A0020025600200A
:1009D000640907007C090700B43A002091D10500A2
:1009E00010290020690E01008829002003462DE906
:1009F000F04148B1008A38B901244FF0140C114974
:100A0000DFF844E0714501D3BDE8F081D1E900761B
:100A1000BB4204D30CFB0672143A93420ED9344401
:100A2000A2B214460831EDE70CFB0578434507D028
:100A300001356219B54292B2F6D1F2E70025F8E726
:100A40001046E1E7640907007C0907002DE9F74F2C
:100A500099464FF6FF73BDF830500746002D08BF8A
:100A60001D46244B90461B88009183423CD203B024
:100A7000BDE8F08F73682344BB4232D29CB2083683
:100A80001D4B9E42F6D3F2E74046895801934AF047
:100A90008BFF019B90B101340AF1010AA4B2736883
:100AA0005345ECD9009B9C42E1D8BC423168F2D35B
:100AB0000BFB0AF28B18B8F1000FE5D1B9F1000F6A
:100AC0000BD1013D1846ADB221460E9A0D9B9847B9
:100AD000002DCCD00028DED1C9E7DA689145DAD103
:100AE000EFE74FF0000ADAE701244FF0140B034E52
:100AF000C6E700BF025600207C0907006409070012
:100B0000002390B5C9B000AF394607F1700207F174
:100B10001000C7E90033C7E902334AF0B1FB98B9C6
:100B20006C4688B06A461D4B53611D4B4FF4C25151
:100B3000936103231B4842F8103F4CF078FAA54616
:100B400007F59277BD4690BD4FF6FF710120164A1A
:100B500007F110034CF011FB144807F110014AF0A3
:100B600024FC20B96C4688B06A46114BDCE70822A9
:100B70000E4B03F11001187811F8014D013A03F8FA
:100B8000014B0870F7D10B4BD3E8EF1F41F0040184
:100B9000C3E8E21F002AD3D0F6E700BF68F80700D9
:100BA00020FA0700BC0907000DCE0500002900202F
:100BB00085F80700B82900202DE9F04114490646C0
:100BC000A1F1300014461D46BDF818705BF054FBCF
:100BD000104BD3E8AF3F590701D4FFF791FF3046E0
:100BE000FFF790FC50B1037ADA0707D50C30D0E854
:100BF000AF3FDB0702D401214CF03DFA10233A4607
:100C0000069329462046BDE8F041034B4CF087B9D6
:100C100040290020B829002000290020002307B522
:100C20000193FFF7E3FE411C89B20846034A01AB7A
:100C30004CF0A3FA019803B05DF804FBB9CD0500B0
:100C40002DE9F84F15468A469422696800AF06469A
:100C50004CF0A0FA8146A8B16C4688B06A46404B79
:100C60004FF4C45153613F4B3F489361032342F813
:100C7000103F4CF0DCF94FF0FF35A5462846BD4645
:100C8000BDE8F88F0222304669684CF0B7FA90B997
:100C90006C4688B06A46354B4FF4C4515361314BB2
:100CA00031489361032342F8103F4CF0C0F96FF0D4
:100CB0001505A546E2E74FF470200021B5F8148031
:100CC000FFF70EFB08F10208044608B31D21284B6C
:100CD000C0F8148042464174C0F80C9043608561AE
:100CE0003046FFF727F88046A8B96D4688B06A46B7
:100CF000204B1D4853611B4B4FF4C4519361032398
:100D000042F8103F4CF093F92046AD46FFF70CFB3C
:100D10006FF00B05B2E701234A46494608F10C0B78
:100D20004CF043F8022158464CF075FF814629F8F3
:100D300002ABA98A58464CF06EFFAA8A2969484638
:100D4000EFF758FF21463046C4F808804BF0F5FF16
:100D50000546002892D02046FFF7E6FA8EE700BF4E
:100D6000A2F80700E0F90700BC090700BCF807007B
:100D7000DBCD0500EBF8070030B504460D468BB01F
:100D8000364BD3E8AF3F5A0761D510B1437B072BF1
:100D900060D168680590FFF729FE2A68ADF8180051
:100DA0003AB305A902912E49002301910121009136
:100DB0004FF6FF710593FFF749FE059B1BB96FF0D6
:100DC00001000BB030BD6B60059B04A918680023BF
:100DD0008DF8103042F60303ADF812304AF0E4FD0E
:100DE00070B90598C3689B799B0605D46FF0150010
:100DF000E7E70028E8D1E2E74CF078F9ADF8180011
:100E0000BDF818003CB1012301462A462046AB75C7
:100E1000FFF716FFD5E76FF07F0307930223ADF8C6
:100E2000203042F60213ADF8123005ABAC750293D8
:100E30000C4B4FF6FF710193012304AA0093234644
:100E400009958DF81040FFF701FE0798B9E76FF09C
:100E50000A00B6E76FF07F00B3E700BFCC000020C8
:100E600001CE0500ED110100034613B550F8082C22
:100E7000A0F12001019200F13004D4E8EF2F22F01C
:100E80000102C4E8E02F0028F7D10D4A002043F802
:100E90001C2C0C4A23F8080C43F8182C01AA43F820
:100EA000102C042223F8060C23F80C2CFFF764FF07
:100EB00018B9012120464CF0DEF802B010BD00BF89
:100EC000A0170700010901002DE9F04F83B09046FB
:100ED0001468444B826805469A4200AF7CD1D0F832
:100EE0000C9009F1010609F1150AB6F8073003B3B1
:100EF0003246204616F8011C4BF0D9F9C8B14FF420
:100F00009572294620464CF045F940B3032814D188
:100F1000EB4688B06A46344B4FF402515361334B71
:100F20003348C2E90635042342F8103F4CF07FF8FD
:100F3000DD460A36B245D8D14EE0052820460CBF22
:100F40004FF0030B4FF0020B4BF0AFF9834506D97E
:100F500098F804305B45ECD288F804B0E9E74946DC
:100F600028464BF02CFF234B994535D1207A04F1CC
:100F70008801FFF7F5FA00282ED00289438952EA4A
:100F8000030129D0BA80FB802046FDF76FFD1823AE
:100F900019491A4A03FB00135A60194A00B29A60B1
:100FA0003A1D1A61042200EB400001EBC0019A8255
:100FB0002046FFF7E1FE78B16C4688B06A46114BD7
:100FC0004FF4C2515361104B09489361032342F817
:100FD000103F4CF02CF8A54601200C37BD46BDE86B
:100FE000F08F00BF1506010016F90700B7F90700DA
:100FF000BC090700940B0020743A0020A0170700DA
:101000008BD005002EF90700ACF907002DE9F04759
:101010001446894600AF9422616806464CF0BAF83F
:10102000A0B16C4688B06A46314B32485361324BAE
:101030004FF4C4519361032342F8103F4BF0F7FF84
:101040004FF0FF30A546BD46BDE8F087012230468F
:1010500061684CF0D3F890B96C4688B06A46274B6B
:1010600024485361244B4FF4C4519361032342F845
:10107000103F4BF0DCFF6FF01500A546E3E7A289B7
:101080001B2130460232FEF755FE054690B96C46EC
:1010900088B06A461A4B17485361174B4FF4C45136
:1010A0009361032342F8103F4BF0C1FF6FF00B0038
:1010B000A546C8E700F10C0A022150464CF0ABFDF2
:1010C000804628F8029BA18950464CF0A4FDA289D5
:1010D000A1684046EFF78EFDD4E9041228460123AB
:1010E0004BF063FE294630464BF0E9FDABE700BF0D
:1010F000A2F80700BC090700D4F90700BCF80700F4
:101100004FF9070030B504460D468BB0344BD3E899
:10111000AF3F5A075DD510B1437B072B5CD16868A0
:101120000590FFF763FC2A68ADF818003AB305A9EB
:1011300002912C4900230191012100914FF6FF718A
:101140000593FFF783FC059B1BB96FF001000BB003
:1011500030BD6B60059B04A9186800238DF8103022
:1011600042F60303ADF812304AF01EFC70B9059840
:10117000C3689B79DB0605D46FF01500E7E700280C
:10118000E8D1E2E74BF0B2FFADF81800BDF8180067
:101190002CB101462A462046FFF738FFD7E76FF00B
:1011A0007F0342F6021207930123ADF8122005AA2D
:1011B00002920D4AADF82030CDE900324FF6FF71B2
:1011C000234604AA09958DF81040FFF73FFC0798C5
:1011D000BDE76FF00A00BAE76FF07F00B7E700BF26
:1011E000CC00002001CE0500ED1101002DE9F04FEB
:1011F00083B015464B4B826880469A4200AF37D188
:10120000D0F80CA0484B9A451AD10026474CDFF87D
:101210002091494620464BF04CFE78B907222146E2
:1012200014F8010CFDF77EFD38BB2B6921461A69C5
:1012300014F8010C53881288FFF76CFA0C34D6B1FD
:101240000AF101060AF1150BB6F80720AB899A429C
:101250000BD1314616F8010CFDF716FD044620B1FE
:10126000437B072B0CD04AF095FF0A36B345EBD1F0
:101270004FF0010950E00126CBE74AF08BFFDDE794
:10128000DAF8203023B14146984708B92046EAE70A
:101290009422414620464BF07DFF814680B1E946CD
:1012A00088B06A46234B4FF4C4515361224B234804
:1012B0009361032342F8103F4BF0B9FECD46E5E7BA
:1012C000AB89022B15D1B6F807309A0705D4204612
:1012D0004AF060FF0023AB60C7E720462A69A9886F
:1012E000FFF7AEFC034680B92A69937D01339375FD
:1012F000EDE7012BEBD1B6F80730DB07E7D5204649
:101300002A69A988FFF782FE034620467B604AF0DF
:1013100041FF7B68002BDDDA48460C37BD46BDE84F
:10132000F08F00BF15060100940B0020EB55002044
:101330006DDF0700A2F80700EEF90700BC090700FF
:1013400090B583B000AF0446386001204FF6FF71BE
:101350003B46114A38714BF010FF20464AF0A5FF7A
:101360003979884214D220464AF073FF80B16C4626
:1013700088B06A46094B4FF402515361084BC2E9E9
:1013800006300423074842F8103F4BF050FEA546B4
:101390000C37BD4690BD00BFC90E01007CF90700A7
:1013A000C2F90700BC090700F8B505460E46174606
:1013B000064B1C684CB154F8043C043C1BB13A4643
:1013C0003146284698476468F4E7F8BDB43A0020EF
:1013D00007B5009001206B464FF6FF71034A8DF868
:1013E00004004BF0CAFE03B05DF804FBC90E010017
:1013F00070B5044603464FF6FF7101200D4A4BF0CD
:10140000BCFE2046FFF77EF8054688B104F1880649
:101410003146207A4AF023FC20B92846BDE87040C6
:10142000FFF764B93146681CBDE870404BF06BBDF6
:1014300070BD00BF4D08010008B5054B01461846B8
:101440004BF0A7FF043B002814BF1846002008BD3E
:10145000C4290020084B00F5D4701A68074BD0E867
:10146000EF1F994204D1C0E8EC2FBCF1000FF6D178
:10147000D0E8AF0F704700BF88390020C029002096
:1014800008B5FFF7E7FF0346C8B1D0E9001221B95C
:10149000002A0CBF0320022010E032B1836813B988
:1014A000094B1B7833B9042008E00749087828B1B4
:1014B0009B6833B9003A18BF0122500008BD0320D1
:1014C000FCE70120FAE700BF7657002010B50C4B6F
:1014D0001B787BB101F00F04FFF7D2FF094B032803
:1014E0001B780CBF04F00B0444F004042BB144F04F
:1014F000010010BD01F00704EEE704F0FE00F8E77C
:10150000765700207857002080B500AF88B06A4633
:10151000064B4FF4C4515361054B064893610323B6
:1015200042F8103F4BF08DFFBD4680BD3BFA0700EF
:1015300069FE0700FC09070080B500AF88B06A4665
:10154000074B4FF4C2515361064B07489361032385
:1015500042F8103F4BF075FF0020BD4680BD00BF34
:1015600058FA070037000800FC09070080B500AFF3
:1015700088B06A46084B4FF401515361074BC2E9EA
:1015800006300423064842F8103F4BF05AFF6FF034
:101590000B00BD4680BD00BF77FA0700C9FF0700FA
:1015A000FC090700054BD3F8EC200AB1FFF7DEBFBA
:1015B0000348EC33586010460B607047C029002088
:1015C000A418070038B50546EC22002137F086F84C
:1015D000102105F12700FCF713FD044648B9052149
:1015E00028464BF03CFFFCF7D5FD034B1860204626
:1015F00038BD0824FBE700BFBC3A0020B0B5044664
:10160000051D0821284600AF4BF029FF0E4904F1C3
:101610005700FCF7CDFDA0B1082128464BF0E0FEB5
:101620006C4688B06A46094B09485361094B4FF430
:10163000C2519361032342F8103F4BF002FF082090
:10164000A546BD46B0BD00BF37D80500A0FA0700CB
:10165000FC09070085FF0700F8B505460B4600AFFB
:101660000D2104304BF095FE78B3DC68D5F8EC30F2
:10167000022003F188063246197A4CF06DF9C8B998
:101680003046F9F7F9FE6C468AB06A46124B4FF4C1
:1016900011515361114BC2E9063040F201331384FA
:1016A0000F4B104842F8103F4BF0CBFE0820A546E8
:1016B000BD46F8BD224600F12A0304F1100152F89C
:1016C000040B8A4243F8040BF9D1284609214BF058
:1016D000C6FE0020ECE700BFBDFA07004FFF070081
:1016E00004000001FC090700F8B505460B4600AFF1
:1016F0000D2104304BF04DFE78B3DC68D5F8EC30AA
:10170000042003F188063246197A4CF025F9C8B94D
:101710003046F9F7B1FE6C468AB06A46124B4FF478
:1017200011515361114BC2E9063040F20133138469
:101730000F4B104842F8103F4BF083FE0820A5469F
:10174000BD46F8BD224600F11A0304F1100152F81B
:10175000040B8A4243F8040BF9D1284607214BF0C9
:101760007EFE0020ECE700BFBDFA07002CFF07005B
:1017700004000001FC090700F0B583B0047A0546B7
:10178000022C02AF23D844B190F8DC30D0F8D84016
:10179000DC4004F0010444F08004032128464BF0AF
:1017A0006EFE064630B310210C304CF034FA009037
:1017B00019482346006805F1270205F157014CF04E
:1017C00023F90446E0B1304601F096FD12E0032C07
:1017D00014D06D4688B002AA104B4FF401515361EA
:1017E0000F4B1048C2E90634042342F8103F4BF077
:1017F00028FEAD4608200437BD46F0BD0024CCE7E6
:101800000246314628464BF0FFFD281D21464BF08D
:10181000E7FD2046EFE700BFBC3A0020DBFA0700F7
:101820001E000800FC0907002DE9F041044600AF46
:10183000FFF710FE251D06460E2128464BF0A9FD98
:10184000C8B9564B2022196804F1570036F082FEC1
:1018500088B96C4688B06A46514B4FF4C451536105
:10186000504B9361032342F8103F4F484BF0E9FD82
:10187000A546082034E00C2120464BF000FE8046AF
:101880000028F6D040210C304CF0C5F9434B0246FD
:101890001B68014603F1200053F804CB834241F852
:1018A00004CBF9D1203203F1200153F8040B8B4211
:1018B00042F8040BF9D10022414620464BF0A4FD2A
:1018C000237A052B59D8DFE803F0033A0E03585565
:1018D000042120464BF0C3FDFFF74EFF00283DD00A
:1018E000BD46BDE8F0812046D4F8EC80FFF7B2FD9C
:1018F0000421064604F1D800FCF782FB0028B8D189
:10190000D4F8D830294A84F8DC00B3FBF2F102FBAA
:101910001133C4F8D83056B1336843B10B2128468F
:101920004BF09DFD40463368D4F8D810984703210A
:1019300020464BF094FD0E214BF091FD0EE0204629
:1019400003214BF08CFD0E214BF089FD28460A2126
:101950004BF085FD7368D4F8EC00984728460721C2
:101960004BF07DFD0820FFF767FDA0B92046FFF78B
:1019700045FEB5E704212046DEE76C4688B06A469E
:101980000B4951610749C2E9061304234FF4015181
:1019900042F8103F69E70020A2E700BFBC3A0020F0
:1019A000FBFA070098FF0700FC09070040420F0000
:1019B000DBFA0700B0B505460C4600AFFFF74AFD5D
:1019C00005F157000246E36803F1200153F8044B88
:1019D0008B4242F8044BF9D105F1770203F1200163
:1019E00053F8044B8B4242F8044BF9D1FCF726FB29
:1019F00048B91E4B1C68002C34D1281D06214BF021
:101A00002EFD20462CE06C4688B06A46184B4FF4F9
:101A1000C6515361174B18489361032342F8103F96
:101A20004BF00FFD0E21A546281D4BF018FDD5F8F3
:101A3000EC40D4F8B83033B9207A04F1880101F0D1
:101A400053FAC4F8B800D4F8B830002BD1D0DA89F2
:101A500002F02402002ACCD05B7B9B07C9D4032070
:101A6000BD46B0BD2846FFF7DFFEF9E7BC3A0020CF
:101A70001AFB0700AEFF0700FC0907002DE9F04341
:101A800083B00D4600AF0446D0F8EC60FFF7E2FCEF
:101A9000D5F80C90804699F80330073B092B04D900
:101AA00006200C37BD46BDE8F083D6F8B8305BB1F0
:101AB000251D0F2128464BF06CFC80B92046FFF70E
:101AC00081FD60B1C0B2ECE7307A06F1880101F027
:101AD0000BFAC6F8B8000028EAD10820E1E7012394
:101AE0006372D9F800302046C4F80A30B9F80430DF
:101AF000E3810223237499F80210FFF7E7FCE074F6
:101B00002046FFF7BDFCA84B60741B78A37410231C
:101B1000237599F8043003F00303637599F80530D1
:101B200003F00103A375E37C1B070DD599F8023080
:101B3000180709D5052128464BF091FC637D03F079
:101B4000020363750023A375E37C990607D599F812
:101B500002309A0603D5142128464BF080FCA37D61
:101B600084F8E830637D84F8E930E37CDB0707D54F
:101B700099F80230D80703D50D2128464BF06FFCA9
:101B8000032128464BF06BFC052199F800904BF09F
:101B900000FC40BBB9F1040F45D8E37AA27C1340A6
:101BA000D9073ED4217BE37C194311F0040111D005
:101BB0002046FFF765FC7D4B09EB8909994419F82C
:101BC0000010042906D1D4F8EC30DB78002B14BFC8
:101BD0000121022121722046D6F8B8104BF0DFFB1C
:101BE00018BB03205DE7237BE07C03EA00021207B9
:101BF00006D5E27A94F812C042EA0C02D207E9D480
